
T11_L51_RTOS_SimpleProject.elf:     file format elf32-littlearm

Sections:
Idx Name          Size      VMA       LMA       File off  Algn
  0 .isr_vector   00000198  08000000  08000000  00010000  2**0
                  CONTENTS, ALLOC, LOAD, READONLY, DATA
  1 .text         00009a74  080001a0  080001a0  000101a0  2**4
                  CONTENTS, ALLOC, LOAD, READONLY, CODE
  2 .rodata       000003b0  08009c18  08009c18  00019c18  2**3
                  CONTENTS, ALLOC, LOAD, READONLY, DATA
  3 .ARM.extab    00000000  08009fc8  08009fc8  00020014  2**0
                  CONTENTS
  4 .ARM          00000008  08009fc8  08009fc8  00019fc8  2**2
                  CONTENTS, ALLOC, LOAD, READONLY, DATA
  5 .preinit_array 00000000  08009fd0  08009fd0  00020014  2**0
                  CONTENTS, ALLOC, LOAD, DATA
  6 .init_array   00000004  08009fd0  08009fd0  00019fd0  2**2
                  CONTENTS, ALLOC, LOAD, DATA
  7 .fini_array   00000004  08009fd4  08009fd4  00019fd4  2**2
                  CONTENTS, ALLOC, LOAD, DATA
  8 .data         00000014  20000000  08009fd8  00020000  2**2
                  CONTENTS, ALLOC, LOAD, DATA
  9 .bss          00004e64  20000014  08009fec  00020014  2**2
                  ALLOC
 10 ._user_heap_stack 00000600  20004e78  08009fec  00024e78  2**0
                  ALLOC
 11 .ARM.attributes 00000030  00000000  00000000  00020014  2**0
                  CONTENTS, READONLY
 12 .debug_info   0001e613  00000000  00000000  00020044  2**0
                  CONTENTS, READONLY, DEBUGGING
 13 .debug_abbrev 00003bac  00000000  00000000  0003e657  2**0
                  CONTENTS, READONLY, DEBUGGING
 14 .debug_aranges 000017e8  00000000  00000000  00042208  2**3
                  CONTENTS, READONLY, DEBUGGING
 15 .debug_ranges 00001648  00000000  00000000  000439f0  2**3
                  CONTENTS, READONLY, DEBUGGING
 16 .debug_macro  0001990d  00000000  00000000  00045038  2**0
                  CONTENTS, READONLY, DEBUGGING
 17 .debug_line   00014085  00000000  00000000  0005e945  2**0
                  CONTENTS, READONLY, DEBUGGING
 18 .debug_str    00099c65  00000000  00000000  000729ca  2**0
                  CONTENTS, READONLY, DEBUGGING
 19 .comment      0000007b  00000000  00000000  0010c62f  2**0
                  CONTENTS, READONLY
 20 .debug_frame  00006680  00000000  00000000  0010c6ac  2**2
                  CONTENTS, READONLY, DEBUGGING

Disassembly of section .text:

080001a0 <__do_global_dtors_aux>:
 80001a0:	b510      	push	{r4, lr}
 80001a2:	4c05      	ldr	r4, [pc, #20]	; (80001b8 <__do_global_dtors_aux+0x18>)
 80001a4:	7823      	ldrb	r3, [r4, #0]
 80001a6:	b933      	cbnz	r3, 80001b6 <__do_global_dtors_aux+0x16>
 80001a8:	4b04      	ldr	r3, [pc, #16]	; (80001bc <__do_global_dtors_aux+0x1c>)
 80001aa:	b113      	cbz	r3, 80001b2 <__do_global_dtors_aux+0x12>
 80001ac:	4804      	ldr	r0, [pc, #16]	; (80001c0 <__do_global_dtors_aux+0x20>)
 80001ae:	f3af 8000 	nop.w
 80001b2:	2301      	movs	r3, #1
 80001b4:	7023      	strb	r3, [r4, #0]
 80001b6:	bd10      	pop	{r4, pc}
 80001b8:	20000014 	.word	0x20000014
 80001bc:	00000000 	.word	0x00000000
 80001c0:	08009bfc 	.word	0x08009bfc

080001c4 <frame_dummy>:
 80001c4:	b508      	push	{r3, lr}
 80001c6:	4b03      	ldr	r3, [pc, #12]	; (80001d4 <frame_dummy+0x10>)
 80001c8:	b11b      	cbz	r3, 80001d2 <frame_dummy+0xe>
 80001ca:	4903      	ldr	r1, [pc, #12]	; (80001d8 <frame_dummy+0x14>)
 80001cc:	4803      	ldr	r0, [pc, #12]	; (80001dc <frame_dummy+0x18>)
 80001ce:	f3af 8000 	nop.w
 80001d2:	bd08      	pop	{r3, pc}
 80001d4:	00000000 	.word	0x00000000
 80001d8:	20000018 	.word	0x20000018
 80001dc:	08009bfc 	.word	0x08009bfc

080001e0 <__aeabi_drsub>:
 80001e0:	f081 4100 	eor.w	r1, r1, #2147483648	; 0x80000000
 80001e4:	e002      	b.n	80001ec <__adddf3>
 80001e6:	bf00      	nop

080001e8 <__aeabi_dsub>:
 80001e8:	f083 4300 	eor.w	r3, r3, #2147483648	; 0x80000000

080001ec <__adddf3>:
 80001ec:	b530      	push	{r4, r5, lr}
 80001ee:	ea4f 0441 	mov.w	r4, r1, lsl #1
 80001f2:	ea4f 0543 	mov.w	r5, r3, lsl #1
 80001f6:	ea94 0f05 	teq	r4, r5
 80001fa:	bf08      	it	eq
 80001fc:	ea90 0f02 	teqeq	r0, r2
 8000200:	bf1f      	itttt	ne
 8000202:	ea54 0c00 	orrsne.w	ip, r4, r0
 8000206:	ea55 0c02 	orrsne.w	ip, r5, r2
 800020a:	ea7f 5c64 	mvnsne.w	ip, r4, asr #21
 800020e:	ea7f 5c65 	mvnsne.w	ip, r5, asr #21
 8000212:	f000 80e2 	beq.w	80003da <__adddf3+0x1ee>
 8000216:	ea4f 5454 	mov.w	r4, r4, lsr #21
 800021a:	ebd4 5555 	rsbs	r5, r4, r5, lsr #21
 800021e:	bfb8      	it	lt
 8000220:	426d      	neglt	r5, r5
 8000222:	dd0c      	ble.n	800023e <__adddf3+0x52>
 8000224:	442c      	add	r4, r5
 8000226:	ea80 0202 	eor.w	r2, r0, r2
 800022a:	ea81 0303 	eor.w	r3, r1, r3
 800022e:	ea82 0000 	eor.w	r0, r2, r0
 8000232:	ea83 0101 	eor.w	r1, r3, r1
 8000236:	ea80 0202 	eor.w	r2, r0, r2
 800023a:	ea81 0303 	eor.w	r3, r1, r3
 800023e:	2d36      	cmp	r5, #54	; 0x36
 8000240:	bf88      	it	hi
 8000242:	bd30      	pophi	{r4, r5, pc}
 8000244:	f011 4f00 	tst.w	r1, #2147483648	; 0x80000000
 8000248:	ea4f 3101 	mov.w	r1, r1, lsl #12
 800024c:	f44f 1c80 	mov.w	ip, #1048576	; 0x100000
 8000250:	ea4c 3111 	orr.w	r1, ip, r1, lsr #12
 8000254:	d002      	beq.n	800025c <__adddf3+0x70>
 8000256:	4240      	negs	r0, r0
 8000258:	eb61 0141 	sbc.w	r1, r1, r1, lsl #1
 800025c:	f013 4f00 	tst.w	r3, #2147483648	; 0x80000000
 8000260:	ea4f 3303 	mov.w	r3, r3, lsl #12
 8000264:	ea4c 3313 	orr.w	r3, ip, r3, lsr #12
 8000268:	d002      	beq.n	8000270 <__adddf3+0x84>
 800026a:	4252      	negs	r2, r2
 800026c:	eb63 0343 	sbc.w	r3, r3, r3, lsl #1
 8000270:	ea94 0f05 	teq	r4, r5
 8000274:	f000 80a7 	beq.w	80003c6 <__adddf3+0x1da>
 8000278:	f1a4 0401 	sub.w	r4, r4, #1
 800027c:	f1d5 0e20 	rsbs	lr, r5, #32
 8000280:	db0d      	blt.n	800029e <__adddf3+0xb2>
 8000282:	fa02 fc0e 	lsl.w	ip, r2, lr
 8000286:	fa22 f205 	lsr.w	r2, r2, r5
 800028a:	1880      	adds	r0, r0, r2
 800028c:	f141 0100 	adc.w	r1, r1, #0
 8000290:	fa03 f20e 	lsl.w	r2, r3, lr
 8000294:	1880      	adds	r0, r0, r2
 8000296:	fa43 f305 	asr.w	r3, r3, r5
 800029a:	4159      	adcs	r1, r3
 800029c:	e00e      	b.n	80002bc <__adddf3+0xd0>
 800029e:	f1a5 0520 	sub.w	r5, r5, #32
 80002a2:	f10e 0e20 	add.w	lr, lr, #32
 80002a6:	2a01      	cmp	r2, #1
 80002a8:	fa03 fc0e 	lsl.w	ip, r3, lr
 80002ac:	bf28      	it	cs
 80002ae:	f04c 0c02 	orrcs.w	ip, ip, #2
 80002b2:	fa43 f305 	asr.w	r3, r3, r5
 80002b6:	18c0      	adds	r0, r0, r3
 80002b8:	eb51 71e3 	adcs.w	r1, r1, r3, asr #31
 80002bc:	f001 4500 	and.w	r5, r1, #2147483648	; 0x80000000
 80002c0:	d507      	bpl.n	80002d2 <__adddf3+0xe6>
 80002c2:	f04f 0e00 	mov.w	lr, #0
 80002c6:	f1dc 0c00 	rsbs	ip, ip, #0
 80002ca:	eb7e 0000 	sbcs.w	r0, lr, r0
 80002ce:	eb6e 0101 	sbc.w	r1, lr, r1
 80002d2:	f5b1 1f80 	cmp.w	r1, #1048576	; 0x100000
 80002d6:	d31b      	bcc.n	8000310 <__adddf3+0x124>
 80002d8:	f5b1 1f00 	cmp.w	r1, #2097152	; 0x200000
 80002dc:	d30c      	bcc.n	80002f8 <__adddf3+0x10c>
 80002de:	0849      	lsrs	r1, r1, #1
 80002e0:	ea5f 0030 	movs.w	r0, r0, rrx
 80002e4:	ea4f 0c3c 	mov.w	ip, ip, rrx
 80002e8:	f104 0401 	add.w	r4, r4, #1
 80002ec:	ea4f 5244 	mov.w	r2, r4, lsl #21
 80002f0:	f512 0f80 	cmn.w	r2, #4194304	; 0x400000
 80002f4:	f080 809a 	bcs.w	800042c <__adddf3+0x240>
 80002f8:	f1bc 4f00 	cmp.w	ip, #2147483648	; 0x80000000
 80002fc:	bf08      	it	eq
 80002fe:	ea5f 0c50 	movseq.w	ip, r0, lsr #1
 8000302:	f150 0000 	adcs.w	r0, r0, #0
 8000306:	eb41 5104 	adc.w	r1, r1, r4, lsl #20
 800030a:	ea41 0105 	orr.w	r1, r1, r5
 800030e:	bd30      	pop	{r4, r5, pc}
 8000310:	ea5f 0c4c 	movs.w	ip, ip, lsl #1
 8000314:	4140      	adcs	r0, r0
 8000316:	eb41 0101 	adc.w	r1, r1, r1
 800031a:	f411 1f80 	tst.w	r1, #1048576	; 0x100000
 800031e:	f1a4 0401 	sub.w	r4, r4, #1
 8000322:	d1e9      	bne.n	80002f8 <__adddf3+0x10c>
 8000324:	f091 0f00 	teq	r1, #0
 8000328:	bf04      	itt	eq
 800032a:	4601      	moveq	r1, r0
 800032c:	2000      	moveq	r0, #0
 800032e:	fab1 f381 	clz	r3, r1
 8000332:	bf08      	it	eq
 8000334:	3320      	addeq	r3, #32
 8000336:	f1a3 030b 	sub.w	r3, r3, #11
 800033a:	f1b3 0220 	subs.w	r2, r3, #32
 800033e:	da0c      	bge.n	800035a <__adddf3+0x16e>
 8000340:	320c      	adds	r2, #12
 8000342:	dd08      	ble.n	8000356 <__adddf3+0x16a>
 8000344:	f102 0c14 	add.w	ip, r2, #20
 8000348:	f1c2 020c 	rsb	r2, r2, #12
 800034c:	fa01 f00c 	lsl.w	r0, r1, ip
 8000350:	fa21 f102 	lsr.w	r1, r1, r2
 8000354:	e00c      	b.n	8000370 <__adddf3+0x184>
 8000356:	f102 0214 	add.w	r2, r2, #20
 800035a:	bfd8      	it	le
 800035c:	f1c2 0c20 	rsble	ip, r2, #32
 8000360:	fa01 f102 	lsl.w	r1, r1, r2
 8000364:	fa20 fc0c 	lsr.w	ip, r0, ip
 8000368:	bfdc      	itt	le
 800036a:	ea41 010c 	orrle.w	r1, r1, ip
 800036e:	4090      	lslle	r0, r2
 8000370:	1ae4      	subs	r4, r4, r3
 8000372:	bfa2      	ittt	ge
 8000374:	eb01 5104 	addge.w	r1, r1, r4, lsl #20
 8000378:	4329      	orrge	r1, r5
 800037a:	bd30      	popge	{r4, r5, pc}
 800037c:	ea6f 0404 	mvn.w	r4, r4
 8000380:	3c1f      	subs	r4, #31
 8000382:	da1c      	bge.n	80003be <__adddf3+0x1d2>
 8000384:	340c      	adds	r4, #12
 8000386:	dc0e      	bgt.n	80003a6 <__adddf3+0x1ba>
 8000388:	f104 0414 	add.w	r4, r4, #20
 800038c:	f1c4 0220 	rsb	r2, r4, #32
 8000390:	fa20 f004 	lsr.w	r0, r0, r4
 8000394:	fa01 f302 	lsl.w	r3, r1, r2
 8000398:	ea40 0003 	orr.w	r0, r0, r3
 800039c:	fa21 f304 	lsr.w	r3, r1, r4
 80003a0:	ea45 0103 	orr.w	r1, r5, r3
 80003a4:	bd30      	pop	{r4, r5, pc}
 80003a6:	f1c4 040c 	rsb	r4, r4, #12
 80003aa:	f1c4 0220 	rsb	r2, r4, #32
 80003ae:	fa20 f002 	lsr.w	r0, r0, r2
 80003b2:	fa01 f304 	lsl.w	r3, r1, r4
 80003b6:	ea40 0003 	orr.w	r0, r0, r3
 80003ba:	4629      	mov	r1, r5
 80003bc:	bd30      	pop	{r4, r5, pc}
 80003be:	fa21 f004 	lsr.w	r0, r1, r4
 80003c2:	4629      	mov	r1, r5
 80003c4:	bd30      	pop	{r4, r5, pc}
 80003c6:	f094 0f00 	teq	r4, #0
 80003ca:	f483 1380 	eor.w	r3, r3, #1048576	; 0x100000
 80003ce:	bf06      	itte	eq
 80003d0:	f481 1180 	eoreq.w	r1, r1, #1048576	; 0x100000
 80003d4:	3401      	addeq	r4, #1
 80003d6:	3d01      	subne	r5, #1
 80003d8:	e74e      	b.n	8000278 <__adddf3+0x8c>
 80003da:	ea7f 5c64 	mvns.w	ip, r4, asr #21
 80003de:	bf18      	it	ne
 80003e0:	ea7f 5c65 	mvnsne.w	ip, r5, asr #21
 80003e4:	d029      	beq.n	800043a <__adddf3+0x24e>
 80003e6:	ea94 0f05 	teq	r4, r5
 80003ea:	bf08      	it	eq
 80003ec:	ea90 0f02 	teqeq	r0, r2
 80003f0:	d005      	beq.n	80003fe <__adddf3+0x212>
 80003f2:	ea54 0c00 	orrs.w	ip, r4, r0
 80003f6:	bf04      	itt	eq
 80003f8:	4619      	moveq	r1, r3
 80003fa:	4610      	moveq	r0, r2
 80003fc:	bd30      	pop	{r4, r5, pc}
 80003fe:	ea91 0f03 	teq	r1, r3
 8000402:	bf1e      	ittt	ne
 8000404:	2100      	movne	r1, #0
 8000406:	2000      	movne	r0, #0
 8000408:	bd30      	popne	{r4, r5, pc}
 800040a:	ea5f 5c54 	movs.w	ip, r4, lsr #21
 800040e:	d105      	bne.n	800041c <__adddf3+0x230>
 8000410:	0040      	lsls	r0, r0, #1
 8000412:	4149      	adcs	r1, r1
 8000414:	bf28      	it	cs
 8000416:	f041 4100 	orrcs.w	r1, r1, #2147483648	; 0x80000000
 800041a:	bd30      	pop	{r4, r5, pc}
 800041c:	f514 0480 	adds.w	r4, r4, #4194304	; 0x400000
 8000420:	bf3c      	itt	cc
 8000422:	f501 1180 	addcc.w	r1, r1, #1048576	; 0x100000
 8000426:	bd30      	popcc	{r4, r5, pc}
 8000428:	f001 4500 	and.w	r5, r1, #2147483648	; 0x80000000
 800042c:	f045 41fe 	orr.w	r1, r5, #2130706432	; 0x7f000000
 8000430:	f441 0170 	orr.w	r1, r1, #15728640	; 0xf00000
 8000434:	f04f 0000 	mov.w	r0, #0
 8000438:	bd30      	pop	{r4, r5, pc}
 800043a:	ea7f 5c64 	mvns.w	ip, r4, asr #21
 800043e:	bf1a      	itte	ne
 8000440:	4619      	movne	r1, r3
 8000442:	4610      	movne	r0, r2
 8000444:	ea7f 5c65 	mvnseq.w	ip, r5, asr #21
 8000448:	bf1c      	itt	ne
 800044a:	460b      	movne	r3, r1
 800044c:	4602      	movne	r2, r0
 800044e:	ea50 3401 	orrs.w	r4, r0, r1, lsl #12
 8000452:	bf06      	itte	eq
 8000454:	ea52 3503 	orrseq.w	r5, r2, r3, lsl #12
 8000458:	ea91 0f03 	teqeq	r1, r3
 800045c:	f441 2100 	orrne.w	r1, r1, #524288	; 0x80000
 8000460:	bd30      	pop	{r4, r5, pc}
 8000462:	bf00      	nop

08000464 <__aeabi_ui2d>:
 8000464:	f090 0f00 	teq	r0, #0
 8000468:	bf04      	itt	eq
 800046a:	2100      	moveq	r1, #0
 800046c:	4770      	bxeq	lr
 800046e:	b530      	push	{r4, r5, lr}
 8000470:	f44f 6480 	mov.w	r4, #1024	; 0x400
 8000474:	f104 0432 	add.w	r4, r4, #50	; 0x32
 8000478:	f04f 0500 	mov.w	r5, #0
 800047c:	f04f 0100 	mov.w	r1, #0
 8000480:	e750      	b.n	8000324 <__adddf3+0x138>
 8000482:	bf00      	nop

08000484 <__aeabi_i2d>:
 8000484:	f090 0f00 	teq	r0, #0
 8000488:	bf04      	itt	eq
 800048a:	2100      	moveq	r1, #0
 800048c:	4770      	bxeq	lr
 800048e:	b530      	push	{r4, r5, lr}
 8000490:	f44f 6480 	mov.w	r4, #1024	; 0x400
 8000494:	f104 0432 	add.w	r4, r4, #50	; 0x32
 8000498:	f010 4500 	ands.w	r5, r0, #2147483648	; 0x80000000
 800049c:	bf48      	it	mi
 800049e:	4240      	negmi	r0, r0
 80004a0:	f04f 0100 	mov.w	r1, #0
 80004a4:	e73e      	b.n	8000324 <__adddf3+0x138>
 80004a6:	bf00      	nop

080004a8 <__aeabi_f2d>:
 80004a8:	0042      	lsls	r2, r0, #1
 80004aa:	ea4f 01e2 	mov.w	r1, r2, asr #3
 80004ae:	ea4f 0131 	mov.w	r1, r1, rrx
 80004b2:	ea4f 7002 	mov.w	r0, r2, lsl #28
 80004b6:	bf1f      	itttt	ne
 80004b8:	f012 437f 	andsne.w	r3, r2, #4278190080	; 0xff000000
 80004bc:	f093 4f7f 	teqne	r3, #4278190080	; 0xff000000
 80004c0:	f081 5160 	eorne.w	r1, r1, #939524096	; 0x38000000
 80004c4:	4770      	bxne	lr
 80004c6:	f032 427f 	bics.w	r2, r2, #4278190080	; 0xff000000
 80004ca:	bf08      	it	eq
 80004cc:	4770      	bxeq	lr
 80004ce:	f093 4f7f 	teq	r3, #4278190080	; 0xff000000
 80004d2:	bf04      	itt	eq
 80004d4:	f441 2100 	orreq.w	r1, r1, #524288	; 0x80000
 80004d8:	4770      	bxeq	lr
 80004da:	b530      	push	{r4, r5, lr}
 80004dc:	f44f 7460 	mov.w	r4, #896	; 0x380
 80004e0:	f001 4500 	and.w	r5, r1, #2147483648	; 0x80000000
 80004e4:	f021 4100 	bic.w	r1, r1, #2147483648	; 0x80000000
 80004e8:	e71c      	b.n	8000324 <__adddf3+0x138>
 80004ea:	bf00      	nop

080004ec <__aeabi_ul2d>:
 80004ec:	ea50 0201 	orrs.w	r2, r0, r1
 80004f0:	bf08      	it	eq
 80004f2:	4770      	bxeq	lr
 80004f4:	b530      	push	{r4, r5, lr}
 80004f6:	f04f 0500 	mov.w	r5, #0
 80004fa:	e00a      	b.n	8000512 <__aeabi_l2d+0x16>

080004fc <__aeabi_l2d>:
 80004fc:	ea50 0201 	orrs.w	r2, r0, r1
 8000500:	bf08      	it	eq
 8000502:	4770      	bxeq	lr
 8000504:	b530      	push	{r4, r5, lr}
 8000506:	f011 4500 	ands.w	r5, r1, #2147483648	; 0x80000000
 800050a:	d502      	bpl.n	8000512 <__aeabi_l2d+0x16>
 800050c:	4240      	negs	r0, r0
 800050e:	eb61 0141 	sbc.w	r1, r1, r1, lsl #1
 8000512:	f44f 6480 	mov.w	r4, #1024	; 0x400
 8000516:	f104 0432 	add.w	r4, r4, #50	; 0x32
 800051a:	ea5f 5c91 	movs.w	ip, r1, lsr #22
 800051e:	f43f aed8 	beq.w	80002d2 <__adddf3+0xe6>
 8000522:	f04f 0203 	mov.w	r2, #3
 8000526:	ea5f 0cdc 	movs.w	ip, ip, lsr #3
 800052a:	bf18      	it	ne
 800052c:	3203      	addne	r2, #3
 800052e:	ea5f 0cdc 	movs.w	ip, ip, lsr #3
 8000532:	bf18      	it	ne
 8000534:	3203      	addne	r2, #3
 8000536:	eb02 02dc 	add.w	r2, r2, ip, lsr #3
 800053a:	f1c2 0320 	rsb	r3, r2, #32
 800053e:	fa00 fc03 	lsl.w	ip, r0, r3
 8000542:	fa20 f002 	lsr.w	r0, r0, r2
 8000546:	fa01 fe03 	lsl.w	lr, r1, r3
 800054a:	ea40 000e 	orr.w	r0, r0, lr
 800054e:	fa21 f102 	lsr.w	r1, r1, r2
 8000552:	4414      	add	r4, r2
 8000554:	e6bd      	b.n	80002d2 <__adddf3+0xe6>
 8000556:	bf00      	nop

08000558 <__aeabi_dmul>:
 8000558:	b570      	push	{r4, r5, r6, lr}
 800055a:	f04f 0cff 	mov.w	ip, #255	; 0xff
 800055e:	f44c 6ce0 	orr.w	ip, ip, #1792	; 0x700
 8000562:	ea1c 5411 	ands.w	r4, ip, r1, lsr #20
 8000566:	bf1d      	ittte	ne
 8000568:	ea1c 5513 	andsne.w	r5, ip, r3, lsr #20
 800056c:	ea94 0f0c 	teqne	r4, ip
 8000570:	ea95 0f0c 	teqne	r5, ip
 8000574:	f000 f8de 	bleq	8000734 <__aeabi_dmul+0x1dc>
 8000578:	442c      	add	r4, r5
 800057a:	ea81 0603 	eor.w	r6, r1, r3
 800057e:	ea21 514c 	bic.w	r1, r1, ip, lsl #21
 8000582:	ea23 534c 	bic.w	r3, r3, ip, lsl #21
 8000586:	ea50 3501 	orrs.w	r5, r0, r1, lsl #12
 800058a:	bf18      	it	ne
 800058c:	ea52 3503 	orrsne.w	r5, r2, r3, lsl #12
 8000590:	f441 1180 	orr.w	r1, r1, #1048576	; 0x100000
 8000594:	f443 1380 	orr.w	r3, r3, #1048576	; 0x100000
 8000598:	d038      	beq.n	800060c <__aeabi_dmul+0xb4>
 800059a:	fba0 ce02 	umull	ip, lr, r0, r2
 800059e:	f04f 0500 	mov.w	r5, #0
 80005a2:	fbe1 e502 	umlal	lr, r5, r1, r2
 80005a6:	f006 4200 	and.w	r2, r6, #2147483648	; 0x80000000
 80005aa:	fbe0 e503 	umlal	lr, r5, r0, r3
 80005ae:	f04f 0600 	mov.w	r6, #0
 80005b2:	fbe1 5603 	umlal	r5, r6, r1, r3
 80005b6:	f09c 0f00 	teq	ip, #0
 80005ba:	bf18      	it	ne
 80005bc:	f04e 0e01 	orrne.w	lr, lr, #1
 80005c0:	f1a4 04ff 	sub.w	r4, r4, #255	; 0xff
 80005c4:	f5b6 7f00 	cmp.w	r6, #512	; 0x200
 80005c8:	f564 7440 	sbc.w	r4, r4, #768	; 0x300
 80005cc:	d204      	bcs.n	80005d8 <__aeabi_dmul+0x80>
 80005ce:	ea5f 0e4e 	movs.w	lr, lr, lsl #1
 80005d2:	416d      	adcs	r5, r5
 80005d4:	eb46 0606 	adc.w	r6, r6, r6
 80005d8:	ea42 21c6 	orr.w	r1, r2, r6, lsl #11
 80005dc:	ea41 5155 	orr.w	r1, r1, r5, lsr #21
 80005e0:	ea4f 20c5 	mov.w	r0, r5, lsl #11
 80005e4:	ea40 505e 	orr.w	r0, r0, lr, lsr #21
 80005e8:	ea4f 2ece 	mov.w	lr, lr, lsl #11
 80005ec:	f1b4 0cfd 	subs.w	ip, r4, #253	; 0xfd
 80005f0:	bf88      	it	hi
 80005f2:	f5bc 6fe0 	cmphi.w	ip, #1792	; 0x700
 80005f6:	d81e      	bhi.n	8000636 <__aeabi_dmul+0xde>
 80005f8:	f1be 4f00 	cmp.w	lr, #2147483648	; 0x80000000
 80005fc:	bf08      	it	eq
 80005fe:	ea5f 0e50 	movseq.w	lr, r0, lsr #1
 8000602:	f150 0000 	adcs.w	r0, r0, #0
 8000606:	eb41 5104 	adc.w	r1, r1, r4, lsl #20
 800060a:	bd70      	pop	{r4, r5, r6, pc}
 800060c:	f006 4600 	and.w	r6, r6, #2147483648	; 0x80000000
 8000610:	ea46 0101 	orr.w	r1, r6, r1
 8000614:	ea40 0002 	orr.w	r0, r0, r2
 8000618:	ea81 0103 	eor.w	r1, r1, r3
 800061c:	ebb4 045c 	subs.w	r4, r4, ip, lsr #1
 8000620:	bfc2      	ittt	gt
 8000622:	ebd4 050c 	rsbsgt	r5, r4, ip
 8000626:	ea41 5104 	orrgt.w	r1, r1, r4, lsl #20
 800062a:	bd70      	popgt	{r4, r5, r6, pc}
 800062c:	f441 1180 	orr.w	r1, r1, #1048576	; 0x100000
 8000630:	f04f 0e00 	mov.w	lr, #0
 8000634:	3c01      	subs	r4, #1
 8000636:	f300 80ab 	bgt.w	8000790 <__aeabi_dmul+0x238>
 800063a:	f114 0f36 	cmn.w	r4, #54	; 0x36
 800063e:	bfde      	ittt	le
 8000640:	2000      	movle	r0, #0
 8000642:	f001 4100 	andle.w	r1, r1, #2147483648	; 0x80000000
 8000646:	bd70      	pople	{r4, r5, r6, pc}
 8000648:	f1c4 0400 	rsb	r4, r4, #0
 800064c:	3c20      	subs	r4, #32
 800064e:	da35      	bge.n	80006bc <__aeabi_dmul+0x164>
 8000650:	340c      	adds	r4, #12
 8000652:	dc1b      	bgt.n	800068c <__aeabi_dmul+0x134>
 8000654:	f104 0414 	add.w	r4, r4, #20
 8000658:	f1c4 0520 	rsb	r5, r4, #32
 800065c:	fa00 f305 	lsl.w	r3, r0, r5
 8000660:	fa20 f004 	lsr.w	r0, r0, r4
 8000664:	fa01 f205 	lsl.w	r2, r1, r5
 8000668:	ea40 0002 	orr.w	r0, r0, r2
 800066c:	f001 4200 	and.w	r2, r1, #2147483648	; 0x80000000
 8000670:	f021 4100 	bic.w	r1, r1, #2147483648	; 0x80000000
 8000674:	eb10 70d3 	adds.w	r0, r0, r3, lsr #31
 8000678:	fa21 f604 	lsr.w	r6, r1, r4
 800067c:	eb42 0106 	adc.w	r1, r2, r6
 8000680:	ea5e 0e43 	orrs.w	lr, lr, r3, lsl #1
 8000684:	bf08      	it	eq
 8000686:	ea20 70d3 	biceq.w	r0, r0, r3, lsr #31
 800068a:	bd70      	pop	{r4, r5, r6, pc}
 800068c:	f1c4 040c 	rsb	r4, r4, #12
 8000690:	f1c4 0520 	rsb	r5, r4, #32
 8000694:	fa00 f304 	lsl.w	r3, r0, r4
 8000698:	fa20 f005 	lsr.w	r0, r0, r5
 800069c:	fa01 f204 	lsl.w	r2, r1, r4
 80006a0:	ea40 0002 	orr.w	r0, r0, r2
 80006a4:	f001 4100 	and.w	r1, r1, #2147483648	; 0x80000000
 80006a8:	eb10 70d3 	adds.w	r0, r0, r3, lsr #31
 80006ac:	f141 0100 	adc.w	r1, r1, #0
 80006b0:	ea5e 0e43 	orrs.w	lr, lr, r3, lsl #1
 80006b4:	bf08      	it	eq
 80006b6:	ea20 70d3 	biceq.w	r0, r0, r3, lsr #31
 80006ba:	bd70      	pop	{r4, r5, r6, pc}
 80006bc:	f1c4 0520 	rsb	r5, r4, #32
 80006c0:	fa00 f205 	lsl.w	r2, r0, r5
 80006c4:	ea4e 0e02 	orr.w	lr, lr, r2
 80006c8:	fa20 f304 	lsr.w	r3, r0, r4
 80006cc:	fa01 f205 	lsl.w	r2, r1, r5
 80006d0:	ea43 0302 	orr.w	r3, r3, r2
 80006d4:	fa21 f004 	lsr.w	r0, r1, r4
 80006d8:	f001 4100 	and.w	r1, r1, #2147483648	; 0x80000000
 80006dc:	fa21 f204 	lsr.w	r2, r1, r4
 80006e0:	ea20 0002 	bic.w	r0, r0, r2
 80006e4:	eb00 70d3 	add.w	r0, r0, r3, lsr #31
 80006e8:	ea5e 0e43 	orrs.w	lr, lr, r3, lsl #1
 80006ec:	bf08      	it	eq
 80006ee:	ea20 70d3 	biceq.w	r0, r0, r3, lsr #31
 80006f2:	bd70      	pop	{r4, r5, r6, pc}
 80006f4:	f094 0f00 	teq	r4, #0
 80006f8:	d10f      	bne.n	800071a <__aeabi_dmul+0x1c2>
 80006fa:	f001 4600 	and.w	r6, r1, #2147483648	; 0x80000000
 80006fe:	0040      	lsls	r0, r0, #1
 8000700:	eb41 0101 	adc.w	r1, r1, r1
 8000704:	f411 1f80 	tst.w	r1, #1048576	; 0x100000
 8000708:	bf08      	it	eq
 800070a:	3c01      	subeq	r4, #1
 800070c:	d0f7      	beq.n	80006fe <__aeabi_dmul+0x1a6>
 800070e:	ea41 0106 	orr.w	r1, r1, r6
 8000712:	f095 0f00 	teq	r5, #0
 8000716:	bf18      	it	ne
 8000718:	4770      	bxne	lr
 800071a:	f003 4600 	and.w	r6, r3, #2147483648	; 0x80000000
 800071e:	0052      	lsls	r2, r2, #1
 8000720:	eb43 0303 	adc.w	r3, r3, r3
 8000724:	f413 1f80 	tst.w	r3, #1048576	; 0x100000
 8000728:	bf08      	it	eq
 800072a:	3d01      	subeq	r5, #1
 800072c:	d0f7      	beq.n	800071e <__aeabi_dmul+0x1c6>
 800072e:	ea43 0306 	orr.w	r3, r3, r6
 8000732:	4770      	bx	lr
 8000734:	ea94 0f0c 	teq	r4, ip
 8000738:	ea0c 5513 	and.w	r5, ip, r3, lsr #20
 800073c:	bf18      	it	ne
 800073e:	ea95 0f0c 	teqne	r5, ip
 8000742:	d00c      	beq.n	800075e <__aeabi_dmul+0x206>
 8000744:	ea50 0641 	orrs.w	r6, r0, r1, lsl #1
 8000748:	bf18      	it	ne
 800074a:	ea52 0643 	orrsne.w	r6, r2, r3, lsl #1
 800074e:	d1d1      	bne.n	80006f4 <__aeabi_dmul+0x19c>
 8000750:	ea81 0103 	eor.w	r1, r1, r3
 8000754:	f001 4100 	and.w	r1, r1, #2147483648	; 0x80000000
 8000758:	f04f 0000 	mov.w	r0, #0
 800075c:	bd70      	pop	{r4, r5, r6, pc}
 800075e:	ea50 0641 	orrs.w	r6, r0, r1, lsl #1
 8000762:	bf06      	itte	eq
 8000764:	4610      	moveq	r0, r2
 8000766:	4619      	moveq	r1, r3
 8000768:	ea52 0643 	orrsne.w	r6, r2, r3, lsl #1
 800076c:	d019      	beq.n	80007a2 <__aeabi_dmul+0x24a>
 800076e:	ea94 0f0c 	teq	r4, ip
 8000772:	d102      	bne.n	800077a <__aeabi_dmul+0x222>
 8000774:	ea50 3601 	orrs.w	r6, r0, r1, lsl #12
 8000778:	d113      	bne.n	80007a2 <__aeabi_dmul+0x24a>
 800077a:	ea95 0f0c 	teq	r5, ip
 800077e:	d105      	bne.n	800078c <__aeabi_dmul+0x234>
 8000780:	ea52 3603 	orrs.w	r6, r2, r3, lsl #12
 8000784:	bf1c      	itt	ne
 8000786:	4610      	movne	r0, r2
 8000788:	4619      	movne	r1, r3
 800078a:	d10a      	bne.n	80007a2 <__aeabi_dmul+0x24a>
 800078c:	ea81 0103 	eor.w	r1, r1, r3
 8000790:	f001 4100 	and.w	r1, r1, #2147483648	; 0x80000000
 8000794:	f041 41fe 	orr.w	r1, r1, #2130706432	; 0x7f000000
 8000798:	f441 0170 	orr.w	r1, r1, #15728640	; 0xf00000
 800079c:	f04f 0000 	mov.w	r0, #0
 80007a0:	bd70      	pop	{r4, r5, r6, pc}
 80007a2:	f041 41fe 	orr.w	r1, r1, #2130706432	; 0x7f000000
 80007a6:	f441 0178 	orr.w	r1, r1, #16252928	; 0xf80000
 80007aa:	bd70      	pop	{r4, r5, r6, pc}

080007ac <__aeabi_ddiv>:
 80007ac:	b570      	push	{r4, r5, r6, lr}
 80007ae:	f04f 0cff 	mov.w	ip, #255	; 0xff
 80007b2:	f44c 6ce0 	orr.w	ip, ip, #1792	; 0x700
 80007b6:	ea1c 5411 	ands.w	r4, ip, r1, lsr #20
 80007ba:	bf1d      	ittte	ne
 80007bc:	ea1c 5513 	andsne.w	r5, ip, r3, lsr #20
 80007c0:	ea94 0f0c 	teqne	r4, ip
 80007c4:	ea95 0f0c 	teqne	r5, ip
 80007c8:	f000 f8a7 	bleq	800091a <__aeabi_ddiv+0x16e>
 80007cc:	eba4 0405 	sub.w	r4, r4, r5
 80007d0:	ea81 0e03 	eor.w	lr, r1, r3
 80007d4:	ea52 3503 	orrs.w	r5, r2, r3, lsl #12
 80007d8:	ea4f 3101 	mov.w	r1, r1, lsl #12
 80007dc:	f000 8088 	beq.w	80008f0 <__aeabi_ddiv+0x144>
 80007e0:	ea4f 3303 	mov.w	r3, r3, lsl #12
 80007e4:	f04f 5580 	mov.w	r5, #268435456	; 0x10000000
 80007e8:	ea45 1313 	orr.w	r3, r5, r3, lsr #4
 80007ec:	ea43 6312 	orr.w	r3, r3, r2, lsr #24
 80007f0:	ea4f 2202 	mov.w	r2, r2, lsl #8
 80007f4:	ea45 1511 	orr.w	r5, r5, r1, lsr #4
 80007f8:	ea45 6510 	orr.w	r5, r5, r0, lsr #24
 80007fc:	ea4f 2600 	mov.w	r6, r0, lsl #8
 8000800:	f00e 4100 	and.w	r1, lr, #2147483648	; 0x80000000
 8000804:	429d      	cmp	r5, r3
 8000806:	bf08      	it	eq
 8000808:	4296      	cmpeq	r6, r2
 800080a:	f144 04fd 	adc.w	r4, r4, #253	; 0xfd
 800080e:	f504 7440 	add.w	r4, r4, #768	; 0x300
 8000812:	d202      	bcs.n	800081a <__aeabi_ddiv+0x6e>
 8000814:	085b      	lsrs	r3, r3, #1
 8000816:	ea4f 0232 	mov.w	r2, r2, rrx
 800081a:	1ab6      	subs	r6, r6, r2
 800081c:	eb65 0503 	sbc.w	r5, r5, r3
 8000820:	085b      	lsrs	r3, r3, #1
 8000822:	ea4f 0232 	mov.w	r2, r2, rrx
 8000826:	f44f 1080 	mov.w	r0, #1048576	; 0x100000
 800082a:	f44f 2c00 	mov.w	ip, #524288	; 0x80000
 800082e:	ebb6 0e02 	subs.w	lr, r6, r2
 8000832:	eb75 0e03 	sbcs.w	lr, r5, r3
 8000836:	bf22      	ittt	cs
 8000838:	1ab6      	subcs	r6, r6, r2
 800083a:	4675      	movcs	r5, lr
 800083c:	ea40 000c 	orrcs.w	r0, r0, ip
 8000840:	085b      	lsrs	r3, r3, #1
 8000842:	ea4f 0232 	mov.w	r2, r2, rrx
 8000846:	ebb6 0e02 	subs.w	lr, r6, r2
 800084a:	eb75 0e03 	sbcs.w	lr, r5, r3
 800084e:	bf22      	ittt	cs
 8000850:	1ab6      	subcs	r6, r6, r2
 8000852:	4675      	movcs	r5, lr
 8000854:	ea40 005c 	orrcs.w	r0, r0, ip, lsr #1
 8000858:	085b      	lsrs	r3, r3, #1
 800085a:	ea4f 0232 	mov.w	r2, r2, rrx
 800085e:	ebb6 0e02 	subs.w	lr, r6, r2
 8000862:	eb75 0e03 	sbcs.w	lr, r5, r3
 8000866:	bf22      	ittt	cs
 8000868:	1ab6      	subcs	r6, r6, r2
 800086a:	4675      	movcs	r5, lr
 800086c:	ea40 009c 	orrcs.w	r0, r0, ip, lsr #2
 8000870:	085b      	lsrs	r3, r3, #1
 8000872:	ea4f 0232 	mov.w	r2, r2, rrx
 8000876:	ebb6 0e02 	subs.w	lr, r6, r2
 800087a:	eb75 0e03 	sbcs.w	lr, r5, r3
 800087e:	bf22      	ittt	cs
 8000880:	1ab6      	subcs	r6, r6, r2
 8000882:	4675      	movcs	r5, lr
 8000884:	ea40 00dc 	orrcs.w	r0, r0, ip, lsr #3
 8000888:	ea55 0e06 	orrs.w	lr, r5, r6
 800088c:	d018      	beq.n	80008c0 <__aeabi_ddiv+0x114>
 800088e:	ea4f 1505 	mov.w	r5, r5, lsl #4
 8000892:	ea45 7516 	orr.w	r5, r5, r6, lsr #28
 8000896:	ea4f 1606 	mov.w	r6, r6, lsl #4
 800089a:	ea4f 03c3 	mov.w	r3, r3, lsl #3
 800089e:	ea43 7352 	orr.w	r3, r3, r2, lsr #29
 80008a2:	ea4f 02c2 	mov.w	r2, r2, lsl #3
 80008a6:	ea5f 1c1c 	movs.w	ip, ip, lsr #4
 80008aa:	d1c0      	bne.n	800082e <__aeabi_ddiv+0x82>
 80008ac:	f411 1f80 	tst.w	r1, #1048576	; 0x100000
 80008b0:	d10b      	bne.n	80008ca <__aeabi_ddiv+0x11e>
 80008b2:	ea41 0100 	orr.w	r1, r1, r0
 80008b6:	f04f 0000 	mov.w	r0, #0
 80008ba:	f04f 4c00 	mov.w	ip, #2147483648	; 0x80000000
 80008be:	e7b6      	b.n	800082e <__aeabi_ddiv+0x82>
 80008c0:	f411 1f80 	tst.w	r1, #1048576	; 0x100000
 80008c4:	bf04      	itt	eq
 80008c6:	4301      	orreq	r1, r0
 80008c8:	2000      	moveq	r0, #0
 80008ca:	f1b4 0cfd 	subs.w	ip, r4, #253	; 0xfd
 80008ce:	bf88      	it	hi
 80008d0:	f5bc 6fe0 	cmphi.w	ip, #1792	; 0x700
 80008d4:	f63f aeaf 	bhi.w	8000636 <__aeabi_dmul+0xde>
 80008d8:	ebb5 0c03 	subs.w	ip, r5, r3
 80008dc:	bf04      	itt	eq
 80008de:	ebb6 0c02 	subseq.w	ip, r6, r2
 80008e2:	ea5f 0c50 	movseq.w	ip, r0, lsr #1
 80008e6:	f150 0000 	adcs.w	r0, r0, #0
 80008ea:	eb41 5104 	adc.w	r1, r1, r4, lsl #20
 80008ee:	bd70      	pop	{r4, r5, r6, pc}
 80008f0:	f00e 4e00 	and.w	lr, lr, #2147483648	; 0x80000000
 80008f4:	ea4e 3111 	orr.w	r1, lr, r1, lsr #12
 80008f8:	eb14 045c 	adds.w	r4, r4, ip, lsr #1
 80008fc:	bfc2      	ittt	gt
 80008fe:	ebd4 050c 	rsbsgt	r5, r4, ip
 8000902:	ea41 5104 	orrgt.w	r1, r1, r4, lsl #20
 8000906:	bd70      	popgt	{r4, r5, r6, pc}
 8000908:	f441 1180 	orr.w	r1, r1, #1048576	; 0x100000
 800090c:	f04f 0e00 	mov.w	lr, #0
 8000910:	3c01      	subs	r4, #1
 8000912:	e690      	b.n	8000636 <__aeabi_dmul+0xde>
 8000914:	ea45 0e06 	orr.w	lr, r5, r6
 8000918:	e68d      	b.n	8000636 <__aeabi_dmul+0xde>
 800091a:	ea0c 5513 	and.w	r5, ip, r3, lsr #20
 800091e:	ea94 0f0c 	teq	r4, ip
 8000922:	bf08      	it	eq
 8000924:	ea95 0f0c 	teqeq	r5, ip
 8000928:	f43f af3b 	beq.w	80007a2 <__aeabi_dmul+0x24a>
 800092c:	ea94 0f0c 	teq	r4, ip
 8000930:	d10a      	bne.n	8000948 <__aeabi_ddiv+0x19c>
 8000932:	ea50 3401 	orrs.w	r4, r0, r1, lsl #12
 8000936:	f47f af34 	bne.w	80007a2 <__aeabi_dmul+0x24a>
 800093a:	ea95 0f0c 	teq	r5, ip
 800093e:	f47f af25 	bne.w	800078c <__aeabi_dmul+0x234>
 8000942:	4610      	mov	r0, r2
 8000944:	4619      	mov	r1, r3
 8000946:	e72c      	b.n	80007a2 <__aeabi_dmul+0x24a>
 8000948:	ea95 0f0c 	teq	r5, ip
 800094c:	d106      	bne.n	800095c <__aeabi_ddiv+0x1b0>
 800094e:	ea52 3503 	orrs.w	r5, r2, r3, lsl #12
 8000952:	f43f aefd 	beq.w	8000750 <__aeabi_dmul+0x1f8>
 8000956:	4610      	mov	r0, r2
 8000958:	4619      	mov	r1, r3
 800095a:	e722      	b.n	80007a2 <__aeabi_dmul+0x24a>
 800095c:	ea50 0641 	orrs.w	r6, r0, r1, lsl #1
 8000960:	bf18      	it	ne
 8000962:	ea52 0643 	orrsne.w	r6, r2, r3, lsl #1
 8000966:	f47f aec5 	bne.w	80006f4 <__aeabi_dmul+0x19c>
 800096a:	ea50 0441 	orrs.w	r4, r0, r1, lsl #1
 800096e:	f47f af0d 	bne.w	800078c <__aeabi_dmul+0x234>
 8000972:	ea52 0543 	orrs.w	r5, r2, r3, lsl #1
 8000976:	f47f aeeb 	bne.w	8000750 <__aeabi_dmul+0x1f8>
 800097a:	e712      	b.n	80007a2 <__aeabi_dmul+0x24a>

0800097c <__gedf2>:
 800097c:	f04f 3cff 	mov.w	ip, #4294967295
 8000980:	e006      	b.n	8000990 <__cmpdf2+0x4>
 8000982:	bf00      	nop

08000984 <__ledf2>:
 8000984:	f04f 0c01 	mov.w	ip, #1
 8000988:	e002      	b.n	8000990 <__cmpdf2+0x4>
 800098a:	bf00      	nop

0800098c <__cmpdf2>:
 800098c:	f04f 0c01 	mov.w	ip, #1
 8000990:	f84d cd04 	str.w	ip, [sp, #-4]!
 8000994:	ea4f 0c41 	mov.w	ip, r1, lsl #1
 8000998:	ea7f 5c6c 	mvns.w	ip, ip, asr #21
 800099c:	ea4f 0c43 	mov.w	ip, r3, lsl #1
 80009a0:	bf18      	it	ne
 80009a2:	ea7f 5c6c 	mvnsne.w	ip, ip, asr #21
 80009a6:	d01b      	beq.n	80009e0 <__cmpdf2+0x54>
 80009a8:	b001      	add	sp, #4
 80009aa:	ea50 0c41 	orrs.w	ip, r0, r1, lsl #1
 80009ae:	bf0c      	ite	eq
 80009b0:	ea52 0c43 	orrseq.w	ip, r2, r3, lsl #1
 80009b4:	ea91 0f03 	teqne	r1, r3
 80009b8:	bf02      	ittt	eq
 80009ba:	ea90 0f02 	teqeq	r0, r2
 80009be:	2000      	moveq	r0, #0
 80009c0:	4770      	bxeq	lr
 80009c2:	f110 0f00 	cmn.w	r0, #0
 80009c6:	ea91 0f03 	teq	r1, r3
 80009ca:	bf58      	it	pl
 80009cc:	4299      	cmppl	r1, r3
 80009ce:	bf08      	it	eq
 80009d0:	4290      	cmpeq	r0, r2
 80009d2:	bf2c      	ite	cs
 80009d4:	17d8      	asrcs	r0, r3, #31
 80009d6:	ea6f 70e3 	mvncc.w	r0, r3, asr #31
 80009da:	f040 0001 	orr.w	r0, r0, #1
 80009de:	4770      	bx	lr
 80009e0:	ea4f 0c41 	mov.w	ip, r1, lsl #1
 80009e4:	ea7f 5c6c 	mvns.w	ip, ip, asr #21
 80009e8:	d102      	bne.n	80009f0 <__cmpdf2+0x64>
 80009ea:	ea50 3c01 	orrs.w	ip, r0, r1, lsl #12
 80009ee:	d107      	bne.n	8000a00 <__cmpdf2+0x74>
 80009f0:	ea4f 0c43 	mov.w	ip, r3, lsl #1
 80009f4:	ea7f 5c6c 	mvns.w	ip, ip, asr #21
 80009f8:	d1d6      	bne.n	80009a8 <__cmpdf2+0x1c>
 80009fa:	ea52 3c03 	orrs.w	ip, r2, r3, lsl #12
 80009fe:	d0d3      	beq.n	80009a8 <__cmpdf2+0x1c>
 8000a00:	f85d 0b04 	ldr.w	r0, [sp], #4
 8000a04:	4770      	bx	lr
 8000a06:	bf00      	nop

08000a08 <__aeabi_cdrcmple>:
 8000a08:	4684      	mov	ip, r0
 8000a0a:	4610      	mov	r0, r2
 8000a0c:	4662      	mov	r2, ip
 8000a0e:	468c      	mov	ip, r1
 8000a10:	4619      	mov	r1, r3
 8000a12:	4663      	mov	r3, ip
 8000a14:	e000      	b.n	8000a18 <__aeabi_cdcmpeq>
 8000a16:	bf00      	nop

08000a18 <__aeabi_cdcmpeq>:
 8000a18:	b501      	push	{r0, lr}
 8000a1a:	f7ff ffb7 	bl	800098c <__cmpdf2>
 8000a1e:	2800      	cmp	r0, #0
 8000a20:	bf48      	it	mi
 8000a22:	f110 0f00 	cmnmi.w	r0, #0
 8000a26:	bd01      	pop	{r0, pc}

08000a28 <__aeabi_dcmpeq>:
 8000a28:	f84d ed08 	str.w	lr, [sp, #-8]!
 8000a2c:	f7ff fff4 	bl	8000a18 <__aeabi_cdcmpeq>
 8000a30:	bf0c      	ite	eq
 8000a32:	2001      	moveq	r0, #1
 8000a34:	2000      	movne	r0, #0
 8000a36:	f85d fb08 	ldr.w	pc, [sp], #8
 8000a3a:	bf00      	nop

08000a3c <__aeabi_dcmplt>:
 8000a3c:	f84d ed08 	str.w	lr, [sp, #-8]!
 8000a40:	f7ff ffea 	bl	8000a18 <__aeabi_cdcmpeq>
 8000a44:	bf34      	ite	cc
 8000a46:	2001      	movcc	r0, #1
 8000a48:	2000      	movcs	r0, #0
 8000a4a:	f85d fb08 	ldr.w	pc, [sp], #8
 8000a4e:	bf00      	nop

08000a50 <__aeabi_dcmple>:
 8000a50:	f84d ed08 	str.w	lr, [sp, #-8]!
 8000a54:	f7ff ffe0 	bl	8000a18 <__aeabi_cdcmpeq>
 8000a58:	bf94      	ite	ls
 8000a5a:	2001      	movls	r0, #1
 8000a5c:	2000      	movhi	r0, #0
 8000a5e:	f85d fb08 	ldr.w	pc, [sp], #8
 8000a62:	bf00      	nop

08000a64 <__aeabi_dcmpge>:
 8000a64:	f84d ed08 	str.w	lr, [sp, #-8]!
 8000a68:	f7ff ffce 	bl	8000a08 <__aeabi_cdrcmple>
 8000a6c:	bf94      	ite	ls
 8000a6e:	2001      	movls	r0, #1
 8000a70:	2000      	movhi	r0, #0
 8000a72:	f85d fb08 	ldr.w	pc, [sp], #8
 8000a76:	bf00      	nop

08000a78 <__aeabi_dcmpgt>:
 8000a78:	f84d ed08 	str.w	lr, [sp, #-8]!
 8000a7c:	f7ff ffc4 	bl	8000a08 <__aeabi_cdrcmple>
 8000a80:	bf34      	ite	cc
 8000a82:	2001      	movcc	r0, #1
 8000a84:	2000      	movcs	r0, #0
 8000a86:	f85d fb08 	ldr.w	pc, [sp], #8
 8000a8a:	bf00      	nop

08000a8c <__aeabi_d2iz>:
 8000a8c:	ea4f 0241 	mov.w	r2, r1, lsl #1
 8000a90:	f512 1200 	adds.w	r2, r2, #2097152	; 0x200000
 8000a94:	d215      	bcs.n	8000ac2 <__aeabi_d2iz+0x36>
 8000a96:	d511      	bpl.n	8000abc <__aeabi_d2iz+0x30>
 8000a98:	f46f 7378 	mvn.w	r3, #992	; 0x3e0
 8000a9c:	ebb3 5262 	subs.w	r2, r3, r2, asr #21
 8000aa0:	d912      	bls.n	8000ac8 <__aeabi_d2iz+0x3c>
 8000aa2:	ea4f 23c1 	mov.w	r3, r1, lsl #11
 8000aa6:	f043 4300 	orr.w	r3, r3, #2147483648	; 0x80000000
 8000aaa:	ea43 5350 	orr.w	r3, r3, r0, lsr #21
 8000aae:	f011 4f00 	tst.w	r1, #2147483648	; 0x80000000
 8000ab2:	fa23 f002 	lsr.w	r0, r3, r2
 8000ab6:	bf18      	it	ne
 8000ab8:	4240      	negne	r0, r0
 8000aba:	4770      	bx	lr
 8000abc:	f04f 0000 	mov.w	r0, #0
 8000ac0:	4770      	bx	lr
 8000ac2:	ea50 3001 	orrs.w	r0, r0, r1, lsl #12
 8000ac6:	d105      	bne.n	8000ad4 <__aeabi_d2iz+0x48>
 8000ac8:	f011 4000 	ands.w	r0, r1, #2147483648	; 0x80000000
 8000acc:	bf08      	it	eq
 8000ace:	f06f 4000 	mvneq.w	r0, #2147483648	; 0x80000000
 8000ad2:	4770      	bx	lr
 8000ad4:	f04f 0000 	mov.w	r0, #0
 8000ad8:	4770      	bx	lr
 8000ada:	bf00      	nop

08000adc <__aeabi_d2uiz>:
 8000adc:	004a      	lsls	r2, r1, #1
 8000ade:	d211      	bcs.n	8000b04 <__aeabi_d2uiz+0x28>
 8000ae0:	f512 1200 	adds.w	r2, r2, #2097152	; 0x200000
 8000ae4:	d211      	bcs.n	8000b0a <__aeabi_d2uiz+0x2e>
 8000ae6:	d50d      	bpl.n	8000b04 <__aeabi_d2uiz+0x28>
 8000ae8:	f46f 7378 	mvn.w	r3, #992	; 0x3e0
 8000aec:	ebb3 5262 	subs.w	r2, r3, r2, asr #21
 8000af0:	d40e      	bmi.n	8000b10 <__aeabi_d2uiz+0x34>
 8000af2:	ea4f 23c1 	mov.w	r3, r1, lsl #11
 8000af6:	f043 4300 	orr.w	r3, r3, #2147483648	; 0x80000000
 8000afa:	ea43 5350 	orr.w	r3, r3, r0, lsr #21
 8000afe:	fa23 f002 	lsr.w	r0, r3, r2
 8000b02:	4770      	bx	lr
 8000b04:	f04f 0000 	mov.w	r0, #0
 8000b08:	4770      	bx	lr
 8000b0a:	ea50 3001 	orrs.w	r0, r0, r1, lsl #12
 8000b0e:	d102      	bne.n	8000b16 <__aeabi_d2uiz+0x3a>
 8000b10:	f04f 30ff 	mov.w	r0, #4294967295
 8000b14:	4770      	bx	lr
 8000b16:	f04f 0000 	mov.w	r0, #0
 8000b1a:	4770      	bx	lr

08000b1c <__aeabi_d2f>:
 8000b1c:	ea4f 0241 	mov.w	r2, r1, lsl #1
 8000b20:	f1b2 43e0 	subs.w	r3, r2, #1879048192	; 0x70000000
 8000b24:	bf24      	itt	cs
 8000b26:	f5b3 1c00 	subscs.w	ip, r3, #2097152	; 0x200000
 8000b2a:	f1dc 5cfe 	rsbscs	ip, ip, #532676608	; 0x1fc00000
 8000b2e:	d90d      	bls.n	8000b4c <__aeabi_d2f+0x30>
 8000b30:	f001 4c00 	and.w	ip, r1, #2147483648	; 0x80000000
 8000b34:	ea4f 02c0 	mov.w	r2, r0, lsl #3
 8000b38:	ea4c 7050 	orr.w	r0, ip, r0, lsr #29
 8000b3c:	f1b2 4f00 	cmp.w	r2, #2147483648	; 0x80000000
 8000b40:	eb40 0083 	adc.w	r0, r0, r3, lsl #2
 8000b44:	bf08      	it	eq
 8000b46:	f020 0001 	biceq.w	r0, r0, #1
 8000b4a:	4770      	bx	lr
 8000b4c:	f011 4f80 	tst.w	r1, #1073741824	; 0x40000000
 8000b50:	d121      	bne.n	8000b96 <__aeabi_d2f+0x7a>
 8000b52:	f113 7238 	adds.w	r2, r3, #48234496	; 0x2e00000
 8000b56:	bfbc      	itt	lt
 8000b58:	f001 4000 	andlt.w	r0, r1, #2147483648	; 0x80000000
 8000b5c:	4770      	bxlt	lr
 8000b5e:	f441 1180 	orr.w	r1, r1, #1048576	; 0x100000
 8000b62:	ea4f 5252 	mov.w	r2, r2, lsr #21
 8000b66:	f1c2 0218 	rsb	r2, r2, #24
 8000b6a:	f1c2 0c20 	rsb	ip, r2, #32
 8000b6e:	fa10 f30c 	lsls.w	r3, r0, ip
 8000b72:	fa20 f002 	lsr.w	r0, r0, r2
 8000b76:	bf18      	it	ne
 8000b78:	f040 0001 	orrne.w	r0, r0, #1
 8000b7c:	ea4f 23c1 	mov.w	r3, r1, lsl #11
 8000b80:	ea4f 23d3 	mov.w	r3, r3, lsr #11
 8000b84:	fa03 fc0c 	lsl.w	ip, r3, ip
 8000b88:	ea40 000c 	orr.w	r0, r0, ip
 8000b8c:	fa23 f302 	lsr.w	r3, r3, r2
 8000b90:	ea4f 0343 	mov.w	r3, r3, lsl #1
 8000b94:	e7cc      	b.n	8000b30 <__aeabi_d2f+0x14>
 8000b96:	ea7f 5362 	mvns.w	r3, r2, asr #21
 8000b9a:	d107      	bne.n	8000bac <__aeabi_d2f+0x90>
 8000b9c:	ea50 3301 	orrs.w	r3, r0, r1, lsl #12
 8000ba0:	bf1e      	ittt	ne
 8000ba2:	f04f 40fe 	movne.w	r0, #2130706432	; 0x7f000000
 8000ba6:	f440 0040 	orrne.w	r0, r0, #12582912	; 0xc00000
 8000baa:	4770      	bxne	lr
 8000bac:	f001 4000 	and.w	r0, r1, #2147483648	; 0x80000000
 8000bb0:	f040 40fe 	orr.w	r0, r0, #2130706432	; 0x7f000000
 8000bb4:	f440 0000 	orr.w	r0, r0, #8388608	; 0x800000
 8000bb8:	4770      	bx	lr
 8000bba:	bf00      	nop

08000bbc <__aeabi_uldivmod>:
 8000bbc:	b953      	cbnz	r3, 8000bd4 <__aeabi_uldivmod+0x18>
 8000bbe:	b94a      	cbnz	r2, 8000bd4 <__aeabi_uldivmod+0x18>
 8000bc0:	2900      	cmp	r1, #0
 8000bc2:	bf08      	it	eq
 8000bc4:	2800      	cmpeq	r0, #0
 8000bc6:	bf1c      	itt	ne
 8000bc8:	f04f 31ff 	movne.w	r1, #4294967295
 8000bcc:	f04f 30ff 	movne.w	r0, #4294967295
 8000bd0:	f000 b972 	b.w	8000eb8 <__aeabi_idiv0>
 8000bd4:	f1ad 0c08 	sub.w	ip, sp, #8
 8000bd8:	e96d ce04 	strd	ip, lr, [sp, #-16]!
 8000bdc:	f000 f806 	bl	8000bec <__udivmoddi4>
 8000be0:	f8dd e004 	ldr.w	lr, [sp, #4]
 8000be4:	e9dd 2302 	ldrd	r2, r3, [sp, #8]
 8000be8:	b004      	add	sp, #16
 8000bea:	4770      	bx	lr

08000bec <__udivmoddi4>:
 8000bec:	e92d 47f0 	stmdb	sp!, {r4, r5, r6, r7, r8, r9, sl, lr}
 8000bf0:	9e08      	ldr	r6, [sp, #32]
 8000bf2:	4604      	mov	r4, r0
 8000bf4:	4688      	mov	r8, r1
 8000bf6:	2b00      	cmp	r3, #0
 8000bf8:	d14b      	bne.n	8000c92 <__udivmoddi4+0xa6>
 8000bfa:	428a      	cmp	r2, r1
 8000bfc:	4615      	mov	r5, r2
 8000bfe:	d967      	bls.n	8000cd0 <__udivmoddi4+0xe4>
 8000c00:	fab2 f282 	clz	r2, r2
 8000c04:	b14a      	cbz	r2, 8000c1a <__udivmoddi4+0x2e>
 8000c06:	f1c2 0720 	rsb	r7, r2, #32
 8000c0a:	fa01 f302 	lsl.w	r3, r1, r2
 8000c0e:	fa20 f707 	lsr.w	r7, r0, r7
 8000c12:	4095      	lsls	r5, r2
 8000c14:	ea47 0803 	orr.w	r8, r7, r3
 8000c18:	4094      	lsls	r4, r2
 8000c1a:	ea4f 4e15 	mov.w	lr, r5, lsr #16
 8000c1e:	0c23      	lsrs	r3, r4, #16
 8000c20:	fbb8 f7fe 	udiv	r7, r8, lr
 8000c24:	fa1f fc85 	uxth.w	ip, r5
 8000c28:	fb0e 8817 	mls	r8, lr, r7, r8
 8000c2c:	ea43 4308 	orr.w	r3, r3, r8, lsl #16
 8000c30:	fb07 f10c 	mul.w	r1, r7, ip
 8000c34:	4299      	cmp	r1, r3
 8000c36:	d909      	bls.n	8000c4c <__udivmoddi4+0x60>
 8000c38:	18eb      	adds	r3, r5, r3
 8000c3a:	f107 30ff 	add.w	r0, r7, #4294967295
 8000c3e:	f080 811b 	bcs.w	8000e78 <__udivmoddi4+0x28c>
 8000c42:	4299      	cmp	r1, r3
 8000c44:	f240 8118 	bls.w	8000e78 <__udivmoddi4+0x28c>
 8000c48:	3f02      	subs	r7, #2
 8000c4a:	442b      	add	r3, r5
 8000c4c:	1a5b      	subs	r3, r3, r1
 8000c4e:	b2a4      	uxth	r4, r4
 8000c50:	fbb3 f0fe 	udiv	r0, r3, lr
 8000c54:	fb0e 3310 	mls	r3, lr, r0, r3
 8000c58:	ea44 4403 	orr.w	r4, r4, r3, lsl #16
 8000c5c:	fb00 fc0c 	mul.w	ip, r0, ip
 8000c60:	45a4      	cmp	ip, r4
 8000c62:	d909      	bls.n	8000c78 <__udivmoddi4+0x8c>
 8000c64:	192c      	adds	r4, r5, r4
 8000c66:	f100 33ff 	add.w	r3, r0, #4294967295
 8000c6a:	f080 8107 	bcs.w	8000e7c <__udivmoddi4+0x290>
 8000c6e:	45a4      	cmp	ip, r4
 8000c70:	f240 8104 	bls.w	8000e7c <__udivmoddi4+0x290>
 8000c74:	3802      	subs	r0, #2
 8000c76:	442c      	add	r4, r5
 8000c78:	ea40 4007 	orr.w	r0, r0, r7, lsl #16
 8000c7c:	eba4 040c 	sub.w	r4, r4, ip
 8000c80:	2700      	movs	r7, #0
 8000c82:	b11e      	cbz	r6, 8000c8c <__udivmoddi4+0xa0>
 8000c84:	40d4      	lsrs	r4, r2
 8000c86:	2300      	movs	r3, #0
 8000c88:	e9c6 4300 	strd	r4, r3, [r6]
 8000c8c:	4639      	mov	r1, r7
 8000c8e:	e8bd 87f0 	ldmia.w	sp!, {r4, r5, r6, r7, r8, r9, sl, pc}
 8000c92:	428b      	cmp	r3, r1
 8000c94:	d909      	bls.n	8000caa <__udivmoddi4+0xbe>
 8000c96:	2e00      	cmp	r6, #0
 8000c98:	f000 80eb 	beq.w	8000e72 <__udivmoddi4+0x286>
 8000c9c:	2700      	movs	r7, #0
 8000c9e:	e9c6 0100 	strd	r0, r1, [r6]
 8000ca2:	4638      	mov	r0, r7
 8000ca4:	4639      	mov	r1, r7
 8000ca6:	e8bd 87f0 	ldmia.w	sp!, {r4, r5, r6, r7, r8, r9, sl, pc}
 8000caa:	fab3 f783 	clz	r7, r3
 8000cae:	2f00      	cmp	r7, #0
 8000cb0:	d147      	bne.n	8000d42 <__udivmoddi4+0x156>
 8000cb2:	428b      	cmp	r3, r1
 8000cb4:	d302      	bcc.n	8000cbc <__udivmoddi4+0xd0>
 8000cb6:	4282      	cmp	r2, r0
 8000cb8:	f200 80fa 	bhi.w	8000eb0 <__udivmoddi4+0x2c4>
 8000cbc:	1a84      	subs	r4, r0, r2
 8000cbe:	eb61 0303 	sbc.w	r3, r1, r3
 8000cc2:	2001      	movs	r0, #1
 8000cc4:	4698      	mov	r8, r3
 8000cc6:	2e00      	cmp	r6, #0
 8000cc8:	d0e0      	beq.n	8000c8c <__udivmoddi4+0xa0>
 8000cca:	e9c6 4800 	strd	r4, r8, [r6]
 8000cce:	e7dd      	b.n	8000c8c <__udivmoddi4+0xa0>
 8000cd0:	b902      	cbnz	r2, 8000cd4 <__udivmoddi4+0xe8>
 8000cd2:	deff      	udf	#255	; 0xff
 8000cd4:	fab2 f282 	clz	r2, r2
 8000cd8:	2a00      	cmp	r2, #0
 8000cda:	f040 808f 	bne.w	8000dfc <__udivmoddi4+0x210>
 8000cde:	1b49      	subs	r1, r1, r5
 8000ce0:	ea4f 4e15 	mov.w	lr, r5, lsr #16
 8000ce4:	fa1f f885 	uxth.w	r8, r5
 8000ce8:	2701      	movs	r7, #1
 8000cea:	fbb1 fcfe 	udiv	ip, r1, lr
 8000cee:	0c23      	lsrs	r3, r4, #16
 8000cf0:	fb0e 111c 	mls	r1, lr, ip, r1
 8000cf4:	ea43 4301 	orr.w	r3, r3, r1, lsl #16
 8000cf8:	fb08 f10c 	mul.w	r1, r8, ip
 8000cfc:	4299      	cmp	r1, r3
 8000cfe:	d907      	bls.n	8000d10 <__udivmoddi4+0x124>
 8000d00:	18eb      	adds	r3, r5, r3
 8000d02:	f10c 30ff 	add.w	r0, ip, #4294967295
 8000d06:	d202      	bcs.n	8000d0e <__udivmoddi4+0x122>
 8000d08:	4299      	cmp	r1, r3
 8000d0a:	f200 80cd 	bhi.w	8000ea8 <__udivmoddi4+0x2bc>
 8000d0e:	4684      	mov	ip, r0
 8000d10:	1a59      	subs	r1, r3, r1
 8000d12:	b2a3      	uxth	r3, r4
 8000d14:	fbb1 f0fe 	udiv	r0, r1, lr
 8000d18:	fb0e 1410 	mls	r4, lr, r0, r1
 8000d1c:	ea43 4404 	orr.w	r4, r3, r4, lsl #16
 8000d20:	fb08 f800 	mul.w	r8, r8, r0
 8000d24:	45a0      	cmp	r8, r4
 8000d26:	d907      	bls.n	8000d38 <__udivmoddi4+0x14c>
 8000d28:	192c      	adds	r4, r5, r4
 8000d2a:	f100 33ff 	add.w	r3, r0, #4294967295
 8000d2e:	d202      	bcs.n	8000d36 <__udivmoddi4+0x14a>
 8000d30:	45a0      	cmp	r8, r4
 8000d32:	f200 80b6 	bhi.w	8000ea2 <__udivmoddi4+0x2b6>
 8000d36:	4618      	mov	r0, r3
 8000d38:	eba4 0408 	sub.w	r4, r4, r8
 8000d3c:	ea40 400c 	orr.w	r0, r0, ip, lsl #16
 8000d40:	e79f      	b.n	8000c82 <__udivmoddi4+0x96>
 8000d42:	f1c7 0c20 	rsb	ip, r7, #32
 8000d46:	40bb      	lsls	r3, r7
 8000d48:	fa22 fe0c 	lsr.w	lr, r2, ip
 8000d4c:	ea4e 0e03 	orr.w	lr, lr, r3
 8000d50:	fa01 f407 	lsl.w	r4, r1, r7
 8000d54:	fa20 f50c 	lsr.w	r5, r0, ip
 8000d58:	fa21 f30c 	lsr.w	r3, r1, ip
 8000d5c:	ea4f 481e 	mov.w	r8, lr, lsr #16
 8000d60:	4325      	orrs	r5, r4
 8000d62:	fbb3 f9f8 	udiv	r9, r3, r8
 8000d66:	0c2c      	lsrs	r4, r5, #16
 8000d68:	fb08 3319 	mls	r3, r8, r9, r3
 8000d6c:	fa1f fa8e 	uxth.w	sl, lr
 8000d70:	ea44 4303 	orr.w	r3, r4, r3, lsl #16
 8000d74:	fb09 f40a 	mul.w	r4, r9, sl
 8000d78:	429c      	cmp	r4, r3
 8000d7a:	fa02 f207 	lsl.w	r2, r2, r7
 8000d7e:	fa00 f107 	lsl.w	r1, r0, r7
 8000d82:	d90b      	bls.n	8000d9c <__udivmoddi4+0x1b0>
 8000d84:	eb1e 0303 	adds.w	r3, lr, r3
 8000d88:	f109 30ff 	add.w	r0, r9, #4294967295
 8000d8c:	f080 8087 	bcs.w	8000e9e <__udivmoddi4+0x2b2>
 8000d90:	429c      	cmp	r4, r3
 8000d92:	f240 8084 	bls.w	8000e9e <__udivmoddi4+0x2b2>
 8000d96:	f1a9 0902 	sub.w	r9, r9, #2
 8000d9a:	4473      	add	r3, lr
 8000d9c:	1b1b      	subs	r3, r3, r4
 8000d9e:	b2ad      	uxth	r5, r5
 8000da0:	fbb3 f0f8 	udiv	r0, r3, r8
 8000da4:	fb08 3310 	mls	r3, r8, r0, r3
 8000da8:	ea45 4403 	orr.w	r4, r5, r3, lsl #16
 8000dac:	fb00 fa0a 	mul.w	sl, r0, sl
 8000db0:	45a2      	cmp	sl, r4
 8000db2:	d908      	bls.n	8000dc6 <__udivmoddi4+0x1da>
 8000db4:	eb1e 0404 	adds.w	r4, lr, r4
 8000db8:	f100 33ff 	add.w	r3, r0, #4294967295
 8000dbc:	d26b      	bcs.n	8000e96 <__udivmoddi4+0x2aa>
 8000dbe:	45a2      	cmp	sl, r4
 8000dc0:	d969      	bls.n	8000e96 <__udivmoddi4+0x2aa>
 8000dc2:	3802      	subs	r0, #2
 8000dc4:	4474      	add	r4, lr
 8000dc6:	ea40 4009 	orr.w	r0, r0, r9, lsl #16
 8000dca:	fba0 8902 	umull	r8, r9, r0, r2
 8000dce:	eba4 040a 	sub.w	r4, r4, sl
 8000dd2:	454c      	cmp	r4, r9
 8000dd4:	46c2      	mov	sl, r8
 8000dd6:	464b      	mov	r3, r9
 8000dd8:	d354      	bcc.n	8000e84 <__udivmoddi4+0x298>
 8000dda:	d051      	beq.n	8000e80 <__udivmoddi4+0x294>
 8000ddc:	2e00      	cmp	r6, #0
 8000dde:	d069      	beq.n	8000eb4 <__udivmoddi4+0x2c8>
 8000de0:	ebb1 050a 	subs.w	r5, r1, sl
 8000de4:	eb64 0403 	sbc.w	r4, r4, r3
 8000de8:	fa04 fc0c 	lsl.w	ip, r4, ip
 8000dec:	40fd      	lsrs	r5, r7
 8000dee:	40fc      	lsrs	r4, r7
 8000df0:	ea4c 0505 	orr.w	r5, ip, r5
 8000df4:	e9c6 5400 	strd	r5, r4, [r6]
 8000df8:	2700      	movs	r7, #0
 8000dfa:	e747      	b.n	8000c8c <__udivmoddi4+0xa0>
 8000dfc:	f1c2 0320 	rsb	r3, r2, #32
 8000e00:	fa20 f703 	lsr.w	r7, r0, r3
 8000e04:	4095      	lsls	r5, r2
 8000e06:	fa01 f002 	lsl.w	r0, r1, r2
 8000e0a:	fa21 f303 	lsr.w	r3, r1, r3
 8000e0e:	ea4f 4e15 	mov.w	lr, r5, lsr #16
 8000e12:	4338      	orrs	r0, r7
 8000e14:	0c01      	lsrs	r1, r0, #16
 8000e16:	fbb3 f7fe 	udiv	r7, r3, lr
 8000e1a:	fa1f f885 	uxth.w	r8, r5
 8000e1e:	fb0e 3317 	mls	r3, lr, r7, r3
 8000e22:	ea41 4103 	orr.w	r1, r1, r3, lsl #16
 8000e26:	fb07 f308 	mul.w	r3, r7, r8
 8000e2a:	428b      	cmp	r3, r1
 8000e2c:	fa04 f402 	lsl.w	r4, r4, r2
 8000e30:	d907      	bls.n	8000e42 <__udivmoddi4+0x256>
 8000e32:	1869      	adds	r1, r5, r1
 8000e34:	f107 3cff 	add.w	ip, r7, #4294967295
 8000e38:	d22f      	bcs.n	8000e9a <__udivmoddi4+0x2ae>
 8000e3a:	428b      	cmp	r3, r1
 8000e3c:	d92d      	bls.n	8000e9a <__udivmoddi4+0x2ae>
 8000e3e:	3f02      	subs	r7, #2
 8000e40:	4429      	add	r1, r5
 8000e42:	1acb      	subs	r3, r1, r3
 8000e44:	b281      	uxth	r1, r0
 8000e46:	fbb3 f0fe 	udiv	r0, r3, lr
 8000e4a:	fb0e 3310 	mls	r3, lr, r0, r3
 8000e4e:	ea41 4103 	orr.w	r1, r1, r3, lsl #16
 8000e52:	fb00 f308 	mul.w	r3, r0, r8
 8000e56:	428b      	cmp	r3, r1
 8000e58:	d907      	bls.n	8000e6a <__udivmoddi4+0x27e>
 8000e5a:	1869      	adds	r1, r5, r1
 8000e5c:	f100 3cff 	add.w	ip, r0, #4294967295
 8000e60:	d217      	bcs.n	8000e92 <__udivmoddi4+0x2a6>
 8000e62:	428b      	cmp	r3, r1
 8000e64:	d915      	bls.n	8000e92 <__udivmoddi4+0x2a6>
 8000e66:	3802      	subs	r0, #2
 8000e68:	4429      	add	r1, r5
 8000e6a:	1ac9      	subs	r1, r1, r3
 8000e6c:	ea40 4707 	orr.w	r7, r0, r7, lsl #16
 8000e70:	e73b      	b.n	8000cea <__udivmoddi4+0xfe>
 8000e72:	4637      	mov	r7, r6
 8000e74:	4630      	mov	r0, r6
 8000e76:	e709      	b.n	8000c8c <__udivmoddi4+0xa0>
 8000e78:	4607      	mov	r7, r0
 8000e7a:	e6e7      	b.n	8000c4c <__udivmoddi4+0x60>
 8000e7c:	4618      	mov	r0, r3
 8000e7e:	e6fb      	b.n	8000c78 <__udivmoddi4+0x8c>
 8000e80:	4541      	cmp	r1, r8
 8000e82:	d2ab      	bcs.n	8000ddc <__udivmoddi4+0x1f0>
 8000e84:	ebb8 0a02 	subs.w	sl, r8, r2
 8000e88:	eb69 020e 	sbc.w	r2, r9, lr
 8000e8c:	3801      	subs	r0, #1
 8000e8e:	4613      	mov	r3, r2
 8000e90:	e7a4      	b.n	8000ddc <__udivmoddi4+0x1f0>
 8000e92:	4660      	mov	r0, ip
 8000e94:	e7e9      	b.n	8000e6a <__udivmoddi4+0x27e>
 8000e96:	4618      	mov	r0, r3
 8000e98:	e795      	b.n	8000dc6 <__udivmoddi4+0x1da>
 8000e9a:	4667      	mov	r7, ip
 8000e9c:	e7d1      	b.n	8000e42 <__udivmoddi4+0x256>
 8000e9e:	4681      	mov	r9, r0
 8000ea0:	e77c      	b.n	8000d9c <__udivmoddi4+0x1b0>
 8000ea2:	3802      	subs	r0, #2
 8000ea4:	442c      	add	r4, r5
 8000ea6:	e747      	b.n	8000d38 <__udivmoddi4+0x14c>
 8000ea8:	f1ac 0c02 	sub.w	ip, ip, #2
 8000eac:	442b      	add	r3, r5
 8000eae:	e72f      	b.n	8000d10 <__udivmoddi4+0x124>
 8000eb0:	4638      	mov	r0, r7
 8000eb2:	e708      	b.n	8000cc6 <__udivmoddi4+0xda>
 8000eb4:	4637      	mov	r7, r6
 8000eb6:	e6e9      	b.n	8000c8c <__udivmoddi4+0xa0>

08000eb8 <__aeabi_idiv0>:
 8000eb8:	4770      	bx	lr
 8000eba:	bf00      	nop

08000ebc <GFX_SetFont>:
#if  USING_STRINGS == 1
const uint8_t* font;
uint8_t size = 1;

void GFX_SetFont(const uint8_t* font_t)
{
 8000ebc:	b480      	push	{r7}
 8000ebe:	b083      	sub	sp, #12
 8000ec0:	af00      	add	r7, sp, #0
 8000ec2:	6078      	str	r0, [r7, #4]
	font = font_t;
 8000ec4:	4a04      	ldr	r2, [pc, #16]	; (8000ed8 <GFX_SetFont+0x1c>)
 8000ec6:	687b      	ldr	r3, [r7, #4]
 8000ec8:	6013      	str	r3, [r2, #0]
}
 8000eca:	bf00      	nop
 8000ecc:	370c      	adds	r7, #12
 8000ece:	46bd      	mov	sp, r7
 8000ed0:	f85d 7b04 	ldr.w	r7, [sp], #4
 8000ed4:	4770      	bx	lr
 8000ed6:	bf00      	nop
 8000ed8:	20004d38 	.word	0x20004d38

08000edc <GFX_DrawChar>:
{
	return size;
}

void GFX_DrawChar(int x, int y, char chr, uint8_t color, uint8_t background)
{
 8000edc:	b590      	push	{r4, r7, lr}
 8000ede:	b089      	sub	sp, #36	; 0x24
 8000ee0:	af02      	add	r7, sp, #8
 8000ee2:	60f8      	str	r0, [r7, #12]
 8000ee4:	60b9      	str	r1, [r7, #8]
 8000ee6:	4611      	mov	r1, r2
 8000ee8:	461a      	mov	r2, r3
 8000eea:	460b      	mov	r3, r1
 8000eec:	71fb      	strb	r3, [r7, #7]
 8000eee:	4613      	mov	r3, r2
 8000ef0:	71bb      	strb	r3, [r7, #6]
	if(chr > 0x7E) return; // chr > '~'
 8000ef2:	79fb      	ldrb	r3, [r7, #7]
 8000ef4:	2b7e      	cmp	r3, #126	; 0x7e
 8000ef6:	f200 80a3 	bhi.w	8001040 <GFX_DrawChar+0x164>

	for(uint8_t i=0; i<font[1]; i++ ) // Each column (Width)
 8000efa:	2300      	movs	r3, #0
 8000efc:	75fb      	strb	r3, [r7, #23]
 8000efe:	e096      	b.n	800102e <GFX_DrawChar+0x152>
	{
        uint8_t line = (uint8_t)font[(chr-0x20) * font[1] + i + 2]; // Takie this line, (chr-0x20) = move 20 chars back,
 8000f00:	4b51      	ldr	r3, [pc, #324]	; (8001048 <GFX_DrawChar+0x16c>)
 8000f02:	681a      	ldr	r2, [r3, #0]
 8000f04:	79fb      	ldrb	r3, [r7, #7]
 8000f06:	3b20      	subs	r3, #32
 8000f08:	494f      	ldr	r1, [pc, #316]	; (8001048 <GFX_DrawChar+0x16c>)
 8000f0a:	6809      	ldr	r1, [r1, #0]
 8000f0c:	3101      	adds	r1, #1
 8000f0e:	7809      	ldrb	r1, [r1, #0]
 8000f10:	fb01 f103 	mul.w	r1, r1, r3
 8000f14:	7dfb      	ldrb	r3, [r7, #23]
 8000f16:	440b      	add	r3, r1
 8000f18:	3302      	adds	r3, #2
 8000f1a:	4413      	add	r3, r2
 8000f1c:	781b      	ldrb	r3, [r3, #0]
 8000f1e:	75bb      	strb	r3, [r7, #22]

        for(int8_t j=0; j<font[0]; j++, line >>= 1) // For each pixel in column
 8000f20:	2300      	movs	r3, #0
 8000f22:	757b      	strb	r3, [r7, #21]
 8000f24:	e078      	b.n	8001018 <GFX_DrawChar+0x13c>
        {
            if(line & 1) // Check last pixel in line
 8000f26:	7dbb      	ldrb	r3, [r7, #22]
 8000f28:	f003 0301 	and.w	r3, r3, #1
 8000f2c:	2b00      	cmp	r3, #0
 8000f2e:	d032      	beq.n	8000f96 <GFX_DrawChar+0xba>
            {
            	if(size == 1)
 8000f30:	4b46      	ldr	r3, [pc, #280]	; (800104c <GFX_DrawChar+0x170>)
 8000f32:	781b      	ldrb	r3, [r3, #0]
 8000f34:	2b01      	cmp	r3, #1
 8000f36:	d113      	bne.n	8000f60 <GFX_DrawChar+0x84>
            		GFX_DrawPixel(x+i, y+j, color); // Draw this pixel
 8000f38:	7dfb      	ldrb	r3, [r7, #23]
 8000f3a:	b29a      	uxth	r2, r3
 8000f3c:	68fb      	ldr	r3, [r7, #12]
 8000f3e:	b29b      	uxth	r3, r3
 8000f40:	4413      	add	r3, r2
 8000f42:	b29b      	uxth	r3, r3
 8000f44:	b218      	sxth	r0, r3
 8000f46:	f997 3015 	ldrsb.w	r3, [r7, #21]
 8000f4a:	b29a      	uxth	r2, r3
 8000f4c:	68bb      	ldr	r3, [r7, #8]
 8000f4e:	b29b      	uxth	r3, r3
 8000f50:	4413      	add	r3, r2
 8000f52:	b29b      	uxth	r3, r3
 8000f54:	b21b      	sxth	r3, r3
 8000f56:	79ba      	ldrb	r2, [r7, #6]
 8000f58:	4619      	mov	r1, r3
 8000f5a:	f000 f9cf 	bl	80012fc <SSD1306_DrawPixel>
 8000f5e:	e052      	b.n	8001006 <GFX_DrawChar+0x12a>
            	else
            		GFX_DrawFillRectangle(x+i*size, y+j*size, size, size, color); // Or bigger pixel
 8000f60:	7dfb      	ldrb	r3, [r7, #23]
 8000f62:	4a3a      	ldr	r2, [pc, #232]	; (800104c <GFX_DrawChar+0x170>)
 8000f64:	7812      	ldrb	r2, [r2, #0]
 8000f66:	fb02 f203 	mul.w	r2, r2, r3
 8000f6a:	68fb      	ldr	r3, [r7, #12]
 8000f6c:	18d0      	adds	r0, r2, r3
 8000f6e:	f997 3015 	ldrsb.w	r3, [r7, #21]
 8000f72:	4a36      	ldr	r2, [pc, #216]	; (800104c <GFX_DrawChar+0x170>)
 8000f74:	7812      	ldrb	r2, [r2, #0]
 8000f76:	fb02 f203 	mul.w	r2, r2, r3
 8000f7a:	68bb      	ldr	r3, [r7, #8]
 8000f7c:	18d1      	adds	r1, r2, r3
 8000f7e:	4b33      	ldr	r3, [pc, #204]	; (800104c <GFX_DrawChar+0x170>)
 8000f80:	781b      	ldrb	r3, [r3, #0]
 8000f82:	b29a      	uxth	r2, r3
 8000f84:	4b31      	ldr	r3, [pc, #196]	; (800104c <GFX_DrawChar+0x170>)
 8000f86:	781b      	ldrb	r3, [r3, #0]
 8000f88:	b29c      	uxth	r4, r3
 8000f8a:	79bb      	ldrb	r3, [r7, #6]
 8000f8c:	9300      	str	r3, [sp, #0]
 8000f8e:	4623      	mov	r3, r4
 8000f90:	f000 f95d 	bl	800124e <GFX_DrawFillRectangle>
 8000f94:	e037      	b.n	8001006 <GFX_DrawChar+0x12a>
            }
            else if(background == 0)
 8000f96:	f897 3028 	ldrb.w	r3, [r7, #40]	; 0x28
 8000f9a:	2b00      	cmp	r3, #0
 8000f9c:	d133      	bne.n	8001006 <GFX_DrawChar+0x12a>
            {
            	if(size == 1)
 8000f9e:	4b2b      	ldr	r3, [pc, #172]	; (800104c <GFX_DrawChar+0x170>)
 8000fa0:	781b      	ldrb	r3, [r3, #0]
 8000fa2:	2b01      	cmp	r3, #1
 8000fa4:	d114      	bne.n	8000fd0 <GFX_DrawChar+0xf4>
					GFX_DrawPixel(x+i, y+j, background); // Draw black BG
 8000fa6:	7dfb      	ldrb	r3, [r7, #23]
 8000fa8:	b29a      	uxth	r2, r3
 8000faa:	68fb      	ldr	r3, [r7, #12]
 8000fac:	b29b      	uxth	r3, r3
 8000fae:	4413      	add	r3, r2
 8000fb0:	b29b      	uxth	r3, r3
 8000fb2:	b218      	sxth	r0, r3
 8000fb4:	f997 3015 	ldrsb.w	r3, [r7, #21]
 8000fb8:	b29a      	uxth	r2, r3
 8000fba:	68bb      	ldr	r3, [r7, #8]
 8000fbc:	b29b      	uxth	r3, r3
 8000fbe:	4413      	add	r3, r2
 8000fc0:	b29b      	uxth	r3, r3
 8000fc2:	b21b      	sxth	r3, r3
 8000fc4:	f897 2028 	ldrb.w	r2, [r7, #40]	; 0x28
 8000fc8:	4619      	mov	r1, r3
 8000fca:	f000 f997 	bl	80012fc <SSD1306_DrawPixel>
 8000fce:	e01a      	b.n	8001006 <GFX_DrawChar+0x12a>
				else
					GFX_DrawFillRectangle(x+i*size, y+j*size, size, size, background); // Or bigger
 8000fd0:	7dfb      	ldrb	r3, [r7, #23]
 8000fd2:	4a1e      	ldr	r2, [pc, #120]	; (800104c <GFX_DrawChar+0x170>)
 8000fd4:	7812      	ldrb	r2, [r2, #0]
 8000fd6:	fb02 f203 	mul.w	r2, r2, r3
 8000fda:	68fb      	ldr	r3, [r7, #12]
 8000fdc:	18d0      	adds	r0, r2, r3
 8000fde:	f997 3015 	ldrsb.w	r3, [r7, #21]
 8000fe2:	4a1a      	ldr	r2, [pc, #104]	; (800104c <GFX_DrawChar+0x170>)
 8000fe4:	7812      	ldrb	r2, [r2, #0]
 8000fe6:	fb02 f203 	mul.w	r2, r2, r3
 8000fea:	68bb      	ldr	r3, [r7, #8]
 8000fec:	18d1      	adds	r1, r2, r3
 8000fee:	4b17      	ldr	r3, [pc, #92]	; (800104c <GFX_DrawChar+0x170>)
 8000ff0:	781b      	ldrb	r3, [r3, #0]
 8000ff2:	b29a      	uxth	r2, r3
 8000ff4:	4b15      	ldr	r3, [pc, #84]	; (800104c <GFX_DrawChar+0x170>)
 8000ff6:	781b      	ldrb	r3, [r3, #0]
 8000ff8:	b29c      	uxth	r4, r3
 8000ffa:	f897 3028 	ldrb.w	r3, [r7, #40]	; 0x28
 8000ffe:	9300      	str	r3, [sp, #0]
 8001000:	4623      	mov	r3, r4
 8001002:	f000 f924 	bl	800124e <GFX_DrawFillRectangle>
        for(int8_t j=0; j<font[0]; j++, line >>= 1) // For each pixel in column
 8001006:	f997 3015 	ldrsb.w	r3, [r7, #21]
 800100a:	b2db      	uxtb	r3, r3
 800100c:	3301      	adds	r3, #1
 800100e:	b2db      	uxtb	r3, r3
 8001010:	757b      	strb	r3, [r7, #21]
 8001012:	7dbb      	ldrb	r3, [r7, #22]
 8001014:	085b      	lsrs	r3, r3, #1
 8001016:	75bb      	strb	r3, [r7, #22]
 8001018:	f997 3015 	ldrsb.w	r3, [r7, #21]
 800101c:	4a0a      	ldr	r2, [pc, #40]	; (8001048 <GFX_DrawChar+0x16c>)
 800101e:	6812      	ldr	r2, [r2, #0]
 8001020:	7812      	ldrb	r2, [r2, #0]
 8001022:	4293      	cmp	r3, r2
 8001024:	f6ff af7f 	blt.w	8000f26 <GFX_DrawChar+0x4a>
	for(uint8_t i=0; i<font[1]; i++ ) // Each column (Width)
 8001028:	7dfb      	ldrb	r3, [r7, #23]
 800102a:	3301      	adds	r3, #1
 800102c:	75fb      	strb	r3, [r7, #23]
 800102e:	4b06      	ldr	r3, [pc, #24]	; (8001048 <GFX_DrawChar+0x16c>)
 8001030:	681b      	ldr	r3, [r3, #0]
 8001032:	3301      	adds	r3, #1
 8001034:	781b      	ldrb	r3, [r3, #0]
 8001036:	7dfa      	ldrb	r2, [r7, #23]
 8001038:	429a      	cmp	r2, r3
 800103a:	f4ff af61 	bcc.w	8000f00 <GFX_DrawChar+0x24>
 800103e:	e000      	b.n	8001042 <GFX_DrawChar+0x166>
	if(chr > 0x7E) return; // chr > '~'
 8001040:	bf00      	nop
            }
        }
    }
}
 8001042:	371c      	adds	r7, #28
 8001044:	46bd      	mov	sp, r7
 8001046:	bd90      	pop	{r4, r7, pc}
 8001048:	20004d38 	.word	0x20004d38
 800104c:	20000000 	.word	0x20000000

08001050 <GFX_DrawString>:

void GFX_DrawString(int x, int y, char* str, uint8_t color, uint8_t background)
{
 8001050:	b580      	push	{r7, lr}
 8001052:	b088      	sub	sp, #32
 8001054:	af02      	add	r7, sp, #8
 8001056:	60f8      	str	r0, [r7, #12]
 8001058:	60b9      	str	r1, [r7, #8]
 800105a:	607a      	str	r2, [r7, #4]
 800105c:	70fb      	strb	r3, [r7, #3]
	int x_tmp = x;
 800105e:	68fb      	ldr	r3, [r7, #12]
 8001060:	617b      	str	r3, [r7, #20]

	char znak;
	znak = *str;
 8001062:	687b      	ldr	r3, [r7, #4]
 8001064:	781b      	ldrb	r3, [r3, #0]
 8001066:	74fb      	strb	r3, [r7, #19]

	while(*str++)
 8001068:	e03e      	b.n	80010e8 <GFX_DrawString+0x98>
	{
		GFX_DrawChar(x_tmp, y, znak, color, background); // Draw current char
 800106a:	78f9      	ldrb	r1, [r7, #3]
 800106c:	7cfa      	ldrb	r2, [r7, #19]
 800106e:	f897 3020 	ldrb.w	r3, [r7, #32]
 8001072:	9300      	str	r3, [sp, #0]
 8001074:	460b      	mov	r3, r1
 8001076:	68b9      	ldr	r1, [r7, #8]
 8001078:	6978      	ldr	r0, [r7, #20]
 800107a:	f7ff ff2f 	bl	8000edc <GFX_DrawChar>

		x_tmp += ((uint8_t)font[1] * size) + 1; // Move X drawing pointer do char width + 1 (space)
 800107e:	4b1f      	ldr	r3, [pc, #124]	; (80010fc <GFX_DrawString+0xac>)
 8001080:	681b      	ldr	r3, [r3, #0]
 8001082:	3301      	adds	r3, #1
 8001084:	781b      	ldrb	r3, [r3, #0]
 8001086:	461a      	mov	r2, r3
 8001088:	4b1d      	ldr	r3, [pc, #116]	; (8001100 <GFX_DrawString+0xb0>)
 800108a:	781b      	ldrb	r3, [r3, #0]
 800108c:	fb03 f302 	mul.w	r3, r3, r2
 8001090:	3301      	adds	r3, #1
 8001092:	697a      	ldr	r2, [r7, #20]
 8001094:	4413      	add	r3, r2
 8001096:	617b      	str	r3, [r7, #20]

		if(background == 0) // Draw black space if needed
 8001098:	f897 3020 	ldrb.w	r3, [r7, #32]
 800109c:	2b00      	cmp	r3, #0
 800109e:	d120      	bne.n	80010e2 <GFX_DrawString+0x92>
		{
			for(uint8_t i=0; i<(font[0]*size); i++)
 80010a0:	2300      	movs	r3, #0
 80010a2:	74bb      	strb	r3, [r7, #18]
 80010a4:	e012      	b.n	80010cc <GFX_DrawString+0x7c>
			{
				GFX_DrawPixel(x_tmp-1, y+i, PIXEL_BLACK);
 80010a6:	697b      	ldr	r3, [r7, #20]
 80010a8:	b29b      	uxth	r3, r3
 80010aa:	3b01      	subs	r3, #1
 80010ac:	b29b      	uxth	r3, r3
 80010ae:	b218      	sxth	r0, r3
 80010b0:	7cbb      	ldrb	r3, [r7, #18]
 80010b2:	b29a      	uxth	r2, r3
 80010b4:	68bb      	ldr	r3, [r7, #8]
 80010b6:	b29b      	uxth	r3, r3
 80010b8:	4413      	add	r3, r2
 80010ba:	b29b      	uxth	r3, r3
 80010bc:	b21b      	sxth	r3, r3
 80010be:	2200      	movs	r2, #0
 80010c0:	4619      	mov	r1, r3
 80010c2:	f000 f91b 	bl	80012fc <SSD1306_DrawPixel>
			for(uint8_t i=0; i<(font[0]*size); i++)
 80010c6:	7cbb      	ldrb	r3, [r7, #18]
 80010c8:	3301      	adds	r3, #1
 80010ca:	74bb      	strb	r3, [r7, #18]
 80010cc:	7cba      	ldrb	r2, [r7, #18]
 80010ce:	4b0b      	ldr	r3, [pc, #44]	; (80010fc <GFX_DrawString+0xac>)
 80010d0:	681b      	ldr	r3, [r3, #0]
 80010d2:	781b      	ldrb	r3, [r3, #0]
 80010d4:	4619      	mov	r1, r3
 80010d6:	4b0a      	ldr	r3, [pc, #40]	; (8001100 <GFX_DrawString+0xb0>)
 80010d8:	781b      	ldrb	r3, [r3, #0]
 80010da:	fb03 f301 	mul.w	r3, r3, r1
 80010de:	429a      	cmp	r2, r3
 80010e0:	dbe1      	blt.n	80010a6 <GFX_DrawString+0x56>
			}
		}

		znak = *str; // Next char
 80010e2:	687b      	ldr	r3, [r7, #4]
 80010e4:	781b      	ldrb	r3, [r3, #0]
 80010e6:	74fb      	strb	r3, [r7, #19]
	while(*str++)
 80010e8:	687b      	ldr	r3, [r7, #4]
 80010ea:	1c5a      	adds	r2, r3, #1
 80010ec:	607a      	str	r2, [r7, #4]
 80010ee:	781b      	ldrb	r3, [r3, #0]
 80010f0:	2b00      	cmp	r3, #0
 80010f2:	d1ba      	bne.n	800106a <GFX_DrawString+0x1a>
	}
}
 80010f4:	bf00      	nop
 80010f6:	3718      	adds	r7, #24
 80010f8:	46bd      	mov	sp, r7
 80010fa:	bd80      	pop	{r7, pc}
 80010fc:	20004d38 	.word	0x20004d38
 8001100:	20000000 	.word	0x20000000

08001104 <GFX_WriteLine>:
#endif
#if USING_LINES == 1
void GFX_WriteLine(int x_start, int y_start, int x_end, int y_end, uint8_t color)
{
 8001104:	b580      	push	{r7, lr}
 8001106:	b08c      	sub	sp, #48	; 0x30
 8001108:	af00      	add	r7, sp, #0
 800110a:	60f8      	str	r0, [r7, #12]
 800110c:	60b9      	str	r1, [r7, #8]
 800110e:	607a      	str	r2, [r7, #4]
 8001110:	603b      	str	r3, [r7, #0]
	int16_t steep = abs(y_end - y_start) > abs(x_end - x_start);
 8001112:	683a      	ldr	r2, [r7, #0]
 8001114:	68bb      	ldr	r3, [r7, #8]
 8001116:	1ad3      	subs	r3, r2, r3
 8001118:	ea83 72e3 	eor.w	r2, r3, r3, asr #31
 800111c:	eba2 72e3 	sub.w	r2, r2, r3, asr #31
 8001120:	6879      	ldr	r1, [r7, #4]
 8001122:	68fb      	ldr	r3, [r7, #12]
 8001124:	1acb      	subs	r3, r1, r3
 8001126:	2b00      	cmp	r3, #0
 8001128:	bfb8      	it	lt
 800112a:	425b      	neglt	r3, r3
 800112c:	429a      	cmp	r2, r3
 800112e:	bfcc      	ite	gt
 8001130:	2301      	movgt	r3, #1
 8001132:	2300      	movle	r3, #0
 8001134:	b2db      	uxtb	r3, r3
 8001136:	857b      	strh	r3, [r7, #42]	; 0x2a

	    if (steep) {
 8001138:	f9b7 302a 	ldrsh.w	r3, [r7, #42]	; 0x2a
 800113c:	2b00      	cmp	r3, #0
 800113e:	d00b      	beq.n	8001158 <GFX_WriteLine+0x54>
	        _swap_int(x_start, y_start);
 8001140:	68fb      	ldr	r3, [r7, #12]
 8001142:	627b      	str	r3, [r7, #36]	; 0x24
 8001144:	68bb      	ldr	r3, [r7, #8]
 8001146:	60fb      	str	r3, [r7, #12]
 8001148:	6a7b      	ldr	r3, [r7, #36]	; 0x24
 800114a:	60bb      	str	r3, [r7, #8]
	        _swap_int(x_end, y_end);
 800114c:	687b      	ldr	r3, [r7, #4]
 800114e:	623b      	str	r3, [r7, #32]
 8001150:	683b      	ldr	r3, [r7, #0]
 8001152:	607b      	str	r3, [r7, #4]
 8001154:	6a3b      	ldr	r3, [r7, #32]
 8001156:	603b      	str	r3, [r7, #0]
	    }

	    if (x_start > x_end) {
 8001158:	68fa      	ldr	r2, [r7, #12]
 800115a:	687b      	ldr	r3, [r7, #4]
 800115c:	429a      	cmp	r2, r3
 800115e:	dd0b      	ble.n	8001178 <GFX_WriteLine+0x74>
	        _swap_int(x_start, x_end);
 8001160:	68fb      	ldr	r3, [r7, #12]
 8001162:	61fb      	str	r3, [r7, #28]
 8001164:	687b      	ldr	r3, [r7, #4]
 8001166:	60fb      	str	r3, [r7, #12]
 8001168:	69fb      	ldr	r3, [r7, #28]
 800116a:	607b      	str	r3, [r7, #4]
	        _swap_int(y_start, y_end);
 800116c:	68bb      	ldr	r3, [r7, #8]
 800116e:	61bb      	str	r3, [r7, #24]
 8001170:	683b      	ldr	r3, [r7, #0]
 8001172:	60bb      	str	r3, [r7, #8]
 8001174:	69bb      	ldr	r3, [r7, #24]
 8001176:	603b      	str	r3, [r7, #0]
	    }

	    int16_t dx, dy;
	    dx = x_end - x_start;
 8001178:	687b      	ldr	r3, [r7, #4]
 800117a:	b29a      	uxth	r2, r3
 800117c:	68fb      	ldr	r3, [r7, #12]
 800117e:	b29b      	uxth	r3, r3
 8001180:	1ad3      	subs	r3, r2, r3
 8001182:	b29b      	uxth	r3, r3
 8001184:	82fb      	strh	r3, [r7, #22]
	    dy = abs(y_end - y_start);
 8001186:	683a      	ldr	r2, [r7, #0]
 8001188:	68bb      	ldr	r3, [r7, #8]
 800118a:	1ad3      	subs	r3, r2, r3
 800118c:	2b00      	cmp	r3, #0
 800118e:	bfb8      	it	lt
 8001190:	425b      	neglt	r3, r3
 8001192:	82bb      	strh	r3, [r7, #20]

	    int16_t err = dx / 2;
 8001194:	f9b7 3016 	ldrsh.w	r3, [r7, #22]
 8001198:	0fda      	lsrs	r2, r3, #31
 800119a:	4413      	add	r3, r2
 800119c:	105b      	asrs	r3, r3, #1
 800119e:	85fb      	strh	r3, [r7, #46]	; 0x2e
	    int16_t ystep;

	    if (y_start < y_end) {
 80011a0:	68ba      	ldr	r2, [r7, #8]
 80011a2:	683b      	ldr	r3, [r7, #0]
 80011a4:	429a      	cmp	r2, r3
 80011a6:	da02      	bge.n	80011ae <GFX_WriteLine+0xaa>
	        ystep = 1;
 80011a8:	2301      	movs	r3, #1
 80011aa:	85bb      	strh	r3, [r7, #44]	; 0x2c
 80011ac:	e030      	b.n	8001210 <GFX_WriteLine+0x10c>
	    } else {
	        ystep = -1;
 80011ae:	f64f 73ff 	movw	r3, #65535	; 0xffff
 80011b2:	85bb      	strh	r3, [r7, #44]	; 0x2c
	    }

	    for (; x_start<=x_end; x_start++) {
 80011b4:	e02c      	b.n	8001210 <GFX_WriteLine+0x10c>
	        if (steep) {
 80011b6:	f9b7 302a 	ldrsh.w	r3, [r7, #42]	; 0x2a
 80011ba:	2b00      	cmp	r3, #0
 80011bc:	d009      	beq.n	80011d2 <GFX_WriteLine+0xce>
	        	GFX_DrawPixel(y_start, x_start, color);
 80011be:	68bb      	ldr	r3, [r7, #8]
 80011c0:	b21b      	sxth	r3, r3
 80011c2:	68fa      	ldr	r2, [r7, #12]
 80011c4:	b211      	sxth	r1, r2
 80011c6:	f897 2038 	ldrb.w	r2, [r7, #56]	; 0x38
 80011ca:	4618      	mov	r0, r3
 80011cc:	f000 f896 	bl	80012fc <SSD1306_DrawPixel>
 80011d0:	e008      	b.n	80011e4 <GFX_WriteLine+0xe0>
	        } else {
	        	GFX_DrawPixel(x_start, y_start, color);
 80011d2:	68fb      	ldr	r3, [r7, #12]
 80011d4:	b21b      	sxth	r3, r3
 80011d6:	68ba      	ldr	r2, [r7, #8]
 80011d8:	b211      	sxth	r1, r2
 80011da:	f897 2038 	ldrb.w	r2, [r7, #56]	; 0x38
 80011de:	4618      	mov	r0, r3
 80011e0:	f000 f88c 	bl	80012fc <SSD1306_DrawPixel>
	        }
	        err -= dy;
 80011e4:	8dfa      	ldrh	r2, [r7, #46]	; 0x2e
 80011e6:	8abb      	ldrh	r3, [r7, #20]
 80011e8:	1ad3      	subs	r3, r2, r3
 80011ea:	b29b      	uxth	r3, r3
 80011ec:	85fb      	strh	r3, [r7, #46]	; 0x2e
	        if (err < 0) {
 80011ee:	f9b7 302e 	ldrsh.w	r3, [r7, #46]	; 0x2e
 80011f2:	2b00      	cmp	r3, #0
 80011f4:	da09      	bge.n	800120a <GFX_WriteLine+0x106>
	            y_start += ystep;
 80011f6:	f9b7 302c 	ldrsh.w	r3, [r7, #44]	; 0x2c
 80011fa:	68ba      	ldr	r2, [r7, #8]
 80011fc:	4413      	add	r3, r2
 80011fe:	60bb      	str	r3, [r7, #8]
	            err += dx;
 8001200:	8dfa      	ldrh	r2, [r7, #46]	; 0x2e
 8001202:	8afb      	ldrh	r3, [r7, #22]
 8001204:	4413      	add	r3, r2
 8001206:	b29b      	uxth	r3, r3
 8001208:	85fb      	strh	r3, [r7, #46]	; 0x2e
	    for (; x_start<=x_end; x_start++) {
 800120a:	68fb      	ldr	r3, [r7, #12]
 800120c:	3301      	adds	r3, #1
 800120e:	60fb      	str	r3, [r7, #12]
 8001210:	68fa      	ldr	r2, [r7, #12]
 8001212:	687b      	ldr	r3, [r7, #4]
 8001214:	429a      	cmp	r2, r3
 8001216:	ddce      	ble.n	80011b6 <GFX_WriteLine+0xb2>
	        }
	    }
}
 8001218:	bf00      	nop
 800121a:	3730      	adds	r7, #48	; 0x30
 800121c:	46bd      	mov	sp, r7
 800121e:	bd80      	pop	{r7, pc}

08001220 <GFX_DrawFastVLine>:

void GFX_DrawFastVLine(int x_start, int y_start, int h, uint8_t color)
{
 8001220:	b580      	push	{r7, lr}
 8001222:	b086      	sub	sp, #24
 8001224:	af02      	add	r7, sp, #8
 8001226:	60f8      	str	r0, [r7, #12]
 8001228:	60b9      	str	r1, [r7, #8]
 800122a:	607a      	str	r2, [r7, #4]
 800122c:	70fb      	strb	r3, [r7, #3]
	GFX_WriteLine(x_start, y_start, x_start, y_start+h-1, color);
 800122e:	68ba      	ldr	r2, [r7, #8]
 8001230:	687b      	ldr	r3, [r7, #4]
 8001232:	4413      	add	r3, r2
 8001234:	1e5a      	subs	r2, r3, #1
 8001236:	78fb      	ldrb	r3, [r7, #3]
 8001238:	9300      	str	r3, [sp, #0]
 800123a:	4613      	mov	r3, r2
 800123c:	68fa      	ldr	r2, [r7, #12]
 800123e:	68b9      	ldr	r1, [r7, #8]
 8001240:	68f8      	ldr	r0, [r7, #12]
 8001242:	f7ff ff5f 	bl	8001104 <GFX_WriteLine>
}
 8001246:	bf00      	nop
 8001248:	3710      	adds	r7, #16
 800124a:	46bd      	mov	sp, r7
 800124c:	bd80      	pop	{r7, pc}

0800124e <GFX_DrawFillRectangle>:

}
#endif
#if USING_FILL_RECTANGLE == 1
void GFX_DrawFillRectangle(int x, int y, uint16_t w, uint16_t h, uint8_t color)
{
 800124e:	b580      	push	{r7, lr}
 8001250:	b086      	sub	sp, #24
 8001252:	af00      	add	r7, sp, #0
 8001254:	60f8      	str	r0, [r7, #12]
 8001256:	60b9      	str	r1, [r7, #8]
 8001258:	4611      	mov	r1, r2
 800125a:	461a      	mov	r2, r3
 800125c:	460b      	mov	r3, r1
 800125e:	80fb      	strh	r3, [r7, #6]
 8001260:	4613      	mov	r3, r2
 8001262:	80bb      	strh	r3, [r7, #4]
    for (int i=x; i<x+w; i++) {
 8001264:	68fb      	ldr	r3, [r7, #12]
 8001266:	617b      	str	r3, [r7, #20]
 8001268:	e009      	b.n	800127e <GFX_DrawFillRectangle+0x30>
    	GFX_DrawFastVLine(i, y, h, color);
 800126a:	88ba      	ldrh	r2, [r7, #4]
 800126c:	f897 3020 	ldrb.w	r3, [r7, #32]
 8001270:	68b9      	ldr	r1, [r7, #8]
 8001272:	6978      	ldr	r0, [r7, #20]
 8001274:	f7ff ffd4 	bl	8001220 <GFX_DrawFastVLine>
    for (int i=x; i<x+w; i++) {
 8001278:	697b      	ldr	r3, [r7, #20]
 800127a:	3301      	adds	r3, #1
 800127c:	617b      	str	r3, [r7, #20]
 800127e:	88fa      	ldrh	r2, [r7, #6]
 8001280:	68fb      	ldr	r3, [r7, #12]
 8001282:	4413      	add	r3, r2
 8001284:	697a      	ldr	r2, [r7, #20]
 8001286:	429a      	cmp	r2, r3
 8001288:	dbef      	blt.n	800126a <GFX_DrawFillRectangle+0x1c>
    }

}
 800128a:	bf00      	nop
 800128c:	3718      	adds	r7, #24
 800128e:	46bd      	mov	sp, r7
 8001290:	bd80      	pop	{r7, pc}
	...

08001294 <SSD1306_Command>:
I2C_HandleTypeDef *oled_i2c;

static uint8_t buffer[SSD1306_BUFFER_SIZE];

void SSD1306_Command(uint8_t Command)
{
 8001294:	b580      	push	{r7, lr}
 8001296:	b086      	sub	sp, #24
 8001298:	af04      	add	r7, sp, #16
 800129a:	4603      	mov	r3, r0
 800129c:	71fb      	strb	r3, [r7, #7]
	HAL_I2C_Mem_Write(oled_i2c, (SSD1306_ADDRESS<<1), 0x00, 1, &Command, 1, SSD1306_TIMEOUT);
 800129e:	4b09      	ldr	r3, [pc, #36]	; (80012c4 <SSD1306_Command+0x30>)
 80012a0:	6818      	ldr	r0, [r3, #0]
 80012a2:	f44f 737a 	mov.w	r3, #1000	; 0x3e8
 80012a6:	9302      	str	r3, [sp, #8]
 80012a8:	2301      	movs	r3, #1
 80012aa:	9301      	str	r3, [sp, #4]
 80012ac:	1dfb      	adds	r3, r7, #7
 80012ae:	9300      	str	r3, [sp, #0]
 80012b0:	2301      	movs	r3, #1
 80012b2:	2200      	movs	r2, #0
 80012b4:	2178      	movs	r1, #120	; 0x78
 80012b6:	f003 f8e5 	bl	8004484 <HAL_I2C_Mem_Write>
}
 80012ba:	bf00      	nop
 80012bc:	3708      	adds	r7, #8
 80012be:	46bd      	mov	sp, r7
 80012c0:	bd80      	pop	{r7, pc}
 80012c2:	bf00      	nop
 80012c4:	20004d3c 	.word	0x20004d3c

080012c8 <SSD1306_Data>:

void SSD1306_Data(uint8_t *Data, uint16_t Size)
{
 80012c8:	b580      	push	{r7, lr}
 80012ca:	b086      	sub	sp, #24
 80012cc:	af04      	add	r7, sp, #16
 80012ce:	6078      	str	r0, [r7, #4]
 80012d0:	460b      	mov	r3, r1
 80012d2:	807b      	strh	r3, [r7, #2]
	if(oled_i2c->hdmatx->State == HAL_DMA_STATE_READY)
	{
		HAL_I2C_Mem_Write_DMA(oled_i2c, (SSD1306_ADDRESS<<1), 0x40, 1, Data, Size);
	}
#else
	HAL_I2C_Mem_Write(oled_i2c, (SSD1306_ADDRESS<<1), 0x40, 1, Data, Size, SSD1306_TIMEOUT);
 80012d4:	4b08      	ldr	r3, [pc, #32]	; (80012f8 <SSD1306_Data+0x30>)
 80012d6:	6818      	ldr	r0, [r3, #0]
 80012d8:	f44f 737a 	mov.w	r3, #1000	; 0x3e8
 80012dc:	9302      	str	r3, [sp, #8]
 80012de:	887b      	ldrh	r3, [r7, #2]
 80012e0:	9301      	str	r3, [sp, #4]
 80012e2:	687b      	ldr	r3, [r7, #4]
 80012e4:	9300      	str	r3, [sp, #0]
 80012e6:	2301      	movs	r3, #1
 80012e8:	2240      	movs	r2, #64	; 0x40
 80012ea:	2178      	movs	r1, #120	; 0x78
 80012ec:	f003 f8ca 	bl	8004484 <HAL_I2C_Mem_Write>
#endif
}
 80012f0:	bf00      	nop
 80012f2:	3708      	adds	r7, #8
 80012f4:	46bd      	mov	sp, r7
 80012f6:	bd80      	pop	{r7, pc}
 80012f8:	20004d3c 	.word	0x20004d3c

080012fc <SSD1306_DrawPixel>:
//
// Functions
//

void SSD1306_DrawPixel(int16_t x, int16_t y, uint8_t Color)
{
 80012fc:	b480      	push	{r7}
 80012fe:	b083      	sub	sp, #12
 8001300:	af00      	add	r7, sp, #0
 8001302:	4603      	mov	r3, r0
 8001304:	80fb      	strh	r3, [r7, #6]
 8001306:	460b      	mov	r3, r1
 8001308:	80bb      	strh	r3, [r7, #4]
 800130a:	4613      	mov	r3, r2
 800130c:	70fb      	strb	r3, [r7, #3]
	if((x < 0) || (x >= SSD1306_LCDWIDTH) || (y < 0) || (y >= SSD1306_LCDHEIGHT))
 800130e:	f9b7 3006 	ldrsh.w	r3, [r7, #6]
 8001312:	2b00      	cmp	r3, #0
 8001314:	db79      	blt.n	800140a <SSD1306_DrawPixel+0x10e>
 8001316:	f9b7 3006 	ldrsh.w	r3, [r7, #6]
 800131a:	2b7f      	cmp	r3, #127	; 0x7f
 800131c:	dc75      	bgt.n	800140a <SSD1306_DrawPixel+0x10e>
 800131e:	f9b7 3004 	ldrsh.w	r3, [r7, #4]
 8001322:	2b00      	cmp	r3, #0
 8001324:	db71      	blt.n	800140a <SSD1306_DrawPixel+0x10e>
 8001326:	f9b7 3004 	ldrsh.w	r3, [r7, #4]
 800132a:	2b3f      	cmp	r3, #63	; 0x3f
 800132c:	dc6d      	bgt.n	800140a <SSD1306_DrawPixel+0x10e>
	  return;

    switch(Color)
 800132e:	78fb      	ldrb	r3, [r7, #3]
 8001330:	2b01      	cmp	r3, #1
 8001332:	d004      	beq.n	800133e <SSD1306_DrawPixel+0x42>
 8001334:	2b02      	cmp	r3, #2
 8001336:	d046      	beq.n	80013c6 <SSD1306_DrawPixel+0xca>
 8001338:	2b00      	cmp	r3, #0
 800133a:	d021      	beq.n	8001380 <SSD1306_DrawPixel+0x84>
 800133c:	e066      	b.n	800140c <SSD1306_DrawPixel+0x110>
    {
    case SSD1306_WHITE:
      buffer[x + (y / 8) * SSD1306_LCDWIDTH] |= (1 << (y & 7));
 800133e:	f9b7 2006 	ldrsh.w	r2, [r7, #6]
 8001342:	f9b7 3004 	ldrsh.w	r3, [r7, #4]
 8001346:	2b00      	cmp	r3, #0
 8001348:	da00      	bge.n	800134c <SSD1306_DrawPixel+0x50>
 800134a:	3307      	adds	r3, #7
 800134c:	10db      	asrs	r3, r3, #3
 800134e:	b218      	sxth	r0, r3
 8001350:	4603      	mov	r3, r0
 8001352:	01db      	lsls	r3, r3, #7
 8001354:	4413      	add	r3, r2
 8001356:	4a30      	ldr	r2, [pc, #192]	; (8001418 <SSD1306_DrawPixel+0x11c>)
 8001358:	5cd3      	ldrb	r3, [r2, r3]
 800135a:	b25a      	sxtb	r2, r3
 800135c:	88bb      	ldrh	r3, [r7, #4]
 800135e:	f003 0307 	and.w	r3, r3, #7
 8001362:	2101      	movs	r1, #1
 8001364:	fa01 f303 	lsl.w	r3, r1, r3
 8001368:	b25b      	sxtb	r3, r3
 800136a:	4313      	orrs	r3, r2
 800136c:	b259      	sxtb	r1, r3
 800136e:	f9b7 2006 	ldrsh.w	r2, [r7, #6]
 8001372:	4603      	mov	r3, r0
 8001374:	01db      	lsls	r3, r3, #7
 8001376:	4413      	add	r3, r2
 8001378:	b2c9      	uxtb	r1, r1
 800137a:	4a27      	ldr	r2, [pc, #156]	; (8001418 <SSD1306_DrawPixel+0x11c>)
 800137c:	54d1      	strb	r1, [r2, r3]
      break;
 800137e:	e045      	b.n	800140c <SSD1306_DrawPixel+0x110>
    case SSD1306_BLACK:
      buffer[x + (y / 8) * SSD1306_LCDWIDTH] &= ~(1 << (y & 7));
 8001380:	f9b7 2006 	ldrsh.w	r2, [r7, #6]
 8001384:	f9b7 3004 	ldrsh.w	r3, [r7, #4]
 8001388:	2b00      	cmp	r3, #0
 800138a:	da00      	bge.n	800138e <SSD1306_DrawPixel+0x92>
 800138c:	3307      	adds	r3, #7
 800138e:	10db      	asrs	r3, r3, #3
 8001390:	b218      	sxth	r0, r3
 8001392:	4603      	mov	r3, r0
 8001394:	01db      	lsls	r3, r3, #7
 8001396:	4413      	add	r3, r2
 8001398:	4a1f      	ldr	r2, [pc, #124]	; (8001418 <SSD1306_DrawPixel+0x11c>)
 800139a:	5cd3      	ldrb	r3, [r2, r3]
 800139c:	b25a      	sxtb	r2, r3
 800139e:	88bb      	ldrh	r3, [r7, #4]
 80013a0:	f003 0307 	and.w	r3, r3, #7
 80013a4:	2101      	movs	r1, #1
 80013a6:	fa01 f303 	lsl.w	r3, r1, r3
 80013aa:	b25b      	sxtb	r3, r3
 80013ac:	43db      	mvns	r3, r3
 80013ae:	b25b      	sxtb	r3, r3
 80013b0:	4013      	ands	r3, r2
 80013b2:	b259      	sxtb	r1, r3
 80013b4:	f9b7 2006 	ldrsh.w	r2, [r7, #6]
 80013b8:	4603      	mov	r3, r0
 80013ba:	01db      	lsls	r3, r3, #7
 80013bc:	4413      	add	r3, r2
 80013be:	b2c9      	uxtb	r1, r1
 80013c0:	4a15      	ldr	r2, [pc, #84]	; (8001418 <SSD1306_DrawPixel+0x11c>)
 80013c2:	54d1      	strb	r1, [r2, r3]
      break;
 80013c4:	e022      	b.n	800140c <SSD1306_DrawPixel+0x110>
    case SSD1306_INVERSE:
      buffer[x + (y / 8) * SSD1306_LCDWIDTH] ^= (1 << (y & 7));
 80013c6:	f9b7 2006 	ldrsh.w	r2, [r7, #6]
 80013ca:	f9b7 3004 	ldrsh.w	r3, [r7, #4]
 80013ce:	2b00      	cmp	r3, #0
 80013d0:	da00      	bge.n	80013d4 <SSD1306_DrawPixel+0xd8>
 80013d2:	3307      	adds	r3, #7
 80013d4:	10db      	asrs	r3, r3, #3
 80013d6:	b218      	sxth	r0, r3
 80013d8:	4603      	mov	r3, r0
 80013da:	01db      	lsls	r3, r3, #7
 80013dc:	4413      	add	r3, r2
 80013de:	4a0e      	ldr	r2, [pc, #56]	; (8001418 <SSD1306_DrawPixel+0x11c>)
 80013e0:	5cd3      	ldrb	r3, [r2, r3]
 80013e2:	b25a      	sxtb	r2, r3
 80013e4:	88bb      	ldrh	r3, [r7, #4]
 80013e6:	f003 0307 	and.w	r3, r3, #7
 80013ea:	2101      	movs	r1, #1
 80013ec:	fa01 f303 	lsl.w	r3, r1, r3
 80013f0:	b25b      	sxtb	r3, r3
 80013f2:	4053      	eors	r3, r2
 80013f4:	b259      	sxtb	r1, r3
 80013f6:	f9b7 2006 	ldrsh.w	r2, [r7, #6]
 80013fa:	4603      	mov	r3, r0
 80013fc:	01db      	lsls	r3, r3, #7
 80013fe:	4413      	add	r3, r2
 8001400:	b2c9      	uxtb	r1, r1
 8001402:	4a05      	ldr	r2, [pc, #20]	; (8001418 <SSD1306_DrawPixel+0x11c>)
 8001404:	54d1      	strb	r1, [r2, r3]
      break;
 8001406:	bf00      	nop
 8001408:	e000      	b.n	800140c <SSD1306_DrawPixel+0x110>
	  return;
 800140a:	bf00      	nop
    }
}
 800140c:	370c      	adds	r7, #12
 800140e:	46bd      	mov	sp, r7
 8001410:	f85d 7b04 	ldr.w	r7, [sp], #4
 8001414:	4770      	bx	lr
 8001416:	bf00      	nop
 8001418:	20000030 	.word	0x20000030

0800141c <SSD1306_Clear>:

void SSD1306_Clear(uint8_t Color)
{
 800141c:	b580      	push	{r7, lr}
 800141e:	b082      	sub	sp, #8
 8001420:	af00      	add	r7, sp, #0
 8001422:	4603      	mov	r3, r0
 8001424:	71fb      	strb	r3, [r7, #7]
	switch(Color)
 8001426:	79fb      	ldrb	r3, [r7, #7]
 8001428:	2b00      	cmp	r3, #0
 800142a:	d009      	beq.n	8001440 <SSD1306_Clear+0x24>
 800142c:	2b01      	cmp	r3, #1
 800142e:	d000      	beq.n	8001432 <SSD1306_Clear+0x16>

	case BLACK:
		memset(buffer, 0x00, SSD1306_BUFFER_SIZE);
		break;
	}
}
 8001430:	e00d      	b.n	800144e <SSD1306_Clear+0x32>
		memset(buffer, 0xFF, SSD1306_BUFFER_SIZE);
 8001432:	f44f 6280 	mov.w	r2, #1024	; 0x400
 8001436:	21ff      	movs	r1, #255	; 0xff
 8001438:	4807      	ldr	r0, [pc, #28]	; (8001458 <SSD1306_Clear+0x3c>)
 800143a:	f008 fbd6 	bl	8009bea <memset>
		break;
 800143e:	e006      	b.n	800144e <SSD1306_Clear+0x32>
		memset(buffer, 0x00, SSD1306_BUFFER_SIZE);
 8001440:	f44f 6280 	mov.w	r2, #1024	; 0x400
 8001444:	2100      	movs	r1, #0
 8001446:	4804      	ldr	r0, [pc, #16]	; (8001458 <SSD1306_Clear+0x3c>)
 8001448:	f008 fbcf 	bl	8009bea <memset>
		break;
 800144c:	bf00      	nop
}
 800144e:	bf00      	nop
 8001450:	3708      	adds	r7, #8
 8001452:	46bd      	mov	sp, r7
 8001454:	bd80      	pop	{r7, pc}
 8001456:	bf00      	nop
 8001458:	20000030 	.word	0x20000030

0800145c <SSD1306_Display>:

void SSD1306_Display(void)
{
 800145c:	b580      	push	{r7, lr}
 800145e:	af00      	add	r7, sp, #0
	SSD1306_Command(SSD1306_PAGEADDR);
 8001460:	2022      	movs	r0, #34	; 0x22
 8001462:	f7ff ff17 	bl	8001294 <SSD1306_Command>
	SSD1306_Command(0);                      // Page start address
 8001466:	2000      	movs	r0, #0
 8001468:	f7ff ff14 	bl	8001294 <SSD1306_Command>
	SSD1306_Command(0xFF);                   // Page end (not really, but works here)
 800146c:	20ff      	movs	r0, #255	; 0xff
 800146e:	f7ff ff11 	bl	8001294 <SSD1306_Command>
	SSD1306_Command(SSD1306_COLUMNADDR);
 8001472:	2021      	movs	r0, #33	; 0x21
 8001474:	f7ff ff0e 	bl	8001294 <SSD1306_Command>
	SSD1306_Command(0); // Column start address
 8001478:	2000      	movs	r0, #0
 800147a:	f7ff ff0b 	bl	8001294 <SSD1306_Command>
	SSD1306_Command(SSD1306_LCDWIDTH - 1); // Column end address
 800147e:	207f      	movs	r0, #127	; 0x7f
 8001480:	f7ff ff08 	bl	8001294 <SSD1306_Command>

	SSD1306_Data(buffer, SSD1306_BUFFER_SIZE);
 8001484:	f44f 6180 	mov.w	r1, #1024	; 0x400
 8001488:	4802      	ldr	r0, [pc, #8]	; (8001494 <SSD1306_Display+0x38>)
 800148a:	f7ff ff1d 	bl	80012c8 <SSD1306_Data>
}
 800148e:	bf00      	nop
 8001490:	bd80      	pop	{r7, pc}
 8001492:	bf00      	nop
 8001494:	20000030 	.word	0x20000030

08001498 <SSD1306_Init>:

void SSD1306_Init(I2C_HandleTypeDef *i2c)
{
 8001498:	b580      	push	{r7, lr}
 800149a:	b082      	sub	sp, #8
 800149c:	af00      	add	r7, sp, #0
 800149e:	6078      	str	r0, [r7, #4]
	oled_i2c = i2c;
 80014a0:	4a28      	ldr	r2, [pc, #160]	; (8001544 <SSD1306_Init+0xac>)
 80014a2:	687b      	ldr	r3, [r7, #4]
 80014a4:	6013      	str	r3, [r2, #0]

	SSD1306_Command(SSD1306_DISPLAYOFF);
 80014a6:	20ae      	movs	r0, #174	; 0xae
 80014a8:	f7ff fef4 	bl	8001294 <SSD1306_Command>

	SSD1306_Command(SSD1306_SETDISPLAYCLOCKDIV);
 80014ac:	20d5      	movs	r0, #213	; 0xd5
 80014ae:	f7ff fef1 	bl	8001294 <SSD1306_Command>
	SSD1306_Command(0x80);
 80014b2:	2080      	movs	r0, #128	; 0x80
 80014b4:	f7ff feee 	bl	8001294 <SSD1306_Command>

	SSD1306_Command(SSD1306_LCDHEIGHT - 1);
 80014b8:	203f      	movs	r0, #63	; 0x3f
 80014ba:	f7ff feeb 	bl	8001294 <SSD1306_Command>

	SSD1306_Command(SSD1306_SETDISPLAYOFFSET);
 80014be:	20d3      	movs	r0, #211	; 0xd3
 80014c0:	f7ff fee8 	bl	8001294 <SSD1306_Command>
	SSD1306_Command(0x00);
 80014c4:	2000      	movs	r0, #0
 80014c6:	f7ff fee5 	bl	8001294 <SSD1306_Command>
	SSD1306_Command(SSD1306_SETSTARTLINE);
 80014ca:	2040      	movs	r0, #64	; 0x40
 80014cc:	f7ff fee2 	bl	8001294 <SSD1306_Command>

	SSD1306_Command(SSD1306_CHARGEPUMP);
 80014d0:	208d      	movs	r0, #141	; 0x8d
 80014d2:	f7ff fedf 	bl	8001294 <SSD1306_Command>
	SSD1306_Command(0x14);
 80014d6:	2014      	movs	r0, #20
 80014d8:	f7ff fedc 	bl	8001294 <SSD1306_Command>

	SSD1306_Command(SSD1306_MEMORYMODE); // 0x20
 80014dc:	2020      	movs	r0, #32
 80014de:	f7ff fed9 	bl	8001294 <SSD1306_Command>
	SSD1306_Command(0x00); // 0x0 act like ks0108
 80014e2:	2000      	movs	r0, #0
 80014e4:	f7ff fed6 	bl	8001294 <SSD1306_Command>
	SSD1306_Command(SSD1306_SEGREMAP | 0x1);
 80014e8:	20a1      	movs	r0, #161	; 0xa1
 80014ea:	f7ff fed3 	bl	8001294 <SSD1306_Command>
	SSD1306_Command(SSD1306_COMSCANDEC);
 80014ee:	20c8      	movs	r0, #200	; 0xc8
 80014f0:	f7ff fed0 	bl	8001294 <SSD1306_Command>

	SSD1306_Command(SSD1306_SETCOMPINS);
 80014f4:	20da      	movs	r0, #218	; 0xda
 80014f6:	f7ff fecd 	bl	8001294 <SSD1306_Command>
	SSD1306_Command(0x12);
 80014fa:	2012      	movs	r0, #18
 80014fc:	f7ff feca 	bl	8001294 <SSD1306_Command>
	SSD1306_Command(SSD1306_SETCONTRAST);
 8001500:	2081      	movs	r0, #129	; 0x81
 8001502:	f7ff fec7 	bl	8001294 <SSD1306_Command>
	SSD1306_Command(0xFF);
 8001506:	20ff      	movs	r0, #255	; 0xff
 8001508:	f7ff fec4 	bl	8001294 <SSD1306_Command>

	SSD1306_Command(SSD1306_SETPRECHARGE); // 0xd9
 800150c:	20d9      	movs	r0, #217	; 0xd9
 800150e:	f7ff fec1 	bl	8001294 <SSD1306_Command>
	SSD1306_Command(0xF1);
 8001512:	20f1      	movs	r0, #241	; 0xf1
 8001514:	f7ff febe 	bl	8001294 <SSD1306_Command>

	SSD1306_Command(SSD1306_SETVCOMDETECT); // 0xDB
 8001518:	20db      	movs	r0, #219	; 0xdb
 800151a:	f7ff febb 	bl	8001294 <SSD1306_Command>
	SSD1306_Command(0x40);
 800151e:	2040      	movs	r0, #64	; 0x40
 8001520:	f7ff feb8 	bl	8001294 <SSD1306_Command>
	SSD1306_Command(SSD1306_DISPLAYALLON_RESUME); // 0xA4
 8001524:	20a4      	movs	r0, #164	; 0xa4
 8001526:	f7ff feb5 	bl	8001294 <SSD1306_Command>
	SSD1306_Command(SSD1306_NORMALDISPLAY);       // 0xA6
 800152a:	20a6      	movs	r0, #166	; 0xa6
 800152c:	f7ff feb2 	bl	8001294 <SSD1306_Command>
	SSD1306_Command(SSD1306_DEACTIVATE_SCROLL);
 8001530:	202e      	movs	r0, #46	; 0x2e
 8001532:	f7ff feaf 	bl	8001294 <SSD1306_Command>

	SSD1306_Command(SSD1306_DISPLAYON); // Main screen turn on
 8001536:	20af      	movs	r0, #175	; 0xaf
 8001538:	f7ff feac 	bl	8001294 <SSD1306_Command>
}
 800153c:	bf00      	nop
 800153e:	3708      	adds	r7, #8
 8001540:	46bd      	mov	sp, r7
 8001542:	bd80      	pop	{r7, pc}
 8001544:	20004d3c 	.word	0x20004d3c

08001548 <Read8>:

//
// Read 8 bits from BMP280 from Register
//
uint8_t Read8(BMP280_t *bmp, uint8_t Register)
{
 8001548:	b580      	push	{r7, lr}
 800154a:	b088      	sub	sp, #32
 800154c:	af04      	add	r7, sp, #16
 800154e:	6078      	str	r0, [r7, #4]
 8001550:	460b      	mov	r3, r1
 8001552:	70fb      	strb	r3, [r7, #3]
	uint8_t Value;

	HAL_I2C_Mem_Read(bmp->bmp_i2c, ((bmp->Address)<<1), Register, 1, &Value, 1, BMP280_I2C_TIMEOUT);
 8001554:	687b      	ldr	r3, [r7, #4]
 8001556:	6818      	ldr	r0, [r3, #0]
 8001558:	687b      	ldr	r3, [r7, #4]
 800155a:	791b      	ldrb	r3, [r3, #4]
 800155c:	b29b      	uxth	r3, r3
 800155e:	005b      	lsls	r3, r3, #1
 8001560:	b299      	uxth	r1, r3
 8001562:	78fb      	ldrb	r3, [r7, #3]
 8001564:	b29a      	uxth	r2, r3
 8001566:	f44f 737a 	mov.w	r3, #1000	; 0x3e8
 800156a:	9302      	str	r3, [sp, #8]
 800156c:	2301      	movs	r3, #1
 800156e:	9301      	str	r3, [sp, #4]
 8001570:	f107 030f 	add.w	r3, r7, #15
 8001574:	9300      	str	r3, [sp, #0]
 8001576:	2301      	movs	r3, #1
 8001578:	f003 f87e 	bl	8004678 <HAL_I2C_Mem_Read>

	return Value;
 800157c:	7bfb      	ldrb	r3, [r7, #15]
}
 800157e:	4618      	mov	r0, r3
 8001580:	3710      	adds	r7, #16
 8001582:	46bd      	mov	sp, r7
 8001584:	bd80      	pop	{r7, pc}

08001586 <Write8>:

//
// Write 8 bits to BMP280 to Register
//
void Write8(BMP280_t *bmp, uint8_t Register, uint8_t Value)
{
 8001586:	b580      	push	{r7, lr}
 8001588:	b086      	sub	sp, #24
 800158a:	af04      	add	r7, sp, #16
 800158c:	6078      	str	r0, [r7, #4]
 800158e:	460b      	mov	r3, r1
 8001590:	70fb      	strb	r3, [r7, #3]
 8001592:	4613      	mov	r3, r2
 8001594:	70bb      	strb	r3, [r7, #2]
	HAL_I2C_Mem_Write(bmp->bmp_i2c, ((bmp->Address)<<1), Register, 1, &Value, 1, BMP280_I2C_TIMEOUT);
 8001596:	687b      	ldr	r3, [r7, #4]
 8001598:	6818      	ldr	r0, [r3, #0]
 800159a:	687b      	ldr	r3, [r7, #4]
 800159c:	791b      	ldrb	r3, [r3, #4]
 800159e:	b29b      	uxth	r3, r3
 80015a0:	005b      	lsls	r3, r3, #1
 80015a2:	b299      	uxth	r1, r3
 80015a4:	78fb      	ldrb	r3, [r7, #3]
 80015a6:	b29a      	uxth	r2, r3
 80015a8:	f44f 737a 	mov.w	r3, #1000	; 0x3e8
 80015ac:	9302      	str	r3, [sp, #8]
 80015ae:	2301      	movs	r3, #1
 80015b0:	9301      	str	r3, [sp, #4]
 80015b2:	1cbb      	adds	r3, r7, #2
 80015b4:	9300      	str	r3, [sp, #0]
 80015b6:	2301      	movs	r3, #1
 80015b8:	f002 ff64 	bl	8004484 <HAL_I2C_Mem_Write>
}
 80015bc:	bf00      	nop
 80015be:	3708      	adds	r7, #8
 80015c0:	46bd      	mov	sp, r7
 80015c2:	bd80      	pop	{r7, pc}

080015c4 <Read16>:

//
// Read 16 bits from BMP280 from Register
//
uint16_t Read16(BMP280_t *bmp, uint8_t Register)
{
 80015c4:	b580      	push	{r7, lr}
 80015c6:	b088      	sub	sp, #32
 80015c8:	af04      	add	r7, sp, #16
 80015ca:	6078      	str	r0, [r7, #4]
 80015cc:	460b      	mov	r3, r1
 80015ce:	70fb      	strb	r3, [r7, #3]
	uint8_t Value[2];

	HAL_I2C_Mem_Read(bmp->bmp_i2c, ((bmp->Address)<<1), Register, 1, Value, 2, BMP280_I2C_TIMEOUT);
 80015d0:	687b      	ldr	r3, [r7, #4]
 80015d2:	6818      	ldr	r0, [r3, #0]
 80015d4:	687b      	ldr	r3, [r7, #4]
 80015d6:	791b      	ldrb	r3, [r3, #4]
 80015d8:	b29b      	uxth	r3, r3
 80015da:	005b      	lsls	r3, r3, #1
 80015dc:	b299      	uxth	r1, r3
 80015de:	78fb      	ldrb	r3, [r7, #3]
 80015e0:	b29a      	uxth	r2, r3
 80015e2:	f44f 737a 	mov.w	r3, #1000	; 0x3e8
 80015e6:	9302      	str	r3, [sp, #8]
 80015e8:	2302      	movs	r3, #2
 80015ea:	9301      	str	r3, [sp, #4]
 80015ec:	f107 030c 	add.w	r3, r7, #12
 80015f0:	9300      	str	r3, [sp, #0]
 80015f2:	2301      	movs	r3, #1
 80015f4:	f003 f840 	bl	8004678 <HAL_I2C_Mem_Read>

	return ((Value[1] << 8) | Value[0]);
 80015f8:	7b7b      	ldrb	r3, [r7, #13]
 80015fa:	021b      	lsls	r3, r3, #8
 80015fc:	b21a      	sxth	r2, r3
 80015fe:	7b3b      	ldrb	r3, [r7, #12]
 8001600:	b21b      	sxth	r3, r3
 8001602:	4313      	orrs	r3, r2
 8001604:	b21b      	sxth	r3, r3
 8001606:	b29b      	uxth	r3, r3
}
 8001608:	4618      	mov	r0, r3
 800160a:	3710      	adds	r7, #16
 800160c:	46bd      	mov	sp, r7
 800160e:	bd80      	pop	{r7, pc}

08001610 <Read24>:

//
// Read 24 bits from BMP280 from Register
//
uint32_t Read24(BMP280_t *bmp, uint8_t Register)
{
 8001610:	b580      	push	{r7, lr}
 8001612:	b088      	sub	sp, #32
 8001614:	af04      	add	r7, sp, #16
 8001616:	6078      	str	r0, [r7, #4]
 8001618:	460b      	mov	r3, r1
 800161a:	70fb      	strb	r3, [r7, #3]
	uint8_t Value[3];

	HAL_I2C_Mem_Read(bmp->bmp_i2c, ((bmp->Address)<<1), Register, 1, Value, 3, BMP280_I2C_TIMEOUT);
 800161c:	687b      	ldr	r3, [r7, #4]
 800161e:	6818      	ldr	r0, [r3, #0]
 8001620:	687b      	ldr	r3, [r7, #4]
 8001622:	791b      	ldrb	r3, [r3, #4]
 8001624:	b29b      	uxth	r3, r3
 8001626:	005b      	lsls	r3, r3, #1
 8001628:	b299      	uxth	r1, r3
 800162a:	78fb      	ldrb	r3, [r7, #3]
 800162c:	b29a      	uxth	r2, r3
 800162e:	f44f 737a 	mov.w	r3, #1000	; 0x3e8
 8001632:	9302      	str	r3, [sp, #8]
 8001634:	2303      	movs	r3, #3
 8001636:	9301      	str	r3, [sp, #4]
 8001638:	f107 030c 	add.w	r3, r7, #12
 800163c:	9300      	str	r3, [sp, #0]
 800163e:	2301      	movs	r3, #1
 8001640:	f003 f81a 	bl	8004678 <HAL_I2C_Mem_Read>

	return ((Value[0] << 16) | (Value[1] << 8) | Value[2]);
 8001644:	7b3b      	ldrb	r3, [r7, #12]
 8001646:	041a      	lsls	r2, r3, #16
 8001648:	7b7b      	ldrb	r3, [r7, #13]
 800164a:	021b      	lsls	r3, r3, #8
 800164c:	4313      	orrs	r3, r2
 800164e:	7bba      	ldrb	r2, [r7, #14]
 8001650:	4313      	orrs	r3, r2
}
 8001652:	4618      	mov	r0, r3
 8001654:	3710      	adds	r7, #16
 8001656:	46bd      	mov	sp, r7
 8001658:	bd80      	pop	{r7, pc}

0800165a <BMP280_SetMode>:

//
// Set mode - Forced or Normal - in Control register
//
void BMP280_SetMode(BMP280_t *bmp, uint8_t Mode)
{
 800165a:	b580      	push	{r7, lr}
 800165c:	b084      	sub	sp, #16
 800165e:	af00      	add	r7, sp, #0
 8001660:	6078      	str	r0, [r7, #4]
 8001662:	460b      	mov	r3, r1
 8001664:	70fb      	strb	r3, [r7, #3]
	uint8_t Tmp;

	if(Mode > 3) Mode = 3;
 8001666:	78fb      	ldrb	r3, [r7, #3]
 8001668:	2b03      	cmp	r3, #3
 800166a:	d901      	bls.n	8001670 <BMP280_SetMode+0x16>
 800166c:	2303      	movs	r3, #3
 800166e:	70fb      	strb	r3, [r7, #3]

	Tmp = Read8(bmp, BMP280_CONTROL);
 8001670:	21f4      	movs	r1, #244	; 0xf4
 8001672:	6878      	ldr	r0, [r7, #4]
 8001674:	f7ff ff68 	bl	8001548 <Read8>
 8001678:	4603      	mov	r3, r0
 800167a:	73fb      	strb	r3, [r7, #15]

	Tmp = Tmp & 0xFC; // Tmp (xxxx xx00)
 800167c:	7bfb      	ldrb	r3, [r7, #15]
 800167e:	f023 0303 	bic.w	r3, r3, #3
 8001682:	73fb      	strb	r3, [r7, #15]
	Tmp |= Mode & 0x03;
 8001684:	f997 3003 	ldrsb.w	r3, [r7, #3]
 8001688:	f003 0303 	and.w	r3, r3, #3
 800168c:	b25a      	sxtb	r2, r3
 800168e:	f997 300f 	ldrsb.w	r3, [r7, #15]
 8001692:	4313      	orrs	r3, r2
 8001694:	b25b      	sxtb	r3, r3
 8001696:	73fb      	strb	r3, [r7, #15]

	Write8(bmp, BMP280_CONTROL, Tmp);
 8001698:	7bfb      	ldrb	r3, [r7, #15]
 800169a:	461a      	mov	r2, r3
 800169c:	21f4      	movs	r1, #244	; 0xf4
 800169e:	6878      	ldr	r0, [r7, #4]
 80016a0:	f7ff ff71 	bl	8001586 <Write8>
}
 80016a4:	bf00      	nop
 80016a6:	3710      	adds	r7, #16
 80016a8:	46bd      	mov	sp, r7
 80016aa:	bd80      	pop	{r7, pc}

080016ac <BMP280_SetPressureOversampling>:

//
// Set pressure oversampling in Control register
//
void BMP280_SetPressureOversampling(BMP280_t *bmp, uint8_t POversampling)
{
 80016ac:	b580      	push	{r7, lr}
 80016ae:	b084      	sub	sp, #16
 80016b0:	af00      	add	r7, sp, #0
 80016b2:	6078      	str	r0, [r7, #4]
 80016b4:	460b      	mov	r3, r1
 80016b6:	70fb      	strb	r3, [r7, #3]
	uint8_t Tmp;

	if(POversampling > 5) POversampling = 5;
 80016b8:	78fb      	ldrb	r3, [r7, #3]
 80016ba:	2b05      	cmp	r3, #5
 80016bc:	d901      	bls.n	80016c2 <BMP280_SetPressureOversampling+0x16>
 80016be:	2305      	movs	r3, #5
 80016c0:	70fb      	strb	r3, [r7, #3]

	Tmp = Read8(bmp, BMP280_CONTROL);
 80016c2:	21f4      	movs	r1, #244	; 0xf4
 80016c4:	6878      	ldr	r0, [r7, #4]
 80016c6:	f7ff ff3f 	bl	8001548 <Read8>
 80016ca:	4603      	mov	r3, r0
 80016cc:	73fb      	strb	r3, [r7, #15]

	Tmp = Tmp & 0xE3; // Tmp (xxx0 00xx)
 80016ce:	7bfb      	ldrb	r3, [r7, #15]
 80016d0:	f023 031c 	bic.w	r3, r3, #28
 80016d4:	73fb      	strb	r3, [r7, #15]
	Tmp |= ((POversampling << 2) & 0x1C);  // (0001 1100)
 80016d6:	78fb      	ldrb	r3, [r7, #3]
 80016d8:	009b      	lsls	r3, r3, #2
 80016da:	b25b      	sxtb	r3, r3
 80016dc:	f003 031c 	and.w	r3, r3, #28
 80016e0:	b25a      	sxtb	r2, r3
 80016e2:	f997 300f 	ldrsb.w	r3, [r7, #15]
 80016e6:	4313      	orrs	r3, r2
 80016e8:	b25b      	sxtb	r3, r3
 80016ea:	73fb      	strb	r3, [r7, #15]

	Write8(bmp, BMP280_CONTROL, Tmp);
 80016ec:	7bfb      	ldrb	r3, [r7, #15]
 80016ee:	461a      	mov	r2, r3
 80016f0:	21f4      	movs	r1, #244	; 0xf4
 80016f2:	6878      	ldr	r0, [r7, #4]
 80016f4:	f7ff ff47 	bl	8001586 <Write8>
}
 80016f8:	bf00      	nop
 80016fa:	3710      	adds	r7, #16
 80016fc:	46bd      	mov	sp, r7
 80016fe:	bd80      	pop	{r7, pc}

08001700 <BMP280_SetTemperatureOversampling>:

//
// Set temperature oversampling in Control register
//
void BMP280_SetTemperatureOversampling(BMP280_t *bmp, uint8_t TOversampling)
{
 8001700:	b580      	push	{r7, lr}
 8001702:	b084      	sub	sp, #16
 8001704:	af00      	add	r7, sp, #0
 8001706:	6078      	str	r0, [r7, #4]
 8001708:	460b      	mov	r3, r1
 800170a:	70fb      	strb	r3, [r7, #3]
	uint8_t Tmp;

	if(TOversampling > 5) TOversampling = 5;
 800170c:	78fb      	ldrb	r3, [r7, #3]
 800170e:	2b05      	cmp	r3, #5
 8001710:	d901      	bls.n	8001716 <BMP280_SetTemperatureOversampling+0x16>
 8001712:	2305      	movs	r3, #5
 8001714:	70fb      	strb	r3, [r7, #3]

	Tmp = Read8(bmp, BMP280_CONTROL);
 8001716:	21f4      	movs	r1, #244	; 0xf4
 8001718:	6878      	ldr	r0, [r7, #4]
 800171a:	f7ff ff15 	bl	8001548 <Read8>
 800171e:	4603      	mov	r3, r0
 8001720:	73fb      	strb	r3, [r7, #15]

	Tmp = Tmp & 0x1F; // Tmp (000x xxxx)
 8001722:	7bfb      	ldrb	r3, [r7, #15]
 8001724:	f003 031f 	and.w	r3, r3, #31
 8001728:	73fb      	strb	r3, [r7, #15]
	Tmp |= ((TOversampling << 5) & 0xE0) ;  // (1110 0000)
 800172a:	78fb      	ldrb	r3, [r7, #3]
 800172c:	015b      	lsls	r3, r3, #5
 800172e:	b25a      	sxtb	r2, r3
 8001730:	f997 300f 	ldrsb.w	r3, [r7, #15]
 8001734:	4313      	orrs	r3, r2
 8001736:	b25b      	sxtb	r3, r3
 8001738:	73fb      	strb	r3, [r7, #15]

	Write8(bmp, BMP280_CONTROL, Tmp);
 800173a:	7bfb      	ldrb	r3, [r7, #15]
 800173c:	461a      	mov	r2, r3
 800173e:	21f4      	movs	r1, #244	; 0xf4
 8001740:	6878      	ldr	r0, [r7, #4]
 8001742:	f7ff ff20 	bl	8001586 <Write8>
}
 8001746:	bf00      	nop
 8001748:	3710      	adds	r7, #16
 800174a:	46bd      	mov	sp, r7
 800174c:	bd80      	pop	{r7, pc}

0800174e <BMP280_ReadTemperatureRaw>:

//
// Read Raw temperature data from BMP280
//
int32_t BMP280_ReadTemperatureRaw(BMP280_t *bmp)
{
 800174e:	b580      	push	{r7, lr}
 8001750:	b084      	sub	sp, #16
 8001752:	af00      	add	r7, sp, #0
 8001754:	6078      	str	r0, [r7, #4]
	int32_t Tmp;

	Tmp = (int32_t)Read24(bmp, BMP280_TEMPDATA);
 8001756:	21fa      	movs	r1, #250	; 0xfa
 8001758:	6878      	ldr	r0, [r7, #4]
 800175a:	f7ff ff59 	bl	8001610 <Read24>
 800175e:	4603      	mov	r3, r0
 8001760:	60fb      	str	r3, [r7, #12]

	Tmp >>= 4; // Move 4 left due to such storing (Datasheet).
 8001762:	68fb      	ldr	r3, [r7, #12]
 8001764:	111b      	asrs	r3, r3, #4
 8001766:	60fb      	str	r3, [r7, #12]

	return Tmp;
 8001768:	68fb      	ldr	r3, [r7, #12]
}
 800176a:	4618      	mov	r0, r3
 800176c:	3710      	adds	r7, #16
 800176e:	46bd      	mov	sp, r7
 8001770:	bd80      	pop	{r7, pc}

08001772 <BMP280_ReadPressureRaw>:

//
// Read Raw pressure data from BMP280
//
int32_t BMP280_ReadPressureRaw(BMP280_t *bmp)
{
 8001772:	b580      	push	{r7, lr}
 8001774:	b084      	sub	sp, #16
 8001776:	af00      	add	r7, sp, #0
 8001778:	6078      	str	r0, [r7, #4]
	int32_t Tmp;

	Tmp = (int32_t)Read24(bmp, BMP280_PRESSUREDATA);
 800177a:	21f7      	movs	r1, #247	; 0xf7
 800177c:	6878      	ldr	r0, [r7, #4]
 800177e:	f7ff ff47 	bl	8001610 <Read24>
 8001782:	4603      	mov	r3, r0
 8001784:	60fb      	str	r3, [r7, #12]

	Tmp >>= 4; // Move 4 left due to such storing (Datasheet).
 8001786:	68fb      	ldr	r3, [r7, #12]
 8001788:	111b      	asrs	r3, r3, #4
 800178a:	60fb      	str	r3, [r7, #12]

	return Tmp;
 800178c:	68fb      	ldr	r3, [r7, #12]
}
 800178e:	4618      	mov	r0, r3
 8001790:	3710      	adds	r7, #16
 8001792:	46bd      	mov	sp, r7
 8001794:	bd80      	pop	{r7, pc}
	...

08001798 <BMP280_ReadTemperature>:
//
// Read and calculate temperature
// Whole procedure is taken from BMP280 Datasheet
//
float BMP280_ReadTemperature(BMP280_t *bmp)
{
 8001798:	b590      	push	{r4, r7, lr}
 800179a:	b087      	sub	sp, #28
 800179c:	af00      	add	r7, sp, #0
 800179e:	6078      	str	r0, [r7, #4]
	int32_t var1, var2, T;

	int32_t adc_T;

	adc_T = BMP280_ReadTemperatureRaw(bmp);
 80017a0:	6878      	ldr	r0, [r7, #4]
 80017a2:	f7ff ffd4 	bl	800174e <BMP280_ReadTemperatureRaw>
 80017a6:	6178      	str	r0, [r7, #20]

	var1 = ((((adc_T>>3) - ((int32_t)(bmp->t1)<<1))) * ((int32_t)(bmp->t2))) >> 11;
 80017a8:	697b      	ldr	r3, [r7, #20]
 80017aa:	10da      	asrs	r2, r3, #3
 80017ac:	687b      	ldr	r3, [r7, #4]
 80017ae:	8b5b      	ldrh	r3, [r3, #26]
 80017b0:	005b      	lsls	r3, r3, #1
 80017b2:	1ad3      	subs	r3, r2, r3
 80017b4:	687a      	ldr	r2, [r7, #4]
 80017b6:	f9b2 2006 	ldrsh.w	r2, [r2, #6]
 80017ba:	fb02 f303 	mul.w	r3, r2, r3
 80017be:	12db      	asrs	r3, r3, #11
 80017c0:	613b      	str	r3, [r7, #16]

	var2 = (((((adc_T>>4) - ((int32_t)(bmp->t1))) * ((adc_T>>4) - ((int32_t)(bmp->t1)))) >> 12) *
 80017c2:	697b      	ldr	r3, [r7, #20]
 80017c4:	111b      	asrs	r3, r3, #4
 80017c6:	687a      	ldr	r2, [r7, #4]
 80017c8:	8b52      	ldrh	r2, [r2, #26]
 80017ca:	1a9b      	subs	r3, r3, r2
 80017cc:	697a      	ldr	r2, [r7, #20]
 80017ce:	1112      	asrs	r2, r2, #4
 80017d0:	6879      	ldr	r1, [r7, #4]
 80017d2:	8b49      	ldrh	r1, [r1, #26]
 80017d4:	1a52      	subs	r2, r2, r1
 80017d6:	fb02 f303 	mul.w	r3, r2, r3
 80017da:	131b      	asrs	r3, r3, #12
	((int32_t)(bmp->t3))) >> 14;
 80017dc:	687a      	ldr	r2, [r7, #4]
 80017de:	f9b2 2008 	ldrsh.w	r2, [r2, #8]
	var2 = (((((adc_T>>4) - ((int32_t)(bmp->t1))) * ((adc_T>>4) - ((int32_t)(bmp->t1)))) >> 12) *
 80017e2:	fb02 f303 	mul.w	r3, r2, r3
 80017e6:	139b      	asrs	r3, r3, #14
 80017e8:	60fb      	str	r3, [r7, #12]

	bmp->t_fine = var1 + var2;
 80017ea:	693a      	ldr	r2, [r7, #16]
 80017ec:	68fb      	ldr	r3, [r7, #12]
 80017ee:	441a      	add	r2, r3
 80017f0:	687b      	ldr	r3, [r7, #4]
 80017f2:	621a      	str	r2, [r3, #32]

	T = ((bmp->t_fine) * 5 + 128) >> 8;
 80017f4:	687b      	ldr	r3, [r7, #4]
 80017f6:	6a1a      	ldr	r2, [r3, #32]
 80017f8:	4613      	mov	r3, r2
 80017fa:	009b      	lsls	r3, r3, #2
 80017fc:	4413      	add	r3, r2
 80017fe:	3380      	adds	r3, #128	; 0x80
 8001800:	121b      	asrs	r3, r3, #8
 8001802:	60bb      	str	r3, [r7, #8]

	return (float)(T/100.0);
 8001804:	68b8      	ldr	r0, [r7, #8]
 8001806:	f7fe fe3d 	bl	8000484 <__aeabi_i2d>
 800180a:	f04f 0200 	mov.w	r2, #0
 800180e:	4b08      	ldr	r3, [pc, #32]	; (8001830 <BMP280_ReadTemperature+0x98>)
 8001810:	f7fe ffcc 	bl	80007ac <__aeabi_ddiv>
 8001814:	4603      	mov	r3, r0
 8001816:	460c      	mov	r4, r1
 8001818:	4618      	mov	r0, r3
 800181a:	4621      	mov	r1, r4
 800181c:	f7ff f97e 	bl	8000b1c <__aeabi_d2f>
 8001820:	4603      	mov	r3, r0
 8001822:	ee07 3a90 	vmov	s15, r3
}
 8001826:	eeb0 0a67 	vmov.f32	s0, s15
 800182a:	371c      	adds	r7, #28
 800182c:	46bd      	mov	sp, r7
 800182e:	bd90      	pop	{r4, r7, pc}
 8001830:	40590000 	.word	0x40590000

08001834 <BMP280_ReadPressureAndTemperature>:
//
// Read and calculate temperature & pressure
// Whole procedure is taken from BMP280 Datasheet
//
uint8_t BMP280_ReadPressureAndTemperature(BMP280_t *bmp, float *Pressure, float *Temperature)
{
 8001834:	b590      	push	{r4, r7, lr}
 8001836:	b089      	sub	sp, #36	; 0x24
 8001838:	af00      	add	r7, sp, #0
 800183a:	60f8      	str	r0, [r7, #12]
 800183c:	60b9      	str	r1, [r7, #8]
 800183e:	607a      	str	r2, [r7, #4]
	// Have to read temperature first
	*Temperature = BMP280_ReadTemperature(bmp);
 8001840:	68f8      	ldr	r0, [r7, #12]
 8001842:	f7ff ffa9 	bl	8001798 <BMP280_ReadTemperature>
 8001846:	eef0 7a40 	vmov.f32	s15, s0
 800184a:	687b      	ldr	r3, [r7, #4]
 800184c:	edc3 7a00 	vstr	s15, [r3]

	int32_t var1, var2;
	uint32_t p;

	var1 = (((int32_t)(bmp->t_fine))>>1) - (int32_t)64000;
 8001850:	68fb      	ldr	r3, [r7, #12]
 8001852:	6a1b      	ldr	r3, [r3, #32]
 8001854:	105b      	asrs	r3, r3, #1
 8001856:	f5a3 437a 	sub.w	r3, r3, #64000	; 0xfa00
 800185a:	61bb      	str	r3, [r7, #24]
	var2 = (((var1>>2) * (var1>>2)) >> 11 ) * ((int32_t)(bmp->p6));
 800185c:	69bb      	ldr	r3, [r7, #24]
 800185e:	109b      	asrs	r3, r3, #2
 8001860:	69ba      	ldr	r2, [r7, #24]
 8001862:	1092      	asrs	r2, r2, #2
 8001864:	fb02 f303 	mul.w	r3, r2, r3
 8001868:	12db      	asrs	r3, r3, #11
 800186a:	68fa      	ldr	r2, [r7, #12]
 800186c:	f9b2 2012 	ldrsh.w	r2, [r2, #18]
 8001870:	fb02 f303 	mul.w	r3, r2, r3
 8001874:	617b      	str	r3, [r7, #20]
	var2 = var2 + ((var1*((int32_t)(bmp->p5)))<<1);
 8001876:	68fb      	ldr	r3, [r7, #12]
 8001878:	f9b3 3010 	ldrsh.w	r3, [r3, #16]
 800187c:	461a      	mov	r2, r3
 800187e:	69bb      	ldr	r3, [r7, #24]
 8001880:	fb03 f302 	mul.w	r3, r3, r2
 8001884:	005b      	lsls	r3, r3, #1
 8001886:	697a      	ldr	r2, [r7, #20]
 8001888:	4413      	add	r3, r2
 800188a:	617b      	str	r3, [r7, #20]
	var2 = (var2>>2)+(((int32_t)(bmp->p4))<<16);
 800188c:	697b      	ldr	r3, [r7, #20]
 800188e:	109a      	asrs	r2, r3, #2
 8001890:	68fb      	ldr	r3, [r7, #12]
 8001892:	f9b3 300e 	ldrsh.w	r3, [r3, #14]
 8001896:	041b      	lsls	r3, r3, #16
 8001898:	4413      	add	r3, r2
 800189a:	617b      	str	r3, [r7, #20]
	var1 = ((((bmp->p3) * (((var1>>2) * (var1>>2)) >> 13 )) >> 3) + ((((int32_t)(bmp->p2)) * var1)>>1))>>18;
 800189c:	68fb      	ldr	r3, [r7, #12]
 800189e:	f9b3 300c 	ldrsh.w	r3, [r3, #12]
 80018a2:	4619      	mov	r1, r3
 80018a4:	69bb      	ldr	r3, [r7, #24]
 80018a6:	109b      	asrs	r3, r3, #2
 80018a8:	69ba      	ldr	r2, [r7, #24]
 80018aa:	1092      	asrs	r2, r2, #2
 80018ac:	fb02 f303 	mul.w	r3, r2, r3
 80018b0:	135b      	asrs	r3, r3, #13
 80018b2:	fb03 f301 	mul.w	r3, r3, r1
 80018b6:	10da      	asrs	r2, r3, #3
 80018b8:	68fb      	ldr	r3, [r7, #12]
 80018ba:	f9b3 300a 	ldrsh.w	r3, [r3, #10]
 80018be:	4619      	mov	r1, r3
 80018c0:	69bb      	ldr	r3, [r7, #24]
 80018c2:	fb03 f301 	mul.w	r3, r3, r1
 80018c6:	105b      	asrs	r3, r3, #1
 80018c8:	4413      	add	r3, r2
 80018ca:	149b      	asrs	r3, r3, #18
 80018cc:	61bb      	str	r3, [r7, #24]
	var1 =((((32768+var1))*((int32_t)(bmp->p1)))>>15);
 80018ce:	69bb      	ldr	r3, [r7, #24]
 80018d0:	f503 4300 	add.w	r3, r3, #32768	; 0x8000
 80018d4:	68fa      	ldr	r2, [r7, #12]
 80018d6:	8b92      	ldrh	r2, [r2, #28]
 80018d8:	fb02 f303 	mul.w	r3, r2, r3
 80018dc:	13db      	asrs	r3, r3, #15
 80018de:	61bb      	str	r3, [r7, #24]

	if (var1 == 0)
 80018e0:	69bb      	ldr	r3, [r7, #24]
 80018e2:	2b00      	cmp	r3, #0
 80018e4:	d101      	bne.n	80018ea <BMP280_ReadPressureAndTemperature+0xb6>
	{
		return 1; // avoid exception caused by division by zero
 80018e6:	2301      	movs	r3, #1
 80018e8:	e054      	b.n	8001994 <BMP280_ReadPressureAndTemperature+0x160>
	}

	// Raw pressure from BMP's ADC
	int32_t adc_P = BMP280_ReadPressureRaw(bmp);
 80018ea:	68f8      	ldr	r0, [r7, #12]
 80018ec:	f7ff ff41 	bl	8001772 <BMP280_ReadPressureRaw>
 80018f0:	6138      	str	r0, [r7, #16]

	p = (((int32_t)(((int32_t)1048576)-adc_P)-(var2>>12)))*3125;
 80018f2:	693b      	ldr	r3, [r7, #16]
 80018f4:	f5c3 1280 	rsb	r2, r3, #1048576	; 0x100000
 80018f8:	697b      	ldr	r3, [r7, #20]
 80018fa:	131b      	asrs	r3, r3, #12
 80018fc:	1ad3      	subs	r3, r2, r3
 80018fe:	f640 4235 	movw	r2, #3125	; 0xc35
 8001902:	fb02 f303 	mul.w	r3, r2, r3
 8001906:	61fb      	str	r3, [r7, #28]
	if (p < 0x80000000)
 8001908:	69fb      	ldr	r3, [r7, #28]
 800190a:	2b00      	cmp	r3, #0
 800190c:	db06      	blt.n	800191c <BMP280_ReadPressureAndTemperature+0xe8>
	{
		p = (p << 1) / ((uint32_t)var1);
 800190e:	69fb      	ldr	r3, [r7, #28]
 8001910:	005a      	lsls	r2, r3, #1
 8001912:	69bb      	ldr	r3, [r7, #24]
 8001914:	fbb2 f3f3 	udiv	r3, r2, r3
 8001918:	61fb      	str	r3, [r7, #28]
 800191a:	e005      	b.n	8001928 <BMP280_ReadPressureAndTemperature+0xf4>
	}
	else
	{
		p = (p / (uint32_t)var1) * 2;
 800191c:	69bb      	ldr	r3, [r7, #24]
 800191e:	69fa      	ldr	r2, [r7, #28]
 8001920:	fbb2 f3f3 	udiv	r3, r2, r3
 8001924:	005b      	lsls	r3, r3, #1
 8001926:	61fb      	str	r3, [r7, #28]
	}
	var1 = (((int32_t)(bmp->p9)) * ((int32_t)(((p>>3) * (p>>3))>>13)))>>12;
 8001928:	68fb      	ldr	r3, [r7, #12]
 800192a:	f9b3 3018 	ldrsh.w	r3, [r3, #24]
 800192e:	4619      	mov	r1, r3
 8001930:	69fb      	ldr	r3, [r7, #28]
 8001932:	08db      	lsrs	r3, r3, #3
 8001934:	69fa      	ldr	r2, [r7, #28]
 8001936:	08d2      	lsrs	r2, r2, #3
 8001938:	fb02 f303 	mul.w	r3, r2, r3
 800193c:	0b5b      	lsrs	r3, r3, #13
 800193e:	fb03 f301 	mul.w	r3, r3, r1
 8001942:	131b      	asrs	r3, r3, #12
 8001944:	61bb      	str	r3, [r7, #24]
	var2 = (((int32_t)(p>>2)) * ((int32_t)(bmp->p8)))>>13;
 8001946:	69fb      	ldr	r3, [r7, #28]
 8001948:	089b      	lsrs	r3, r3, #2
 800194a:	461a      	mov	r2, r3
 800194c:	68fb      	ldr	r3, [r7, #12]
 800194e:	f9b3 3016 	ldrsh.w	r3, [r3, #22]
 8001952:	fb03 f302 	mul.w	r3, r3, r2
 8001956:	135b      	asrs	r3, r3, #13
 8001958:	617b      	str	r3, [r7, #20]

	p = (uint32_t)((int32_t)p + ((var1 + var2 + (bmp->p7)) >> 4));
 800195a:	69ba      	ldr	r2, [r7, #24]
 800195c:	697b      	ldr	r3, [r7, #20]
 800195e:	4413      	add	r3, r2
 8001960:	68fa      	ldr	r2, [r7, #12]
 8001962:	f9b2 2014 	ldrsh.w	r2, [r2, #20]
 8001966:	4413      	add	r3, r2
 8001968:	111a      	asrs	r2, r3, #4
 800196a:	69fb      	ldr	r3, [r7, #28]
 800196c:	4413      	add	r3, r2
 800196e:	61fb      	str	r3, [r7, #28]

	// Convert Pa to hPa
	*Pressure = (float)(p/100.0);
 8001970:	69f8      	ldr	r0, [r7, #28]
 8001972:	f7fe fd77 	bl	8000464 <__aeabi_ui2d>
 8001976:	f04f 0200 	mov.w	r2, #0
 800197a:	4b08      	ldr	r3, [pc, #32]	; (800199c <BMP280_ReadPressureAndTemperature+0x168>)
 800197c:	f7fe ff16 	bl	80007ac <__aeabi_ddiv>
 8001980:	4603      	mov	r3, r0
 8001982:	460c      	mov	r4, r1
 8001984:	4618      	mov	r0, r3
 8001986:	4621      	mov	r1, r4
 8001988:	f7ff f8c8 	bl	8000b1c <__aeabi_d2f>
 800198c:	4602      	mov	r2, r0
 800198e:	68bb      	ldr	r3, [r7, #8]
 8001990:	601a      	str	r2, [r3, #0]

	return 0;
 8001992:	2300      	movs	r3, #0
}
 8001994:	4618      	mov	r0, r3
 8001996:	3724      	adds	r7, #36	; 0x24
 8001998:	46bd      	mov	sp, r7
 800199a:	bd90      	pop	{r4, r7, pc}
 800199c:	40590000 	.word	0x40590000

080019a0 <BMP280_Init>:

//
// Init
//
uint8_t BMP280_Init(BMP280_t *bmp, I2C_HandleTypeDef *i2c, uint8_t Address)
{
 80019a0:	b580      	push	{r7, lr}
 80019a2:	b086      	sub	sp, #24
 80019a4:	af00      	add	r7, sp, #0
 80019a6:	60f8      	str	r0, [r7, #12]
 80019a8:	60b9      	str	r1, [r7, #8]
 80019aa:	4613      	mov	r3, r2
 80019ac:	71fb      	strb	r3, [r7, #7]
	uint8_t ChipID;

	// Save I2C handler and address
	bmp->bmp_i2c = i2c;
 80019ae:	68fb      	ldr	r3, [r7, #12]
 80019b0:	68ba      	ldr	r2, [r7, #8]
 80019b2:	601a      	str	r2, [r3, #0]
	bmp->Address = Address;
 80019b4:	68fb      	ldr	r3, [r7, #12]
 80019b6:	79fa      	ldrb	r2, [r7, #7]
 80019b8:	711a      	strb	r2, [r3, #4]

	//Read Chip ID
	ChipID = Read8(bmp, BMP280_CHIPID);
 80019ba:	21d0      	movs	r1, #208	; 0xd0
 80019bc:	68f8      	ldr	r0, [r7, #12]
 80019be:	f7ff fdc3 	bl	8001548 <Read8>
 80019c2:	4603      	mov	r3, r0
 80019c4:	75fb      	strb	r3, [r7, #23]

	// Check if ID is correct
	if(ChipID != 0x58)
 80019c6:	7dfb      	ldrb	r3, [r7, #23]
 80019c8:	2b58      	cmp	r3, #88	; 0x58
 80019ca:	d001      	beq.n	80019d0 <BMP280_Init+0x30>
	{
		return 1;
 80019cc:	2301      	movs	r3, #1
 80019ce:	e06c      	b.n	8001aaa <BMP280_Init+0x10a>
	}

	// Read all coefficients
	bmp->t1 = Read16(bmp, BMP280_DIG_T1);
 80019d0:	2188      	movs	r1, #136	; 0x88
 80019d2:	68f8      	ldr	r0, [r7, #12]
 80019d4:	f7ff fdf6 	bl	80015c4 <Read16>
 80019d8:	4603      	mov	r3, r0
 80019da:	461a      	mov	r2, r3
 80019dc:	68fb      	ldr	r3, [r7, #12]
 80019de:	835a      	strh	r2, [r3, #26]
	bmp->t2 = Read16(bmp, BMP280_DIG_T2);
 80019e0:	218a      	movs	r1, #138	; 0x8a
 80019e2:	68f8      	ldr	r0, [r7, #12]
 80019e4:	f7ff fdee 	bl	80015c4 <Read16>
 80019e8:	4603      	mov	r3, r0
 80019ea:	b21a      	sxth	r2, r3
 80019ec:	68fb      	ldr	r3, [r7, #12]
 80019ee:	80da      	strh	r2, [r3, #6]
	bmp->t3 = Read16(bmp, BMP280_DIG_T3);
 80019f0:	218c      	movs	r1, #140	; 0x8c
 80019f2:	68f8      	ldr	r0, [r7, #12]
 80019f4:	f7ff fde6 	bl	80015c4 <Read16>
 80019f8:	4603      	mov	r3, r0
 80019fa:	b21a      	sxth	r2, r3
 80019fc:	68fb      	ldr	r3, [r7, #12]
 80019fe:	811a      	strh	r2, [r3, #8]

	bmp->p1 = Read16(bmp, BMP280_DIG_P1);
 8001a00:	218e      	movs	r1, #142	; 0x8e
 8001a02:	68f8      	ldr	r0, [r7, #12]
 8001a04:	f7ff fdde 	bl	80015c4 <Read16>
 8001a08:	4603      	mov	r3, r0
 8001a0a:	461a      	mov	r2, r3
 8001a0c:	68fb      	ldr	r3, [r7, #12]
 8001a0e:	839a      	strh	r2, [r3, #28]
	bmp->p2 = Read16(bmp, BMP280_DIG_P2);
 8001a10:	2190      	movs	r1, #144	; 0x90
 8001a12:	68f8      	ldr	r0, [r7, #12]
 8001a14:	f7ff fdd6 	bl	80015c4 <Read16>
 8001a18:	4603      	mov	r3, r0
 8001a1a:	b21a      	sxth	r2, r3
 8001a1c:	68fb      	ldr	r3, [r7, #12]
 8001a1e:	815a      	strh	r2, [r3, #10]
	bmp->p3 = Read16(bmp, BMP280_DIG_P3);
 8001a20:	2192      	movs	r1, #146	; 0x92
 8001a22:	68f8      	ldr	r0, [r7, #12]
 8001a24:	f7ff fdce 	bl	80015c4 <Read16>
 8001a28:	4603      	mov	r3, r0
 8001a2a:	b21a      	sxth	r2, r3
 8001a2c:	68fb      	ldr	r3, [r7, #12]
 8001a2e:	819a      	strh	r2, [r3, #12]
	bmp->p4 = Read16(bmp, BMP280_DIG_P4);
 8001a30:	2194      	movs	r1, #148	; 0x94
 8001a32:	68f8      	ldr	r0, [r7, #12]
 8001a34:	f7ff fdc6 	bl	80015c4 <Read16>
 8001a38:	4603      	mov	r3, r0
 8001a3a:	b21a      	sxth	r2, r3
 8001a3c:	68fb      	ldr	r3, [r7, #12]
 8001a3e:	81da      	strh	r2, [r3, #14]
	bmp->p5 = Read16(bmp, BMP280_DIG_P5);
 8001a40:	2196      	movs	r1, #150	; 0x96
 8001a42:	68f8      	ldr	r0, [r7, #12]
 8001a44:	f7ff fdbe 	bl	80015c4 <Read16>
 8001a48:	4603      	mov	r3, r0
 8001a4a:	b21a      	sxth	r2, r3
 8001a4c:	68fb      	ldr	r3, [r7, #12]
 8001a4e:	821a      	strh	r2, [r3, #16]
	bmp->p6 = Read16(bmp, BMP280_DIG_P6);
 8001a50:	2198      	movs	r1, #152	; 0x98
 8001a52:	68f8      	ldr	r0, [r7, #12]
 8001a54:	f7ff fdb6 	bl	80015c4 <Read16>
 8001a58:	4603      	mov	r3, r0
 8001a5a:	b21a      	sxth	r2, r3
 8001a5c:	68fb      	ldr	r3, [r7, #12]
 8001a5e:	825a      	strh	r2, [r3, #18]
	bmp->p7 = Read16(bmp, BMP280_DIG_P7);
 8001a60:	219a      	movs	r1, #154	; 0x9a
 8001a62:	68f8      	ldr	r0, [r7, #12]
 8001a64:	f7ff fdae 	bl	80015c4 <Read16>
 8001a68:	4603      	mov	r3, r0
 8001a6a:	b21a      	sxth	r2, r3
 8001a6c:	68fb      	ldr	r3, [r7, #12]
 8001a6e:	829a      	strh	r2, [r3, #20]
	bmp->p8 = Read16(bmp, BMP280_DIG_P8);
 8001a70:	219c      	movs	r1, #156	; 0x9c
 8001a72:	68f8      	ldr	r0, [r7, #12]
 8001a74:	f7ff fda6 	bl	80015c4 <Read16>
 8001a78:	4603      	mov	r3, r0
 8001a7a:	b21a      	sxth	r2, r3
 8001a7c:	68fb      	ldr	r3, [r7, #12]
 8001a7e:	82da      	strh	r2, [r3, #22]
	bmp->p9 = Read16(bmp, BMP280_DIG_P9);
 8001a80:	219e      	movs	r1, #158	; 0x9e
 8001a82:	68f8      	ldr	r0, [r7, #12]
 8001a84:	f7ff fd9e 	bl	80015c4 <Read16>
 8001a88:	4603      	mov	r3, r0
 8001a8a:	b21a      	sxth	r2, r3
 8001a8c:	68fb      	ldr	r3, [r7, #12]
 8001a8e:	831a      	strh	r2, [r3, #24]

	// Set base settings
	BMP280_SetTemperatureOversampling(bmp, BMP280_TEMPERATURE_20BIT);
 8001a90:	2105      	movs	r1, #5
 8001a92:	68f8      	ldr	r0, [r7, #12]
 8001a94:	f7ff fe34 	bl	8001700 <BMP280_SetTemperatureOversampling>
	BMP280_SetPressureOversampling(bmp, BMP280_ULTRAHIGHRES);
 8001a98:	2105      	movs	r1, #5
 8001a9a:	68f8      	ldr	r0, [r7, #12]
 8001a9c:	f7ff fe06 	bl	80016ac <BMP280_SetPressureOversampling>
	BMP280_SetMode(bmp, BMP280_NORMALMODE);
 8001aa0:	2103      	movs	r1, #3
 8001aa2:	68f8      	ldr	r0, [r7, #12]
 8001aa4:	f7ff fdd9 	bl	800165a <BMP280_SetMode>

	return 0;
 8001aa8:	2300      	movs	r3, #0
}
 8001aaa:	4618      	mov	r0, r3
 8001aac:	3718      	adds	r7, #24
 8001aae:	46bd      	mov	sp, r7
 8001ab0:	bd80      	pop	{r7, pc}
	...

08001ab4 <_putchar>:
};

/* Private function prototypes -----------------------------------------------*/
/* USER CODE BEGIN FunctionPrototypes */
void _putchar(char character)
{
 8001ab4:	b580      	push	{r7, lr}
 8001ab6:	b082      	sub	sp, #8
 8001ab8:	af00      	add	r7, sp, #0
 8001aba:	4603      	mov	r3, r0
 8001abc:	71fb      	strb	r3, [r7, #7]
  // send char to console etc.
	osMutexAcquire(MutexPrintfHandle, osWaitForever);
 8001abe:	4b0b      	ldr	r3, [pc, #44]	; (8001aec <_putchar+0x38>)
 8001ac0:	681b      	ldr	r3, [r3, #0]
 8001ac2:	f04f 31ff 	mov.w	r1, #4294967295
 8001ac6:	4618      	mov	r0, r3
 8001ac8:	f005 f896 	bl	8006bf8 <osMutexAcquire>
	HAL_UART_Transmit(&huart2, (uint8_t*)&character, 1, 1000);
 8001acc:	1df9      	adds	r1, r7, #7
 8001ace:	f44f 737a 	mov.w	r3, #1000	; 0x3e8
 8001ad2:	2201      	movs	r2, #1
 8001ad4:	4806      	ldr	r0, [pc, #24]	; (8001af0 <_putchar+0x3c>)
 8001ad6:	f004 fa50 	bl	8005f7a <HAL_UART_Transmit>
	osMutexRelease(MutexPrintfHandle);
 8001ada:	4b04      	ldr	r3, [pc, #16]	; (8001aec <_putchar+0x38>)
 8001adc:	681b      	ldr	r3, [r3, #0]
 8001ade:	4618      	mov	r0, r3
 8001ae0:	f005 f8e8 	bl	8006cb4 <osMutexRelease>
}
 8001ae4:	bf00      	nop
 8001ae6:	3708      	adds	r7, #8
 8001ae8:	46bd      	mov	sp, r7
 8001aea:	bd80      	pop	{r7, pc}
 8001aec:	20004d48 	.word	0x20004d48
 8001af0:	20004df4 	.word	0x20004df4

08001af4 <MX_FREERTOS_Init>:
/**
  * @brief  FreeRTOS initialization
  * @param  None
  * @retval None
  */
void MX_FREERTOS_Init(void) {
 8001af4:	b580      	push	{r7, lr}
 8001af6:	af00      	add	r7, sp, #0
  /* USER CODE BEGIN Init */

  /* USER CODE END Init */
  /* Create the mutex(es) */
  /* creation of MutexPrintf */
  MutexPrintfHandle = osMutexNew(&MutexPrintf_attributes);
 8001af8:	4815      	ldr	r0, [pc, #84]	; (8001b50 <MX_FREERTOS_Init+0x5c>)
 8001afa:	f004 ffe3 	bl	8006ac4 <osMutexNew>
 8001afe:	4602      	mov	r2, r0
 8001b00:	4b14      	ldr	r3, [pc, #80]	; (8001b54 <MX_FREERTOS_Init+0x60>)
 8001b02:	601a      	str	r2, [r3, #0]

  /* creation of MutexI2C1 */
  MutexI2C1Handle = osMutexNew(&MutexI2C1_attributes);
 8001b04:	4814      	ldr	r0, [pc, #80]	; (8001b58 <MX_FREERTOS_Init+0x64>)
 8001b06:	f004 ffdd 	bl	8006ac4 <osMutexNew>
 8001b0a:	4602      	mov	r2, r0
 8001b0c:	4b13      	ldr	r3, [pc, #76]	; (8001b5c <MX_FREERTOS_Init+0x68>)
 8001b0e:	601a      	str	r2, [r3, #0]

  /* creation of MutexBmpData */
  MutexBmpDataHandle = osMutexNew(&MutexBmpData_attributes);
 8001b10:	4813      	ldr	r0, [pc, #76]	; (8001b60 <MX_FREERTOS_Init+0x6c>)
 8001b12:	f004 ffd7 	bl	8006ac4 <osMutexNew>
 8001b16:	4602      	mov	r2, r0
 8001b18:	4b12      	ldr	r3, [pc, #72]	; (8001b64 <MX_FREERTOS_Init+0x70>)
 8001b1a:	601a      	str	r2, [r3, #0]
  /* add queues, ... */
  /* USER CODE END RTOS_QUEUES */

  /* Create the thread(s) */
  /* creation of HeartbeatTask */
  HeartbeatTaskHandle = osThreadNew(StartHeartbeatTask, NULL, &HeartbeatTask_attributes);
 8001b1c:	4a12      	ldr	r2, [pc, #72]	; (8001b68 <MX_FREERTOS_Init+0x74>)
 8001b1e:	2100      	movs	r1, #0
 8001b20:	4812      	ldr	r0, [pc, #72]	; (8001b6c <MX_FREERTOS_Init+0x78>)
 8001b22:	f004 fefb 	bl	800691c <osThreadNew>
 8001b26:	4602      	mov	r2, r0
 8001b28:	4b11      	ldr	r3, [pc, #68]	; (8001b70 <MX_FREERTOS_Init+0x7c>)
 8001b2a:	601a      	str	r2, [r3, #0]

  /* creation of Bmp280Task */
  Bmp280TaskHandle = osThreadNew(StartBmp280Task, NULL, &Bmp280Task_attributes);
 8001b2c:	4a11      	ldr	r2, [pc, #68]	; (8001b74 <MX_FREERTOS_Init+0x80>)
 8001b2e:	2100      	movs	r1, #0
 8001b30:	4811      	ldr	r0, [pc, #68]	; (8001b78 <MX_FREERTOS_Init+0x84>)
 8001b32:	f004 fef3 	bl	800691c <osThreadNew>
 8001b36:	4602      	mov	r2, r0
 8001b38:	4b10      	ldr	r3, [pc, #64]	; (8001b7c <MX_FREERTOS_Init+0x88>)
 8001b3a:	601a      	str	r2, [r3, #0]

  /* creation of OledTask */
  OledTaskHandle = osThreadNew(StartOledTask, NULL, &OledTask_attributes);
 8001b3c:	4a10      	ldr	r2, [pc, #64]	; (8001b80 <MX_FREERTOS_Init+0x8c>)
 8001b3e:	2100      	movs	r1, #0
 8001b40:	4810      	ldr	r0, [pc, #64]	; (8001b84 <MX_FREERTOS_Init+0x90>)
 8001b42:	f004 feeb 	bl	800691c <osThreadNew>
 8001b46:	4602      	mov	r2, r0
 8001b48:	4b0f      	ldr	r3, [pc, #60]	; (8001b88 <MX_FREERTOS_Init+0x94>)
 8001b4a:	601a      	str	r2, [r3, #0]

  /* USER CODE BEGIN RTOS_EVENTS */
  /* add events, ... */
  /* USER CODE END RTOS_EVENTS */

}
 8001b4c:	bf00      	nop
 8001b4e:	bd80      	pop	{r7, pc}
 8001b50:	08009f2c 	.word	0x08009f2c
 8001b54:	20004d48 	.word	0x20004d48
 8001b58:	08009f3c 	.word	0x08009f3c
 8001b5c:	20004d4c 	.word	0x20004d4c
 8001b60:	08009f4c 	.word	0x08009f4c
 8001b64:	20004d54 	.word	0x20004d54
 8001b68:	08009ec0 	.word	0x08009ec0
 8001b6c:	08001b8d 	.word	0x08001b8d
 8001b70:	20004d5c 	.word	0x20004d5c
 8001b74:	08009ee4 	.word	0x08009ee4
 8001b78:	08001bad 	.word	0x08001bad
 8001b7c:	20004d50 	.word	0x20004d50
 8001b80:	08009f08 	.word	0x08009f08
 8001b84:	08001c71 	.word	0x08001c71
 8001b88:	20004d44 	.word	0x20004d44

08001b8c <StartHeartbeatTask>:
  * @param  argument: Not used
  * @retval None
  */
/* USER CODE END Header_StartHeartbeatTask */
void StartHeartbeatTask(void *argument)
{
 8001b8c:	b580      	push	{r7, lr}
 8001b8e:	b082      	sub	sp, #8
 8001b90:	af00      	add	r7, sp, #0
 8001b92:	6078      	str	r0, [r7, #4]
  /* USER CODE BEGIN StartHeartbeatTask */
  /* Infinite loop */
  for(;;)
  {
	  HAL_GPIO_TogglePin(LD2_GPIO_Port, LD2_Pin);
 8001b94:	2120      	movs	r1, #32
 8001b96:	4804      	ldr	r0, [pc, #16]	; (8001ba8 <StartHeartbeatTask+0x1c>)
 8001b98:	f002 fb21 	bl	80041de <HAL_GPIO_TogglePin>
	  osDelay(500);
 8001b9c:	f44f 70fa 	mov.w	r0, #500	; 0x1f4
 8001ba0:	f004 ff62 	bl	8006a68 <osDelay>
	  HAL_GPIO_TogglePin(LD2_GPIO_Port, LD2_Pin);
 8001ba4:	e7f6      	b.n	8001b94 <StartHeartbeatTask+0x8>
 8001ba6:	bf00      	nop
 8001ba8:	40020000 	.word	0x40020000

08001bac <StartBmp280Task>:
* @param argument: Not used
* @retval None
*/
/* USER CODE END Header_StartBmp280Task */
void StartBmp280Task(void *argument)
{
 8001bac:	b5f0      	push	{r4, r5, r6, r7, lr}
 8001bae:	b091      	sub	sp, #68	; 0x44
 8001bb0:	af02      	add	r7, sp, #8
 8001bb2:	6078      	str	r0, [r7, #4]
  /* USER CODE BEGIN StartBmp280Task */
	BMP280_t Bmp280;
	float _Pressure, _Temperature;

	osMutexAcquire(MutexI2C1Handle, osWaitForever);
 8001bb4:	4b28      	ldr	r3, [pc, #160]	; (8001c58 <StartBmp280Task+0xac>)
 8001bb6:	681b      	ldr	r3, [r3, #0]
 8001bb8:	f04f 31ff 	mov.w	r1, #4294967295
 8001bbc:	4618      	mov	r0, r3
 8001bbe:	f005 f81b 	bl	8006bf8 <osMutexAcquire>
	BMP280_Init(&Bmp280, &hi2c1, 0x76);
 8001bc2:	f107 0314 	add.w	r3, r7, #20
 8001bc6:	2276      	movs	r2, #118	; 0x76
 8001bc8:	4924      	ldr	r1, [pc, #144]	; (8001c5c <StartBmp280Task+0xb0>)
 8001bca:	4618      	mov	r0, r3
 8001bcc:	f7ff fee8 	bl	80019a0 <BMP280_Init>
	osMutexRelease(MutexI2C1Handle);
 8001bd0:	4b21      	ldr	r3, [pc, #132]	; (8001c58 <StartBmp280Task+0xac>)
 8001bd2:	681b      	ldr	r3, [r3, #0]
 8001bd4:	4618      	mov	r0, r3
 8001bd6:	f005 f86d 	bl	8006cb4 <osMutexRelease>
  /* Infinite loop */
  for(;;)
  {
	  osMutexAcquire(MutexI2C1Handle, osWaitForever);
 8001bda:	4b1f      	ldr	r3, [pc, #124]	; (8001c58 <StartBmp280Task+0xac>)
 8001bdc:	681b      	ldr	r3, [r3, #0]
 8001bde:	f04f 31ff 	mov.w	r1, #4294967295
 8001be2:	4618      	mov	r0, r3
 8001be4:	f005 f808 	bl	8006bf8 <osMutexAcquire>
	  BMP280_ReadPressureAndTemperature(&Bmp280, &_Pressure, &_Temperature);
 8001be8:	f107 020c 	add.w	r2, r7, #12
 8001bec:	f107 0110 	add.w	r1, r7, #16
 8001bf0:	f107 0314 	add.w	r3, r7, #20
 8001bf4:	4618      	mov	r0, r3
 8001bf6:	f7ff fe1d 	bl	8001834 <BMP280_ReadPressureAndTemperature>
	  osMutexRelease(MutexI2C1Handle);
 8001bfa:	4b17      	ldr	r3, [pc, #92]	; (8001c58 <StartBmp280Task+0xac>)
 8001bfc:	681b      	ldr	r3, [r3, #0]
 8001bfe:	4618      	mov	r0, r3
 8001c00:	f005 f858 	bl	8006cb4 <osMutexRelease>

	  osMutexAcquire(MutexBmpDataHandle, osWaitForever);
 8001c04:	4b16      	ldr	r3, [pc, #88]	; (8001c60 <StartBmp280Task+0xb4>)
 8001c06:	681b      	ldr	r3, [r3, #0]
 8001c08:	f04f 31ff 	mov.w	r1, #4294967295
 8001c0c:	4618      	mov	r0, r3
 8001c0e:	f004 fff3 	bl	8006bf8 <osMutexAcquire>
	  Pressure = _Pressure;
 8001c12:	693b      	ldr	r3, [r7, #16]
 8001c14:	4a13      	ldr	r2, [pc, #76]	; (8001c64 <StartBmp280Task+0xb8>)
 8001c16:	6013      	str	r3, [r2, #0]
	  Temperature = _Temperature;
 8001c18:	68fb      	ldr	r3, [r7, #12]
 8001c1a:	4a13      	ldr	r2, [pc, #76]	; (8001c68 <StartBmp280Task+0xbc>)
 8001c1c:	6013      	str	r3, [r2, #0]
	  osMutexRelease(MutexBmpDataHandle);
 8001c1e:	4b10      	ldr	r3, [pc, #64]	; (8001c60 <StartBmp280Task+0xb4>)
 8001c20:	681b      	ldr	r3, [r3, #0]
 8001c22:	4618      	mov	r0, r3
 8001c24:	f005 f846 	bl	8006cb4 <osMutexRelease>

	  printf("Temperature: %.2f, Pressure: %.2f\n\r", _Temperature, _Pressure);
 8001c28:	68fb      	ldr	r3, [r7, #12]
 8001c2a:	4618      	mov	r0, r3
 8001c2c:	f7fe fc3c 	bl	80004a8 <__aeabi_f2d>
 8001c30:	4605      	mov	r5, r0
 8001c32:	460e      	mov	r6, r1
 8001c34:	693b      	ldr	r3, [r7, #16]
 8001c36:	4618      	mov	r0, r3
 8001c38:	f7fe fc36 	bl	80004a8 <__aeabi_f2d>
 8001c3c:	4603      	mov	r3, r0
 8001c3e:	460c      	mov	r4, r1
 8001c40:	e9cd 3400 	strd	r3, r4, [sp]
 8001c44:	462a      	mov	r2, r5
 8001c46:	4633      	mov	r3, r6
 8001c48:	4808      	ldr	r0, [pc, #32]	; (8001c6c <StartBmp280Task+0xc0>)
 8001c4a:	f001 fe7b 	bl	8003944 <printf_>

	  osDelay(10);
 8001c4e:	200a      	movs	r0, #10
 8001c50:	f004 ff0a 	bl	8006a68 <osDelay>
	  osMutexAcquire(MutexI2C1Handle, osWaitForever);
 8001c54:	e7c1      	b.n	8001bda <StartBmp280Task+0x2e>
 8001c56:	bf00      	nop
 8001c58:	20004d4c 	.word	0x20004d4c
 8001c5c:	20004d60 	.word	0x20004d60
 8001c60:	20004d54 	.word	0x20004d54
 8001c64:	20004d58 	.word	0x20004d58
 8001c68:	20004d40 	.word	0x20004d40
 8001c6c:	08009c68 	.word	0x08009c68

08001c70 <StartOledTask>:
* @param argument: Not used
* @retval None
*/
/* USER CODE END Header_StartOledTask */
void StartOledTask(void *argument)
{
 8001c70:	b590      	push	{r4, r7, lr}
 8001c72:	b091      	sub	sp, #68	; 0x44
 8001c74:	af02      	add	r7, sp, #8
 8001c76:	6078      	str	r0, [r7, #4]
  /* USER CODE BEGIN StartOledTask */
	char Message[32];
	uint8_t i = 0;
 8001c78:	2300      	movs	r3, #0
 8001c7a:	f887 3037 	strb.w	r3, [r7, #55]	; 0x37

	float _Pressure, _Temperature;

	osMutexAcquire(MutexI2C1Handle, osWaitForever);
 8001c7e:	4b44      	ldr	r3, [pc, #272]	; (8001d90 <StartOledTask+0x120>)
 8001c80:	681b      	ldr	r3, [r3, #0]
 8001c82:	f04f 31ff 	mov.w	r1, #4294967295
 8001c86:	4618      	mov	r0, r3
 8001c88:	f004 ffb6 	bl	8006bf8 <osMutexAcquire>
	SSD1306_Init(&hi2c1);
 8001c8c:	4841      	ldr	r0, [pc, #260]	; (8001d94 <StartOledTask+0x124>)
 8001c8e:	f7ff fc03 	bl	8001498 <SSD1306_Init>
	osMutexRelease(MutexI2C1Handle);
 8001c92:	4b3f      	ldr	r3, [pc, #252]	; (8001d90 <StartOledTask+0x120>)
 8001c94:	681b      	ldr	r3, [r3, #0]
 8001c96:	4618      	mov	r0, r3
 8001c98:	f005 f80c 	bl	8006cb4 <osMutexRelease>

	GFX_SetFont(font_8x5);
 8001c9c:	483e      	ldr	r0, [pc, #248]	; (8001d98 <StartOledTask+0x128>)
 8001c9e:	f7ff f90d 	bl	8000ebc <GFX_SetFont>

	SSD1306_Clear(BLACK);
 8001ca2:	2000      	movs	r0, #0
 8001ca4:	f7ff fbba 	bl	800141c <SSD1306_Clear>

	osMutexAcquire(MutexI2C1Handle, osWaitForever);
 8001ca8:	4b39      	ldr	r3, [pc, #228]	; (8001d90 <StartOledTask+0x120>)
 8001caa:	681b      	ldr	r3, [r3, #0]
 8001cac:	f04f 31ff 	mov.w	r1, #4294967295
 8001cb0:	4618      	mov	r0, r3
 8001cb2:	f004 ffa1 	bl	8006bf8 <osMutexAcquire>
	SSD1306_Display();
 8001cb6:	f7ff fbd1 	bl	800145c <SSD1306_Display>
	osMutexRelease(MutexI2C1Handle);
 8001cba:	4b35      	ldr	r3, [pc, #212]	; (8001d90 <StartOledTask+0x120>)
 8001cbc:	681b      	ldr	r3, [r3, #0]
 8001cbe:	4618      	mov	r0, r3
 8001cc0:	f004 fff8 	bl	8006cb4 <osMutexRelease>

  /* Infinite loop */
  for(;;)
  {
	SSD1306_Clear(BLACK);
 8001cc4:	2000      	movs	r0, #0
 8001cc6:	f7ff fba9 	bl	800141c <SSD1306_Clear>

	sprintf(Message, "Hello %d", i++);
 8001cca:	f897 3037 	ldrb.w	r3, [r7, #55]	; 0x37
 8001cce:	1c5a      	adds	r2, r3, #1
 8001cd0:	f887 2037 	strb.w	r2, [r7, #55]	; 0x37
 8001cd4:	461a      	mov	r2, r3
 8001cd6:	f107 030c 	add.w	r3, r7, #12
 8001cda:	4930      	ldr	r1, [pc, #192]	; (8001d9c <StartOledTask+0x12c>)
 8001cdc:	4618      	mov	r0, r3
 8001cde:	f001 fe4d 	bl	800397c <sprintf_>

	GFX_DrawString(0, 0, Message, WHITE, 0);
 8001ce2:	f107 020c 	add.w	r2, r7, #12
 8001ce6:	2300      	movs	r3, #0
 8001ce8:	9300      	str	r3, [sp, #0]
 8001cea:	2301      	movs	r3, #1
 8001cec:	2100      	movs	r1, #0
 8001cee:	2000      	movs	r0, #0
 8001cf0:	f7ff f9ae 	bl	8001050 <GFX_DrawString>

	osMutexAcquire(MutexBmpDataHandle, osWaitForever);
 8001cf4:	4b2a      	ldr	r3, [pc, #168]	; (8001da0 <StartOledTask+0x130>)
 8001cf6:	681b      	ldr	r3, [r3, #0]
 8001cf8:	f04f 31ff 	mov.w	r1, #4294967295
 8001cfc:	4618      	mov	r0, r3
 8001cfe:	f004 ff7b 	bl	8006bf8 <osMutexAcquire>
	_Pressure = Pressure;
 8001d02:	4b28      	ldr	r3, [pc, #160]	; (8001da4 <StartOledTask+0x134>)
 8001d04:	681b      	ldr	r3, [r3, #0]
 8001d06:	633b      	str	r3, [r7, #48]	; 0x30
	_Temperature = Temperature;
 8001d08:	4b27      	ldr	r3, [pc, #156]	; (8001da8 <StartOledTask+0x138>)
 8001d0a:	681b      	ldr	r3, [r3, #0]
 8001d0c:	62fb      	str	r3, [r7, #44]	; 0x2c
	osMutexRelease(MutexBmpDataHandle);
 8001d0e:	4b24      	ldr	r3, [pc, #144]	; (8001da0 <StartOledTask+0x130>)
 8001d10:	681b      	ldr	r3, [r3, #0]
 8001d12:	4618      	mov	r0, r3
 8001d14:	f004 ffce 	bl	8006cb4 <osMutexRelease>

	sprintf(Message, "Press: %.2f", _Pressure);
 8001d18:	6b38      	ldr	r0, [r7, #48]	; 0x30
 8001d1a:	f7fe fbc5 	bl	80004a8 <__aeabi_f2d>
 8001d1e:	4603      	mov	r3, r0
 8001d20:	460c      	mov	r4, r1
 8001d22:	f107 000c 	add.w	r0, r7, #12
 8001d26:	461a      	mov	r2, r3
 8001d28:	4623      	mov	r3, r4
 8001d2a:	4920      	ldr	r1, [pc, #128]	; (8001dac <StartOledTask+0x13c>)
 8001d2c:	f001 fe26 	bl	800397c <sprintf_>
	GFX_DrawString(0, 10, Message, WHITE, 0);
 8001d30:	f107 020c 	add.w	r2, r7, #12
 8001d34:	2300      	movs	r3, #0
 8001d36:	9300      	str	r3, [sp, #0]
 8001d38:	2301      	movs	r3, #1
 8001d3a:	210a      	movs	r1, #10
 8001d3c:	2000      	movs	r0, #0
 8001d3e:	f7ff f987 	bl	8001050 <GFX_DrawString>

	sprintf(Message, "Temp: %.2f", _Temperature);
 8001d42:	6af8      	ldr	r0, [r7, #44]	; 0x2c
 8001d44:	f7fe fbb0 	bl	80004a8 <__aeabi_f2d>
 8001d48:	4603      	mov	r3, r0
 8001d4a:	460c      	mov	r4, r1
 8001d4c:	f107 000c 	add.w	r0, r7, #12
 8001d50:	461a      	mov	r2, r3
 8001d52:	4623      	mov	r3, r4
 8001d54:	4916      	ldr	r1, [pc, #88]	; (8001db0 <StartOledTask+0x140>)
 8001d56:	f001 fe11 	bl	800397c <sprintf_>
	GFX_DrawString(0, 20, Message, WHITE, 0);
 8001d5a:	f107 020c 	add.w	r2, r7, #12
 8001d5e:	2300      	movs	r3, #0
 8001d60:	9300      	str	r3, [sp, #0]
 8001d62:	2301      	movs	r3, #1
 8001d64:	2114      	movs	r1, #20
 8001d66:	2000      	movs	r0, #0
 8001d68:	f7ff f972 	bl	8001050 <GFX_DrawString>

	osMutexAcquire(MutexI2C1Handle, osWaitForever);
 8001d6c:	4b08      	ldr	r3, [pc, #32]	; (8001d90 <StartOledTask+0x120>)
 8001d6e:	681b      	ldr	r3, [r3, #0]
 8001d70:	f04f 31ff 	mov.w	r1, #4294967295
 8001d74:	4618      	mov	r0, r3
 8001d76:	f004 ff3f 	bl	8006bf8 <osMutexAcquire>
	SSD1306_Display();
 8001d7a:	f7ff fb6f 	bl	800145c <SSD1306_Display>
	osMutexRelease(MutexI2C1Handle);
 8001d7e:	4b04      	ldr	r3, [pc, #16]	; (8001d90 <StartOledTask+0x120>)
 8001d80:	681b      	ldr	r3, [r3, #0]
 8001d82:	4618      	mov	r0, r3
 8001d84:	f004 ff96 	bl	8006cb4 <osMutexRelease>
    osDelay(100);
 8001d88:	2064      	movs	r0, #100	; 0x64
 8001d8a:	f004 fe6d 	bl	8006a68 <osDelay>
	SSD1306_Clear(BLACK);
 8001d8e:	e799      	b.n	8001cc4 <StartOledTask+0x54>
 8001d90:	20004d4c 	.word	0x20004d4c
 8001d94:	20004d60 	.word	0x20004d60
 8001d98:	08009ce0 	.word	0x08009ce0
 8001d9c:	08009c8c 	.word	0x08009c8c
 8001da0:	20004d54 	.word	0x20004d54
 8001da4:	20004d58 	.word	0x20004d58
 8001da8:	20004d40 	.word	0x20004d40
 8001dac:	08009c98 	.word	0x08009c98
 8001db0:	08009ca4 	.word	0x08009ca4

08001db4 <MX_GPIO_Init>:
        * Output
        * EVENT_OUT
        * EXTI
*/
void MX_GPIO_Init(void)
{
 8001db4:	b580      	push	{r7, lr}
 8001db6:	b08a      	sub	sp, #40	; 0x28
 8001db8:	af00      	add	r7, sp, #0

  GPIO_InitTypeDef GPIO_InitStruct = {0};
 8001dba:	f107 0314 	add.w	r3, r7, #20
 8001dbe:	2200      	movs	r2, #0
 8001dc0:	601a      	str	r2, [r3, #0]
 8001dc2:	605a      	str	r2, [r3, #4]
 8001dc4:	609a      	str	r2, [r3, #8]
 8001dc6:	60da      	str	r2, [r3, #12]
 8001dc8:	611a      	str	r2, [r3, #16]

  /* GPIO Ports Clock Enable */
  __HAL_RCC_GPIOC_CLK_ENABLE();
 8001dca:	2300      	movs	r3, #0
 8001dcc:	613b      	str	r3, [r7, #16]
 8001dce:	4b2d      	ldr	r3, [pc, #180]	; (8001e84 <MX_GPIO_Init+0xd0>)
 8001dd0:	6b1b      	ldr	r3, [r3, #48]	; 0x30
 8001dd2:	4a2c      	ldr	r2, [pc, #176]	; (8001e84 <MX_GPIO_Init+0xd0>)
 8001dd4:	f043 0304 	orr.w	r3, r3, #4
 8001dd8:	6313      	str	r3, [r2, #48]	; 0x30
 8001dda:	4b2a      	ldr	r3, [pc, #168]	; (8001e84 <MX_GPIO_Init+0xd0>)
 8001ddc:	6b1b      	ldr	r3, [r3, #48]	; 0x30
 8001dde:	f003 0304 	and.w	r3, r3, #4
 8001de2:	613b      	str	r3, [r7, #16]
 8001de4:	693b      	ldr	r3, [r7, #16]
  __HAL_RCC_GPIOH_CLK_ENABLE();
 8001de6:	2300      	movs	r3, #0
 8001de8:	60fb      	str	r3, [r7, #12]
 8001dea:	4b26      	ldr	r3, [pc, #152]	; (8001e84 <MX_GPIO_Init+0xd0>)
 8001dec:	6b1b      	ldr	r3, [r3, #48]	; 0x30
 8001dee:	4a25      	ldr	r2, [pc, #148]	; (8001e84 <MX_GPIO_Init+0xd0>)
 8001df0:	f043 0380 	orr.w	r3, r3, #128	; 0x80
 8001df4:	6313      	str	r3, [r2, #48]	; 0x30
 8001df6:	4b23      	ldr	r3, [pc, #140]	; (8001e84 <MX_GPIO_Init+0xd0>)
 8001df8:	6b1b      	ldr	r3, [r3, #48]	; 0x30
 8001dfa:	f003 0380 	and.w	r3, r3, #128	; 0x80
 8001dfe:	60fb      	str	r3, [r7, #12]
 8001e00:	68fb      	ldr	r3, [r7, #12]
  __HAL_RCC_GPIOA_CLK_ENABLE();
 8001e02:	2300      	movs	r3, #0
 8001e04:	60bb      	str	r3, [r7, #8]
 8001e06:	4b1f      	ldr	r3, [pc, #124]	; (8001e84 <MX_GPIO_Init+0xd0>)
 8001e08:	6b1b      	ldr	r3, [r3, #48]	; 0x30
 8001e0a:	4a1e      	ldr	r2, [pc, #120]	; (8001e84 <MX_GPIO_Init+0xd0>)
 8001e0c:	f043 0301 	orr.w	r3, r3, #1
 8001e10:	6313      	str	r3, [r2, #48]	; 0x30
 8001e12:	4b1c      	ldr	r3, [pc, #112]	; (8001e84 <MX_GPIO_Init+0xd0>)
 8001e14:	6b1b      	ldr	r3, [r3, #48]	; 0x30
 8001e16:	f003 0301 	and.w	r3, r3, #1
 8001e1a:	60bb      	str	r3, [r7, #8]
 8001e1c:	68bb      	ldr	r3, [r7, #8]
  __HAL_RCC_GPIOB_CLK_ENABLE();
 8001e1e:	2300      	movs	r3, #0
 8001e20:	607b      	str	r3, [r7, #4]
 8001e22:	4b18      	ldr	r3, [pc, #96]	; (8001e84 <MX_GPIO_Init+0xd0>)
 8001e24:	6b1b      	ldr	r3, [r3, #48]	; 0x30
 8001e26:	4a17      	ldr	r2, [pc, #92]	; (8001e84 <MX_GPIO_Init+0xd0>)
 8001e28:	f043 0302 	orr.w	r3, r3, #2
 8001e2c:	6313      	str	r3, [r2, #48]	; 0x30
 8001e2e:	4b15      	ldr	r3, [pc, #84]	; (8001e84 <MX_GPIO_Init+0xd0>)
 8001e30:	6b1b      	ldr	r3, [r3, #48]	; 0x30
 8001e32:	f003 0302 	and.w	r3, r3, #2
 8001e36:	607b      	str	r3, [r7, #4]
 8001e38:	687b      	ldr	r3, [r7, #4]

  /*Configure GPIO pin Output Level */
  HAL_GPIO_WritePin(LD2_GPIO_Port, LD2_Pin, GPIO_PIN_RESET);
 8001e3a:	2200      	movs	r2, #0
 8001e3c:	2120      	movs	r1, #32
 8001e3e:	4812      	ldr	r0, [pc, #72]	; (8001e88 <MX_GPIO_Init+0xd4>)
 8001e40:	f002 f9b4 	bl	80041ac <HAL_GPIO_WritePin>

  /*Configure GPIO pin : PtPin */
  GPIO_InitStruct.Pin = B1_Pin;
 8001e44:	f44f 5300 	mov.w	r3, #8192	; 0x2000
 8001e48:	617b      	str	r3, [r7, #20]
  GPIO_InitStruct.Mode = GPIO_MODE_IT_FALLING;
 8001e4a:	4b10      	ldr	r3, [pc, #64]	; (8001e8c <MX_GPIO_Init+0xd8>)
 8001e4c:	61bb      	str	r3, [r7, #24]
  GPIO_InitStruct.Pull = GPIO_NOPULL;
 8001e4e:	2300      	movs	r3, #0
 8001e50:	61fb      	str	r3, [r7, #28]
  HAL_GPIO_Init(B1_GPIO_Port, &GPIO_InitStruct);
 8001e52:	f107 0314 	add.w	r3, r7, #20
 8001e56:	4619      	mov	r1, r3
 8001e58:	480d      	ldr	r0, [pc, #52]	; (8001e90 <MX_GPIO_Init+0xdc>)
 8001e5a:	f002 f825 	bl	8003ea8 <HAL_GPIO_Init>

  /*Configure GPIO pin : PtPin */
  GPIO_InitStruct.Pin = LD2_Pin;
 8001e5e:	2320      	movs	r3, #32
 8001e60:	617b      	str	r3, [r7, #20]
  GPIO_InitStruct.Mode = GPIO_MODE_OUTPUT_PP;
 8001e62:	2301      	movs	r3, #1
 8001e64:	61bb      	str	r3, [r7, #24]
  GPIO_InitStruct.Pull = GPIO_NOPULL;
 8001e66:	2300      	movs	r3, #0
 8001e68:	61fb      	str	r3, [r7, #28]
  GPIO_InitStruct.Speed = GPIO_SPEED_FREQ_LOW;
 8001e6a:	2300      	movs	r3, #0
 8001e6c:	623b      	str	r3, [r7, #32]
  HAL_GPIO_Init(LD2_GPIO_Port, &GPIO_InitStruct);
 8001e6e:	f107 0314 	add.w	r3, r7, #20
 8001e72:	4619      	mov	r1, r3
 8001e74:	4804      	ldr	r0, [pc, #16]	; (8001e88 <MX_GPIO_Init+0xd4>)
 8001e76:	f002 f817 	bl	8003ea8 <HAL_GPIO_Init>

}
 8001e7a:	bf00      	nop
 8001e7c:	3728      	adds	r7, #40	; 0x28
 8001e7e:	46bd      	mov	sp, r7
 8001e80:	bd80      	pop	{r7, pc}
 8001e82:	bf00      	nop
 8001e84:	40023800 	.word	0x40023800
 8001e88:	40020000 	.word	0x40020000
 8001e8c:	10210000 	.word	0x10210000
 8001e90:	40020800 	.word	0x40020800

08001e94 <MX_I2C1_Init>:

I2C_HandleTypeDef hi2c1;

/* I2C1 init function */
void MX_I2C1_Init(void)
{
 8001e94:	b580      	push	{r7, lr}
 8001e96:	af00      	add	r7, sp, #0

  hi2c1.Instance = I2C1;
 8001e98:	4b12      	ldr	r3, [pc, #72]	; (8001ee4 <MX_I2C1_Init+0x50>)
 8001e9a:	4a13      	ldr	r2, [pc, #76]	; (8001ee8 <MX_I2C1_Init+0x54>)
 8001e9c:	601a      	str	r2, [r3, #0]
  hi2c1.Init.ClockSpeed = 400000;
 8001e9e:	4b11      	ldr	r3, [pc, #68]	; (8001ee4 <MX_I2C1_Init+0x50>)
 8001ea0:	4a12      	ldr	r2, [pc, #72]	; (8001eec <MX_I2C1_Init+0x58>)
 8001ea2:	605a      	str	r2, [r3, #4]
  hi2c1.Init.DutyCycle = I2C_DUTYCYCLE_2;
 8001ea4:	4b0f      	ldr	r3, [pc, #60]	; (8001ee4 <MX_I2C1_Init+0x50>)
 8001ea6:	2200      	movs	r2, #0
 8001ea8:	609a      	str	r2, [r3, #8]
  hi2c1.Init.OwnAddress1 = 0;
 8001eaa:	4b0e      	ldr	r3, [pc, #56]	; (8001ee4 <MX_I2C1_Init+0x50>)
 8001eac:	2200      	movs	r2, #0
 8001eae:	60da      	str	r2, [r3, #12]
  hi2c1.Init.AddressingMode = I2C_ADDRESSINGMODE_7BIT;
 8001eb0:	4b0c      	ldr	r3, [pc, #48]	; (8001ee4 <MX_I2C1_Init+0x50>)
 8001eb2:	f44f 4280 	mov.w	r2, #16384	; 0x4000
 8001eb6:	611a      	str	r2, [r3, #16]
  hi2c1.Init.DualAddressMode = I2C_DUALADDRESS_DISABLE;
 8001eb8:	4b0a      	ldr	r3, [pc, #40]	; (8001ee4 <MX_I2C1_Init+0x50>)
 8001eba:	2200      	movs	r2, #0
 8001ebc:	615a      	str	r2, [r3, #20]
  hi2c1.Init.OwnAddress2 = 0;
 8001ebe:	4b09      	ldr	r3, [pc, #36]	; (8001ee4 <MX_I2C1_Init+0x50>)
 8001ec0:	2200      	movs	r2, #0
 8001ec2:	619a      	str	r2, [r3, #24]
  hi2c1.Init.GeneralCallMode = I2C_GENERALCALL_DISABLE;
 8001ec4:	4b07      	ldr	r3, [pc, #28]	; (8001ee4 <MX_I2C1_Init+0x50>)
 8001ec6:	2200      	movs	r2, #0
 8001ec8:	61da      	str	r2, [r3, #28]
  hi2c1.Init.NoStretchMode = I2C_NOSTRETCH_DISABLE;
 8001eca:	4b06      	ldr	r3, [pc, #24]	; (8001ee4 <MX_I2C1_Init+0x50>)
 8001ecc:	2200      	movs	r2, #0
 8001ece:	621a      	str	r2, [r3, #32]
  if (HAL_I2C_Init(&hi2c1) != HAL_OK)
 8001ed0:	4804      	ldr	r0, [pc, #16]	; (8001ee4 <MX_I2C1_Init+0x50>)
 8001ed2:	f002 f99f 	bl	8004214 <HAL_I2C_Init>
 8001ed6:	4603      	mov	r3, r0
 8001ed8:	2b00      	cmp	r3, #0
 8001eda:	d001      	beq.n	8001ee0 <MX_I2C1_Init+0x4c>
  {
    Error_Handler();
 8001edc:	f000 f8e0 	bl	80020a0 <Error_Handler>
  }

}
 8001ee0:	bf00      	nop
 8001ee2:	bd80      	pop	{r7, pc}
 8001ee4:	20004d60 	.word	0x20004d60
 8001ee8:	40005400 	.word	0x40005400
 8001eec:	00061a80 	.word	0x00061a80

08001ef0 <HAL_I2C_MspInit>:

void HAL_I2C_MspInit(I2C_HandleTypeDef* i2cHandle)
{
 8001ef0:	b580      	push	{r7, lr}
 8001ef2:	b08a      	sub	sp, #40	; 0x28
 8001ef4:	af00      	add	r7, sp, #0
 8001ef6:	6078      	str	r0, [r7, #4]

  GPIO_InitTypeDef GPIO_InitStruct = {0};
 8001ef8:	f107 0314 	add.w	r3, r7, #20
 8001efc:	2200      	movs	r2, #0
 8001efe:	601a      	str	r2, [r3, #0]
 8001f00:	605a      	str	r2, [r3, #4]
 8001f02:	609a      	str	r2, [r3, #8]
 8001f04:	60da      	str	r2, [r3, #12]
 8001f06:	611a      	str	r2, [r3, #16]
  if(i2cHandle->Instance==I2C1)
 8001f08:	687b      	ldr	r3, [r7, #4]
 8001f0a:	681b      	ldr	r3, [r3, #0]
 8001f0c:	4a19      	ldr	r2, [pc, #100]	; (8001f74 <HAL_I2C_MspInit+0x84>)
 8001f0e:	4293      	cmp	r3, r2
 8001f10:	d12c      	bne.n	8001f6c <HAL_I2C_MspInit+0x7c>
  {
  /* USER CODE BEGIN I2C1_MspInit 0 */

  /* USER CODE END I2C1_MspInit 0 */

    __HAL_RCC_GPIOB_CLK_ENABLE();
 8001f12:	2300      	movs	r3, #0
 8001f14:	613b      	str	r3, [r7, #16]
 8001f16:	4b18      	ldr	r3, [pc, #96]	; (8001f78 <HAL_I2C_MspInit+0x88>)
 8001f18:	6b1b      	ldr	r3, [r3, #48]	; 0x30
 8001f1a:	4a17      	ldr	r2, [pc, #92]	; (8001f78 <HAL_I2C_MspInit+0x88>)
 8001f1c:	f043 0302 	orr.w	r3, r3, #2
 8001f20:	6313      	str	r3, [r2, #48]	; 0x30
 8001f22:	4b15      	ldr	r3, [pc, #84]	; (8001f78 <HAL_I2C_MspInit+0x88>)
 8001f24:	6b1b      	ldr	r3, [r3, #48]	; 0x30
 8001f26:	f003 0302 	and.w	r3, r3, #2
 8001f2a:	613b      	str	r3, [r7, #16]
 8001f2c:	693b      	ldr	r3, [r7, #16]
    /**I2C1 GPIO Configuration
    PB8     ------> I2C1_SCL
    PB9     ------> I2C1_SDA
    */
    GPIO_InitStruct.Pin = GPIO_PIN_8|GPIO_PIN_9;
 8001f2e:	f44f 7340 	mov.w	r3, #768	; 0x300
 8001f32:	617b      	str	r3, [r7, #20]
    GPIO_InitStruct.Mode = GPIO_MODE_AF_OD;
 8001f34:	2312      	movs	r3, #18
 8001f36:	61bb      	str	r3, [r7, #24]
    GPIO_InitStruct.Pull = GPIO_PULLUP;
 8001f38:	2301      	movs	r3, #1
 8001f3a:	61fb      	str	r3, [r7, #28]
    GPIO_InitStruct.Speed = GPIO_SPEED_FREQ_VERY_HIGH;
 8001f3c:	2303      	movs	r3, #3
 8001f3e:	623b      	str	r3, [r7, #32]
    GPIO_InitStruct.Alternate = GPIO_AF4_I2C1;
 8001f40:	2304      	movs	r3, #4
 8001f42:	627b      	str	r3, [r7, #36]	; 0x24
    HAL_GPIO_Init(GPIOB, &GPIO_InitStruct);
 8001f44:	f107 0314 	add.w	r3, r7, #20
 8001f48:	4619      	mov	r1, r3
 8001f4a:	480c      	ldr	r0, [pc, #48]	; (8001f7c <HAL_I2C_MspInit+0x8c>)
 8001f4c:	f001 ffac 	bl	8003ea8 <HAL_GPIO_Init>

    /* I2C1 clock enable */
    __HAL_RCC_I2C1_CLK_ENABLE();
 8001f50:	2300      	movs	r3, #0
 8001f52:	60fb      	str	r3, [r7, #12]
 8001f54:	4b08      	ldr	r3, [pc, #32]	; (8001f78 <HAL_I2C_MspInit+0x88>)
 8001f56:	6c1b      	ldr	r3, [r3, #64]	; 0x40
 8001f58:	4a07      	ldr	r2, [pc, #28]	; (8001f78 <HAL_I2C_MspInit+0x88>)
 8001f5a:	f443 1300 	orr.w	r3, r3, #2097152	; 0x200000
 8001f5e:	6413      	str	r3, [r2, #64]	; 0x40
 8001f60:	4b05      	ldr	r3, [pc, #20]	; (8001f78 <HAL_I2C_MspInit+0x88>)
 8001f62:	6c1b      	ldr	r3, [r3, #64]	; 0x40
 8001f64:	f403 1300 	and.w	r3, r3, #2097152	; 0x200000
 8001f68:	60fb      	str	r3, [r7, #12]
 8001f6a:	68fb      	ldr	r3, [r7, #12]
  /* USER CODE BEGIN I2C1_MspInit 1 */

  /* USER CODE END I2C1_MspInit 1 */
  }
}
 8001f6c:	bf00      	nop
 8001f6e:	3728      	adds	r7, #40	; 0x28
 8001f70:	46bd      	mov	sp, r7
 8001f72:	bd80      	pop	{r7, pc}
 8001f74:	40005400 	.word	0x40005400
 8001f78:	40023800 	.word	0x40023800
 8001f7c:	40020400 	.word	0x40020400

08001f80 <main>:
/**
  * @brief  The application entry point.
  * @retval int
  */
int main(void)
{
 8001f80:	b580      	push	{r7, lr}
 8001f82:	af00      	add	r7, sp, #0
  /* USER CODE END 1 */

  /* MCU Configuration--------------------------------------------------------*/

  /* Reset of all peripherals, Initializes the Flash interface and the Systick. */
  HAL_Init();
 8001f84:	f001 fe6c 	bl	8003c60 <HAL_Init>
  /* USER CODE BEGIN Init */

  /* USER CODE END Init */

  /* Configure the system clock */
  SystemClock_Config();
 8001f88:	f000 f80e 	bl	8001fa8 <SystemClock_Config>
  /* USER CODE BEGIN SysInit */

  /* USER CODE END SysInit */

  /* Initialize all configured peripherals */
  MX_GPIO_Init();
 8001f8c:	f7ff ff12 	bl	8001db4 <MX_GPIO_Init>
  MX_USART2_UART_Init();
 8001f90:	f001 fdca 	bl	8003b28 <MX_USART2_UART_Init>
  MX_I2C1_Init();
 8001f94:	f7ff ff7e 	bl	8001e94 <MX_I2C1_Init>
  /* USER CODE BEGIN 2 */

  /* USER CODE END 2 */

  /* Init scheduler */
  osKernelInitialize();  /* Call init function for freertos objects (in freertos.c) */
 8001f98:	f004 fc56 	bl	8006848 <osKernelInitialize>
  MX_FREERTOS_Init();
 8001f9c:	f7ff fdaa 	bl	8001af4 <MX_FREERTOS_Init>
  /* Start scheduler */
  osKernelStart();
 8001fa0:	f004 fc86 	bl	80068b0 <osKernelStart>

  /* We should never get here as control is now taken by the scheduler */
  /* Infinite loop */
  /* USER CODE BEGIN WHILE */
  while (1)
 8001fa4:	e7fe      	b.n	8001fa4 <main+0x24>
	...

08001fa8 <SystemClock_Config>:
/**
  * @brief System Clock Configuration
  * @retval None
  */
void SystemClock_Config(void)
{
 8001fa8:	b580      	push	{r7, lr}
 8001faa:	b094      	sub	sp, #80	; 0x50
 8001fac:	af00      	add	r7, sp, #0
  RCC_OscInitTypeDef RCC_OscInitStruct = {0};
 8001fae:	f107 0320 	add.w	r3, r7, #32
 8001fb2:	2230      	movs	r2, #48	; 0x30
 8001fb4:	2100      	movs	r1, #0
 8001fb6:	4618      	mov	r0, r3
 8001fb8:	f007 fe17 	bl	8009bea <memset>
  RCC_ClkInitTypeDef RCC_ClkInitStruct = {0};
 8001fbc:	f107 030c 	add.w	r3, r7, #12
 8001fc0:	2200      	movs	r2, #0
 8001fc2:	601a      	str	r2, [r3, #0]
 8001fc4:	605a      	str	r2, [r3, #4]
 8001fc6:	609a      	str	r2, [r3, #8]
 8001fc8:	60da      	str	r2, [r3, #12]
 8001fca:	611a      	str	r2, [r3, #16]

  /** Configure the main internal regulator output voltage
  */
  __HAL_RCC_PWR_CLK_ENABLE();
 8001fcc:	2300      	movs	r3, #0
 8001fce:	60bb      	str	r3, [r7, #8]
 8001fd0:	4b28      	ldr	r3, [pc, #160]	; (8002074 <SystemClock_Config+0xcc>)
 8001fd2:	6c1b      	ldr	r3, [r3, #64]	; 0x40
 8001fd4:	4a27      	ldr	r2, [pc, #156]	; (8002074 <SystemClock_Config+0xcc>)
 8001fd6:	f043 5380 	orr.w	r3, r3, #268435456	; 0x10000000
 8001fda:	6413      	str	r3, [r2, #64]	; 0x40
 8001fdc:	4b25      	ldr	r3, [pc, #148]	; (8002074 <SystemClock_Config+0xcc>)
 8001fde:	6c1b      	ldr	r3, [r3, #64]	; 0x40
 8001fe0:	f003 5380 	and.w	r3, r3, #268435456	; 0x10000000
 8001fe4:	60bb      	str	r3, [r7, #8]
 8001fe6:	68bb      	ldr	r3, [r7, #8]
  __HAL_PWR_VOLTAGESCALING_CONFIG(PWR_REGULATOR_VOLTAGE_SCALE1);
 8001fe8:	2300      	movs	r3, #0
 8001fea:	607b      	str	r3, [r7, #4]
 8001fec:	4b22      	ldr	r3, [pc, #136]	; (8002078 <SystemClock_Config+0xd0>)
 8001fee:	681b      	ldr	r3, [r3, #0]
 8001ff0:	4a21      	ldr	r2, [pc, #132]	; (8002078 <SystemClock_Config+0xd0>)
 8001ff2:	f443 4340 	orr.w	r3, r3, #49152	; 0xc000
 8001ff6:	6013      	str	r3, [r2, #0]
 8001ff8:	4b1f      	ldr	r3, [pc, #124]	; (8002078 <SystemClock_Config+0xd0>)
 8001ffa:	681b      	ldr	r3, [r3, #0]
 8001ffc:	f403 4340 	and.w	r3, r3, #49152	; 0xc000
 8002000:	607b      	str	r3, [r7, #4]
 8002002:	687b      	ldr	r3, [r7, #4]
  /** Initializes the RCC Oscillators according to the specified parameters
  * in the RCC_OscInitTypeDef structure.
  */
  RCC_OscInitStruct.OscillatorType = RCC_OSCILLATORTYPE_HSI;
 8002004:	2302      	movs	r3, #2
 8002006:	623b      	str	r3, [r7, #32]
  RCC_OscInitStruct.HSIState = RCC_HSI_ON;
 8002008:	2301      	movs	r3, #1
 800200a:	62fb      	str	r3, [r7, #44]	; 0x2c
  RCC_OscInitStruct.HSICalibrationValue = RCC_HSICALIBRATION_DEFAULT;
 800200c:	2310      	movs	r3, #16
 800200e:	633b      	str	r3, [r7, #48]	; 0x30
  RCC_OscInitStruct.PLL.PLLState = RCC_PLL_ON;
 8002010:	2302      	movs	r3, #2
 8002012:	63bb      	str	r3, [r7, #56]	; 0x38
  RCC_OscInitStruct.PLL.PLLSource = RCC_PLLSOURCE_HSI;
 8002014:	2300      	movs	r3, #0
 8002016:	63fb      	str	r3, [r7, #60]	; 0x3c
  RCC_OscInitStruct.PLL.PLLM = 16;
 8002018:	2310      	movs	r3, #16
 800201a:	643b      	str	r3, [r7, #64]	; 0x40
  RCC_OscInitStruct.PLL.PLLN = 336;
 800201c:	f44f 73a8 	mov.w	r3, #336	; 0x150
 8002020:	647b      	str	r3, [r7, #68]	; 0x44
  RCC_OscInitStruct.PLL.PLLP = RCC_PLLP_DIV4;
 8002022:	2304      	movs	r3, #4
 8002024:	64bb      	str	r3, [r7, #72]	; 0x48
  RCC_OscInitStruct.PLL.PLLQ = 4;
 8002026:	2304      	movs	r3, #4
 8002028:	64fb      	str	r3, [r7, #76]	; 0x4c
  if (HAL_RCC_OscConfig(&RCC_OscInitStruct) != HAL_OK)
 800202a:	f107 0320 	add.w	r3, r7, #32
 800202e:	4618      	mov	r0, r3
 8002030:	f003 f8a4 	bl	800517c <HAL_RCC_OscConfig>
 8002034:	4603      	mov	r3, r0
 8002036:	2b00      	cmp	r3, #0
 8002038:	d001      	beq.n	800203e <SystemClock_Config+0x96>
  {
    Error_Handler();
 800203a:	f000 f831 	bl	80020a0 <Error_Handler>
  }
  /** Initializes the CPU, AHB and APB buses clocks
  */
  RCC_ClkInitStruct.ClockType = RCC_CLOCKTYPE_HCLK|RCC_CLOCKTYPE_SYSCLK
 800203e:	230f      	movs	r3, #15
 8002040:	60fb      	str	r3, [r7, #12]
                              |RCC_CLOCKTYPE_PCLK1|RCC_CLOCKTYPE_PCLK2;
  RCC_ClkInitStruct.SYSCLKSource = RCC_SYSCLKSOURCE_PLLCLK;
 8002042:	2302      	movs	r3, #2
 8002044:	613b      	str	r3, [r7, #16]
  RCC_ClkInitStruct.AHBCLKDivider = RCC_SYSCLK_DIV1;
 8002046:	2300      	movs	r3, #0
 8002048:	617b      	str	r3, [r7, #20]
  RCC_ClkInitStruct.APB1CLKDivider = RCC_HCLK_DIV2;
 800204a:	f44f 5380 	mov.w	r3, #4096	; 0x1000
 800204e:	61bb      	str	r3, [r7, #24]
  RCC_ClkInitStruct.APB2CLKDivider = RCC_HCLK_DIV1;
 8002050:	2300      	movs	r3, #0
 8002052:	61fb      	str	r3, [r7, #28]

  if (HAL_RCC_ClockConfig(&RCC_ClkInitStruct, FLASH_LATENCY_2) != HAL_OK)
 8002054:	f107 030c 	add.w	r3, r7, #12
 8002058:	2102      	movs	r1, #2
 800205a:	4618      	mov	r0, r3
 800205c:	f003 fafe 	bl	800565c <HAL_RCC_ClockConfig>
 8002060:	4603      	mov	r3, r0
 8002062:	2b00      	cmp	r3, #0
 8002064:	d001      	beq.n	800206a <SystemClock_Config+0xc2>
  {
    Error_Handler();
 8002066:	f000 f81b 	bl	80020a0 <Error_Handler>
  }
}
 800206a:	bf00      	nop
 800206c:	3750      	adds	r7, #80	; 0x50
 800206e:	46bd      	mov	sp, r7
 8002070:	bd80      	pop	{r7, pc}
 8002072:	bf00      	nop
 8002074:	40023800 	.word	0x40023800
 8002078:	40007000 	.word	0x40007000

0800207c <HAL_TIM_PeriodElapsedCallback>:
  * a global variable "uwTick" used as application time base.
  * @param  htim : TIM handle
  * @retval None
  */
void HAL_TIM_PeriodElapsedCallback(TIM_HandleTypeDef *htim)
{
 800207c:	b580      	push	{r7, lr}
 800207e:	b082      	sub	sp, #8
 8002080:	af00      	add	r7, sp, #0
 8002082:	6078      	str	r0, [r7, #4]
  /* USER CODE BEGIN Callback 0 */

  /* USER CODE END Callback 0 */
  if (htim->Instance == TIM10) {
 8002084:	687b      	ldr	r3, [r7, #4]
 8002086:	681b      	ldr	r3, [r3, #0]
 8002088:	4a04      	ldr	r2, [pc, #16]	; (800209c <HAL_TIM_PeriodElapsedCallback+0x20>)
 800208a:	4293      	cmp	r3, r2
 800208c:	d101      	bne.n	8002092 <HAL_TIM_PeriodElapsedCallback+0x16>
    HAL_IncTick();
 800208e:	f001 fe09 	bl	8003ca4 <HAL_IncTick>
  }
  /* USER CODE BEGIN Callback 1 */

  /* USER CODE END Callback 1 */
}
 8002092:	bf00      	nop
 8002094:	3708      	adds	r7, #8
 8002096:	46bd      	mov	sp, r7
 8002098:	bd80      	pop	{r7, pc}
 800209a:	bf00      	nop
 800209c:	40014400 	.word	0x40014400

080020a0 <Error_Handler>:
/**
  * @brief  This function is executed in case of error occurrence.
  * @retval None
  */
void Error_Handler(void)
{
 80020a0:	b480      	push	{r7}
 80020a2:	af00      	add	r7, sp, #0
  \details Disables IRQ interrupts by setting the I-bit in the CPSR.
           Can only be executed in Privileged modes.
 */
__STATIC_FORCEINLINE void __disable_irq(void)
{
  __ASM volatile ("cpsid i" : : : "memory");
 80020a4:	b672      	cpsid	i
  /* USER CODE BEGIN Error_Handler_Debug */
  /* User can add his own implementation to report the HAL error return state */
  __disable_irq();
  while (1)
 80020a6:	e7fe      	b.n	80020a6 <Error_Handler+0x6>

080020a8 <_out_buffer>:
} out_fct_wrap_type;


// internal buffer output
static inline void _out_buffer(char character, void* buffer, size_t idx, size_t maxlen)
{
 80020a8:	b480      	push	{r7}
 80020aa:	b085      	sub	sp, #20
 80020ac:	af00      	add	r7, sp, #0
 80020ae:	60b9      	str	r1, [r7, #8]
 80020b0:	607a      	str	r2, [r7, #4]
 80020b2:	603b      	str	r3, [r7, #0]
 80020b4:	4603      	mov	r3, r0
 80020b6:	73fb      	strb	r3, [r7, #15]
  if (idx < maxlen) {
 80020b8:	687a      	ldr	r2, [r7, #4]
 80020ba:	683b      	ldr	r3, [r7, #0]
 80020bc:	429a      	cmp	r2, r3
 80020be:	d204      	bcs.n	80020ca <_out_buffer+0x22>
    ((char*)buffer)[idx] = character;
 80020c0:	68ba      	ldr	r2, [r7, #8]
 80020c2:	687b      	ldr	r3, [r7, #4]
 80020c4:	4413      	add	r3, r2
 80020c6:	7bfa      	ldrb	r2, [r7, #15]
 80020c8:	701a      	strb	r2, [r3, #0]
  }
}
 80020ca:	bf00      	nop
 80020cc:	3714      	adds	r7, #20
 80020ce:	46bd      	mov	sp, r7
 80020d0:	f85d 7b04 	ldr.w	r7, [sp], #4
 80020d4:	4770      	bx	lr

080020d6 <_out_null>:


// internal null output
static inline void _out_null(char character, void* buffer, size_t idx, size_t maxlen)
{
 80020d6:	b480      	push	{r7}
 80020d8:	b085      	sub	sp, #20
 80020da:	af00      	add	r7, sp, #0
 80020dc:	60b9      	str	r1, [r7, #8]
 80020de:	607a      	str	r2, [r7, #4]
 80020e0:	603b      	str	r3, [r7, #0]
 80020e2:	4603      	mov	r3, r0
 80020e4:	73fb      	strb	r3, [r7, #15]
  (void)character; (void)buffer; (void)idx; (void)maxlen;
}
 80020e6:	bf00      	nop
 80020e8:	3714      	adds	r7, #20
 80020ea:	46bd      	mov	sp, r7
 80020ec:	f85d 7b04 	ldr.w	r7, [sp], #4
 80020f0:	4770      	bx	lr

080020f2 <_out_char>:


// internal _putchar wrapper
static inline void _out_char(char character, void* buffer, size_t idx, size_t maxlen)
{
 80020f2:	b580      	push	{r7, lr}
 80020f4:	b084      	sub	sp, #16
 80020f6:	af00      	add	r7, sp, #0
 80020f8:	60b9      	str	r1, [r7, #8]
 80020fa:	607a      	str	r2, [r7, #4]
 80020fc:	603b      	str	r3, [r7, #0]
 80020fe:	4603      	mov	r3, r0
 8002100:	73fb      	strb	r3, [r7, #15]
  (void)buffer; (void)idx; (void)maxlen;
  if (character) {
 8002102:	7bfb      	ldrb	r3, [r7, #15]
 8002104:	2b00      	cmp	r3, #0
 8002106:	d003      	beq.n	8002110 <_out_char+0x1e>
    _putchar(character);
 8002108:	7bfb      	ldrb	r3, [r7, #15]
 800210a:	4618      	mov	r0, r3
 800210c:	f7ff fcd2 	bl	8001ab4 <_putchar>
  }
}
 8002110:	bf00      	nop
 8002112:	3710      	adds	r7, #16
 8002114:	46bd      	mov	sp, r7
 8002116:	bd80      	pop	{r7, pc}

08002118 <_strnlen_s>:


// internal secure strlen
// \return The length of the string (excluding the terminating 0) limited by 'maxsize'
static inline unsigned int _strnlen_s(const char* str, size_t maxsize)
{
 8002118:	b480      	push	{r7}
 800211a:	b085      	sub	sp, #20
 800211c:	af00      	add	r7, sp, #0
 800211e:	6078      	str	r0, [r7, #4]
 8002120:	6039      	str	r1, [r7, #0]
  const char* s;
  for (s = str; *s && maxsize--; ++s);
 8002122:	687b      	ldr	r3, [r7, #4]
 8002124:	60fb      	str	r3, [r7, #12]
 8002126:	e002      	b.n	800212e <_strnlen_s+0x16>
 8002128:	68fb      	ldr	r3, [r7, #12]
 800212a:	3301      	adds	r3, #1
 800212c:	60fb      	str	r3, [r7, #12]
 800212e:	68fb      	ldr	r3, [r7, #12]
 8002130:	781b      	ldrb	r3, [r3, #0]
 8002132:	2b00      	cmp	r3, #0
 8002134:	d004      	beq.n	8002140 <_strnlen_s+0x28>
 8002136:	683b      	ldr	r3, [r7, #0]
 8002138:	1e5a      	subs	r2, r3, #1
 800213a:	603a      	str	r2, [r7, #0]
 800213c:	2b00      	cmp	r3, #0
 800213e:	d1f3      	bne.n	8002128 <_strnlen_s+0x10>
  return (unsigned int)(s - str);
 8002140:	68fa      	ldr	r2, [r7, #12]
 8002142:	687b      	ldr	r3, [r7, #4]
 8002144:	1ad3      	subs	r3, r2, r3
}
 8002146:	4618      	mov	r0, r3
 8002148:	3714      	adds	r7, #20
 800214a:	46bd      	mov	sp, r7
 800214c:	f85d 7b04 	ldr.w	r7, [sp], #4
 8002150:	4770      	bx	lr

08002152 <_is_digit>:


// internal test if char is a digit (0-9)
// \return true if char is a digit
static inline bool _is_digit(char ch)
{
 8002152:	b480      	push	{r7}
 8002154:	b083      	sub	sp, #12
 8002156:	af00      	add	r7, sp, #0
 8002158:	4603      	mov	r3, r0
 800215a:	71fb      	strb	r3, [r7, #7]
  return (ch >= '0') && (ch <= '9');
 800215c:	79fb      	ldrb	r3, [r7, #7]
 800215e:	2b2f      	cmp	r3, #47	; 0x2f
 8002160:	d904      	bls.n	800216c <_is_digit+0x1a>
 8002162:	79fb      	ldrb	r3, [r7, #7]
 8002164:	2b39      	cmp	r3, #57	; 0x39
 8002166:	d801      	bhi.n	800216c <_is_digit+0x1a>
 8002168:	2301      	movs	r3, #1
 800216a:	e000      	b.n	800216e <_is_digit+0x1c>
 800216c:	2300      	movs	r3, #0
 800216e:	f003 0301 	and.w	r3, r3, #1
 8002172:	b2db      	uxtb	r3, r3
}
 8002174:	4618      	mov	r0, r3
 8002176:	370c      	adds	r7, #12
 8002178:	46bd      	mov	sp, r7
 800217a:	f85d 7b04 	ldr.w	r7, [sp], #4
 800217e:	4770      	bx	lr

08002180 <_atoi>:


// internal ASCII string to unsigned int conversion
static unsigned int _atoi(const char** str)
{
 8002180:	b580      	push	{r7, lr}
 8002182:	b084      	sub	sp, #16
 8002184:	af00      	add	r7, sp, #0
 8002186:	6078      	str	r0, [r7, #4]
  unsigned int i = 0U;
 8002188:	2300      	movs	r3, #0
 800218a:	60fb      	str	r3, [r7, #12]
  while (_is_digit(**str)) {
 800218c:	e00e      	b.n	80021ac <_atoi+0x2c>
    i = i * 10U + (unsigned int)(*((*str)++) - '0');
 800218e:	68fa      	ldr	r2, [r7, #12]
 8002190:	4613      	mov	r3, r2
 8002192:	009b      	lsls	r3, r3, #2
 8002194:	4413      	add	r3, r2
 8002196:	005b      	lsls	r3, r3, #1
 8002198:	4618      	mov	r0, r3
 800219a:	687b      	ldr	r3, [r7, #4]
 800219c:	681b      	ldr	r3, [r3, #0]
 800219e:	1c59      	adds	r1, r3, #1
 80021a0:	687a      	ldr	r2, [r7, #4]
 80021a2:	6011      	str	r1, [r2, #0]
 80021a4:	781b      	ldrb	r3, [r3, #0]
 80021a6:	4403      	add	r3, r0
 80021a8:	3b30      	subs	r3, #48	; 0x30
 80021aa:	60fb      	str	r3, [r7, #12]
  while (_is_digit(**str)) {
 80021ac:	687b      	ldr	r3, [r7, #4]
 80021ae:	681b      	ldr	r3, [r3, #0]
 80021b0:	781b      	ldrb	r3, [r3, #0]
 80021b2:	4618      	mov	r0, r3
 80021b4:	f7ff ffcd 	bl	8002152 <_is_digit>
 80021b8:	4603      	mov	r3, r0
 80021ba:	2b00      	cmp	r3, #0
 80021bc:	d1e7      	bne.n	800218e <_atoi+0xe>
  }
  return i;
 80021be:	68fb      	ldr	r3, [r7, #12]
}
 80021c0:	4618      	mov	r0, r3
 80021c2:	3710      	adds	r7, #16
 80021c4:	46bd      	mov	sp, r7
 80021c6:	bd80      	pop	{r7, pc}

080021c8 <_out_rev>:


// output the specified string in reverse, taking care of any zero-padding
static size_t _out_rev(out_fct_type out, char* buffer, size_t idx, size_t maxlen, const char* buf, size_t len, unsigned int width, unsigned int flags)
{
 80021c8:	b590      	push	{r4, r7, lr}
 80021ca:	b087      	sub	sp, #28
 80021cc:	af00      	add	r7, sp, #0
 80021ce:	60f8      	str	r0, [r7, #12]
 80021d0:	60b9      	str	r1, [r7, #8]
 80021d2:	607a      	str	r2, [r7, #4]
 80021d4:	603b      	str	r3, [r7, #0]
  const size_t start_idx = idx;
 80021d6:	687b      	ldr	r3, [r7, #4]
 80021d8:	613b      	str	r3, [r7, #16]

  // pad spaces up to given width
  if (!(flags & FLAGS_LEFT) && !(flags & FLAGS_ZEROPAD)) {
 80021da:	6b7b      	ldr	r3, [r7, #52]	; 0x34
 80021dc:	f003 0302 	and.w	r3, r3, #2
 80021e0:	2b00      	cmp	r3, #0
 80021e2:	d125      	bne.n	8002230 <_out_rev+0x68>
 80021e4:	6b7b      	ldr	r3, [r7, #52]	; 0x34
 80021e6:	f003 0301 	and.w	r3, r3, #1
 80021ea:	2b00      	cmp	r3, #0
 80021ec:	d120      	bne.n	8002230 <_out_rev+0x68>
    for (size_t i = len; i < width; i++) {
 80021ee:	6afb      	ldr	r3, [r7, #44]	; 0x2c
 80021f0:	617b      	str	r3, [r7, #20]
 80021f2:	e00a      	b.n	800220a <_out_rev+0x42>
      out(' ', buffer, idx++, maxlen);
 80021f4:	687a      	ldr	r2, [r7, #4]
 80021f6:	1c53      	adds	r3, r2, #1
 80021f8:	607b      	str	r3, [r7, #4]
 80021fa:	68fc      	ldr	r4, [r7, #12]
 80021fc:	683b      	ldr	r3, [r7, #0]
 80021fe:	68b9      	ldr	r1, [r7, #8]
 8002200:	2020      	movs	r0, #32
 8002202:	47a0      	blx	r4
    for (size_t i = len; i < width; i++) {
 8002204:	697b      	ldr	r3, [r7, #20]
 8002206:	3301      	adds	r3, #1
 8002208:	617b      	str	r3, [r7, #20]
 800220a:	697a      	ldr	r2, [r7, #20]
 800220c:	6b3b      	ldr	r3, [r7, #48]	; 0x30
 800220e:	429a      	cmp	r2, r3
 8002210:	d3f0      	bcc.n	80021f4 <_out_rev+0x2c>
    }
  }

  // reverse string
  while (len) {
 8002212:	e00d      	b.n	8002230 <_out_rev+0x68>
    out(buf[--len], buffer, idx++, maxlen);
 8002214:	6afb      	ldr	r3, [r7, #44]	; 0x2c
 8002216:	3b01      	subs	r3, #1
 8002218:	62fb      	str	r3, [r7, #44]	; 0x2c
 800221a:	6aba      	ldr	r2, [r7, #40]	; 0x28
 800221c:	6afb      	ldr	r3, [r7, #44]	; 0x2c
 800221e:	4413      	add	r3, r2
 8002220:	7818      	ldrb	r0, [r3, #0]
 8002222:	687a      	ldr	r2, [r7, #4]
 8002224:	1c53      	adds	r3, r2, #1
 8002226:	607b      	str	r3, [r7, #4]
 8002228:	68fc      	ldr	r4, [r7, #12]
 800222a:	683b      	ldr	r3, [r7, #0]
 800222c:	68b9      	ldr	r1, [r7, #8]
 800222e:	47a0      	blx	r4
  while (len) {
 8002230:	6afb      	ldr	r3, [r7, #44]	; 0x2c
 8002232:	2b00      	cmp	r3, #0
 8002234:	d1ee      	bne.n	8002214 <_out_rev+0x4c>
  }

  // append pad spaces up to given width
  if (flags & FLAGS_LEFT) {
 8002236:	6b7b      	ldr	r3, [r7, #52]	; 0x34
 8002238:	f003 0302 	and.w	r3, r3, #2
 800223c:	2b00      	cmp	r3, #0
 800223e:	d00e      	beq.n	800225e <_out_rev+0x96>
    while (idx - start_idx < width) {
 8002240:	e007      	b.n	8002252 <_out_rev+0x8a>
      out(' ', buffer, idx++, maxlen);
 8002242:	687a      	ldr	r2, [r7, #4]
 8002244:	1c53      	adds	r3, r2, #1
 8002246:	607b      	str	r3, [r7, #4]
 8002248:	68fc      	ldr	r4, [r7, #12]
 800224a:	683b      	ldr	r3, [r7, #0]
 800224c:	68b9      	ldr	r1, [r7, #8]
 800224e:	2020      	movs	r0, #32
 8002250:	47a0      	blx	r4
    while (idx - start_idx < width) {
 8002252:	687a      	ldr	r2, [r7, #4]
 8002254:	693b      	ldr	r3, [r7, #16]
 8002256:	1ad3      	subs	r3, r2, r3
 8002258:	6b3a      	ldr	r2, [r7, #48]	; 0x30
 800225a:	429a      	cmp	r2, r3
 800225c:	d8f1      	bhi.n	8002242 <_out_rev+0x7a>
    }
  }

  return idx;
 800225e:	687b      	ldr	r3, [r7, #4]
}
 8002260:	4618      	mov	r0, r3
 8002262:	371c      	adds	r7, #28
 8002264:	46bd      	mov	sp, r7
 8002266:	bd90      	pop	{r4, r7, pc}

08002268 <_ntoa_format>:


// internal itoa format
static size_t _ntoa_format(out_fct_type out, char* buffer, size_t idx, size_t maxlen, char* buf, size_t len, bool negative, unsigned int base, unsigned int prec, unsigned int width, unsigned int flags)
{
 8002268:	b580      	push	{r7, lr}
 800226a:	b088      	sub	sp, #32
 800226c:	af04      	add	r7, sp, #16
 800226e:	60f8      	str	r0, [r7, #12]
 8002270:	60b9      	str	r1, [r7, #8]
 8002272:	607a      	str	r2, [r7, #4]
 8002274:	603b      	str	r3, [r7, #0]
  // pad leading zeros
  if (!(flags & FLAGS_LEFT)) {
 8002276:	6b3b      	ldr	r3, [r7, #48]	; 0x30
 8002278:	f003 0302 	and.w	r3, r3, #2
 800227c:	2b00      	cmp	r3, #0
 800227e:	d136      	bne.n	80022ee <_ntoa_format+0x86>
    if (width && (flags & FLAGS_ZEROPAD) && (negative || (flags & (FLAGS_PLUS | FLAGS_SPACE)))) {
 8002280:	6afb      	ldr	r3, [r7, #44]	; 0x2c
 8002282:	2b00      	cmp	r3, #0
 8002284:	d018      	beq.n	80022b8 <_ntoa_format+0x50>
 8002286:	6b3b      	ldr	r3, [r7, #48]	; 0x30
 8002288:	f003 0301 	and.w	r3, r3, #1
 800228c:	2b00      	cmp	r3, #0
 800228e:	d013      	beq.n	80022b8 <_ntoa_format+0x50>
 8002290:	f897 3020 	ldrb.w	r3, [r7, #32]
 8002294:	2b00      	cmp	r3, #0
 8002296:	d104      	bne.n	80022a2 <_ntoa_format+0x3a>
 8002298:	6b3b      	ldr	r3, [r7, #48]	; 0x30
 800229a:	f003 030c 	and.w	r3, r3, #12
 800229e:	2b00      	cmp	r3, #0
 80022a0:	d00a      	beq.n	80022b8 <_ntoa_format+0x50>
      width--;
 80022a2:	6afb      	ldr	r3, [r7, #44]	; 0x2c
 80022a4:	3b01      	subs	r3, #1
 80022a6:	62fb      	str	r3, [r7, #44]	; 0x2c
    }
    while ((len < prec) && (len < PRINTF_NTOA_BUFFER_SIZE)) {
 80022a8:	e006      	b.n	80022b8 <_ntoa_format+0x50>
      buf[len++] = '0';
 80022aa:	69fb      	ldr	r3, [r7, #28]
 80022ac:	1c5a      	adds	r2, r3, #1
 80022ae:	61fa      	str	r2, [r7, #28]
 80022b0:	69ba      	ldr	r2, [r7, #24]
 80022b2:	4413      	add	r3, r2
 80022b4:	2230      	movs	r2, #48	; 0x30
 80022b6:	701a      	strb	r2, [r3, #0]
    while ((len < prec) && (len < PRINTF_NTOA_BUFFER_SIZE)) {
 80022b8:	69fa      	ldr	r2, [r7, #28]
 80022ba:	6abb      	ldr	r3, [r7, #40]	; 0x28
 80022bc:	429a      	cmp	r2, r3
 80022be:	d20a      	bcs.n	80022d6 <_ntoa_format+0x6e>
 80022c0:	69fb      	ldr	r3, [r7, #28]
 80022c2:	2b1f      	cmp	r3, #31
 80022c4:	d9f1      	bls.n	80022aa <_ntoa_format+0x42>
    }
    while ((flags & FLAGS_ZEROPAD) && (len < width) && (len < PRINTF_NTOA_BUFFER_SIZE)) {
 80022c6:	e006      	b.n	80022d6 <_ntoa_format+0x6e>
      buf[len++] = '0';
 80022c8:	69fb      	ldr	r3, [r7, #28]
 80022ca:	1c5a      	adds	r2, r3, #1
 80022cc:	61fa      	str	r2, [r7, #28]
 80022ce:	69ba      	ldr	r2, [r7, #24]
 80022d0:	4413      	add	r3, r2
 80022d2:	2230      	movs	r2, #48	; 0x30
 80022d4:	701a      	strb	r2, [r3, #0]
    while ((flags & FLAGS_ZEROPAD) && (len < width) && (len < PRINTF_NTOA_BUFFER_SIZE)) {
 80022d6:	6b3b      	ldr	r3, [r7, #48]	; 0x30
 80022d8:	f003 0301 	and.w	r3, r3, #1
 80022dc:	2b00      	cmp	r3, #0
 80022de:	d006      	beq.n	80022ee <_ntoa_format+0x86>
 80022e0:	69fa      	ldr	r2, [r7, #28]
 80022e2:	6afb      	ldr	r3, [r7, #44]	; 0x2c
 80022e4:	429a      	cmp	r2, r3
 80022e6:	d202      	bcs.n	80022ee <_ntoa_format+0x86>
 80022e8:	69fb      	ldr	r3, [r7, #28]
 80022ea:	2b1f      	cmp	r3, #31
 80022ec:	d9ec      	bls.n	80022c8 <_ntoa_format+0x60>
    }
  }

  // handle hash
  if (flags & FLAGS_HASH) {
 80022ee:	6b3b      	ldr	r3, [r7, #48]	; 0x30
 80022f0:	f003 0310 	and.w	r3, r3, #16
 80022f4:	2b00      	cmp	r3, #0
 80022f6:	d058      	beq.n	80023aa <_ntoa_format+0x142>
    if (!(flags & FLAGS_PRECISION) && len && ((len == prec) || (len == width))) {
 80022f8:	6b3b      	ldr	r3, [r7, #48]	; 0x30
 80022fa:	f403 6380 	and.w	r3, r3, #1024	; 0x400
 80022fe:	2b00      	cmp	r3, #0
 8002300:	d116      	bne.n	8002330 <_ntoa_format+0xc8>
 8002302:	69fb      	ldr	r3, [r7, #28]
 8002304:	2b00      	cmp	r3, #0
 8002306:	d013      	beq.n	8002330 <_ntoa_format+0xc8>
 8002308:	69fa      	ldr	r2, [r7, #28]
 800230a:	6abb      	ldr	r3, [r7, #40]	; 0x28
 800230c:	429a      	cmp	r2, r3
 800230e:	d003      	beq.n	8002318 <_ntoa_format+0xb0>
 8002310:	69fa      	ldr	r2, [r7, #28]
 8002312:	6afb      	ldr	r3, [r7, #44]	; 0x2c
 8002314:	429a      	cmp	r2, r3
 8002316:	d10b      	bne.n	8002330 <_ntoa_format+0xc8>
      len--;
 8002318:	69fb      	ldr	r3, [r7, #28]
 800231a:	3b01      	subs	r3, #1
 800231c:	61fb      	str	r3, [r7, #28]
      if (len && (base == 16U)) {
 800231e:	69fb      	ldr	r3, [r7, #28]
 8002320:	2b00      	cmp	r3, #0
 8002322:	d005      	beq.n	8002330 <_ntoa_format+0xc8>
 8002324:	6a7b      	ldr	r3, [r7, #36]	; 0x24
 8002326:	2b10      	cmp	r3, #16
 8002328:	d102      	bne.n	8002330 <_ntoa_format+0xc8>
        len--;
 800232a:	69fb      	ldr	r3, [r7, #28]
 800232c:	3b01      	subs	r3, #1
 800232e:	61fb      	str	r3, [r7, #28]
      }
    }
    if ((base == 16U) && !(flags & FLAGS_UPPERCASE) && (len < PRINTF_NTOA_BUFFER_SIZE)) {
 8002330:	6a7b      	ldr	r3, [r7, #36]	; 0x24
 8002332:	2b10      	cmp	r3, #16
 8002334:	d10f      	bne.n	8002356 <_ntoa_format+0xee>
 8002336:	6b3b      	ldr	r3, [r7, #48]	; 0x30
 8002338:	f003 0320 	and.w	r3, r3, #32
 800233c:	2b00      	cmp	r3, #0
 800233e:	d10a      	bne.n	8002356 <_ntoa_format+0xee>
 8002340:	69fb      	ldr	r3, [r7, #28]
 8002342:	2b1f      	cmp	r3, #31
 8002344:	d807      	bhi.n	8002356 <_ntoa_format+0xee>
      buf[len++] = 'x';
 8002346:	69fb      	ldr	r3, [r7, #28]
 8002348:	1c5a      	adds	r2, r3, #1
 800234a:	61fa      	str	r2, [r7, #28]
 800234c:	69ba      	ldr	r2, [r7, #24]
 800234e:	4413      	add	r3, r2
 8002350:	2278      	movs	r2, #120	; 0x78
 8002352:	701a      	strb	r2, [r3, #0]
 8002354:	e01f      	b.n	8002396 <_ntoa_format+0x12e>
    }
    else if ((base == 16U) && (flags & FLAGS_UPPERCASE) && (len < PRINTF_NTOA_BUFFER_SIZE)) {
 8002356:	6a7b      	ldr	r3, [r7, #36]	; 0x24
 8002358:	2b10      	cmp	r3, #16
 800235a:	d10f      	bne.n	800237c <_ntoa_format+0x114>
 800235c:	6b3b      	ldr	r3, [r7, #48]	; 0x30
 800235e:	f003 0320 	and.w	r3, r3, #32
 8002362:	2b00      	cmp	r3, #0
 8002364:	d00a      	beq.n	800237c <_ntoa_format+0x114>
 8002366:	69fb      	ldr	r3, [r7, #28]
 8002368:	2b1f      	cmp	r3, #31
 800236a:	d807      	bhi.n	800237c <_ntoa_format+0x114>
      buf[len++] = 'X';
 800236c:	69fb      	ldr	r3, [r7, #28]
 800236e:	1c5a      	adds	r2, r3, #1
 8002370:	61fa      	str	r2, [r7, #28]
 8002372:	69ba      	ldr	r2, [r7, #24]
 8002374:	4413      	add	r3, r2
 8002376:	2258      	movs	r2, #88	; 0x58
 8002378:	701a      	strb	r2, [r3, #0]
 800237a:	e00c      	b.n	8002396 <_ntoa_format+0x12e>
    }
    else if ((base == 2U) && (len < PRINTF_NTOA_BUFFER_SIZE)) {
 800237c:	6a7b      	ldr	r3, [r7, #36]	; 0x24
 800237e:	2b02      	cmp	r3, #2
 8002380:	d109      	bne.n	8002396 <_ntoa_format+0x12e>
 8002382:	69fb      	ldr	r3, [r7, #28]
 8002384:	2b1f      	cmp	r3, #31
 8002386:	d806      	bhi.n	8002396 <_ntoa_format+0x12e>
      buf[len++] = 'b';
 8002388:	69fb      	ldr	r3, [r7, #28]
 800238a:	1c5a      	adds	r2, r3, #1
 800238c:	61fa      	str	r2, [r7, #28]
 800238e:	69ba      	ldr	r2, [r7, #24]
 8002390:	4413      	add	r3, r2
 8002392:	2262      	movs	r2, #98	; 0x62
 8002394:	701a      	strb	r2, [r3, #0]
    }
    if (len < PRINTF_NTOA_BUFFER_SIZE) {
 8002396:	69fb      	ldr	r3, [r7, #28]
 8002398:	2b1f      	cmp	r3, #31
 800239a:	d806      	bhi.n	80023aa <_ntoa_format+0x142>
      buf[len++] = '0';
 800239c:	69fb      	ldr	r3, [r7, #28]
 800239e:	1c5a      	adds	r2, r3, #1
 80023a0:	61fa      	str	r2, [r7, #28]
 80023a2:	69ba      	ldr	r2, [r7, #24]
 80023a4:	4413      	add	r3, r2
 80023a6:	2230      	movs	r2, #48	; 0x30
 80023a8:	701a      	strb	r2, [r3, #0]
    }
  }

  if (len < PRINTF_NTOA_BUFFER_SIZE) {
 80023aa:	69fb      	ldr	r3, [r7, #28]
 80023ac:	2b1f      	cmp	r3, #31
 80023ae:	d824      	bhi.n	80023fa <_ntoa_format+0x192>
    if (negative) {
 80023b0:	f897 3020 	ldrb.w	r3, [r7, #32]
 80023b4:	2b00      	cmp	r3, #0
 80023b6:	d007      	beq.n	80023c8 <_ntoa_format+0x160>
      buf[len++] = '-';
 80023b8:	69fb      	ldr	r3, [r7, #28]
 80023ba:	1c5a      	adds	r2, r3, #1
 80023bc:	61fa      	str	r2, [r7, #28]
 80023be:	69ba      	ldr	r2, [r7, #24]
 80023c0:	4413      	add	r3, r2
 80023c2:	222d      	movs	r2, #45	; 0x2d
 80023c4:	701a      	strb	r2, [r3, #0]
 80023c6:	e018      	b.n	80023fa <_ntoa_format+0x192>
    }
    else if (flags & FLAGS_PLUS) {
 80023c8:	6b3b      	ldr	r3, [r7, #48]	; 0x30
 80023ca:	f003 0304 	and.w	r3, r3, #4
 80023ce:	2b00      	cmp	r3, #0
 80023d0:	d007      	beq.n	80023e2 <_ntoa_format+0x17a>
      buf[len++] = '+';  // ignore the space if the '+' exists
 80023d2:	69fb      	ldr	r3, [r7, #28]
 80023d4:	1c5a      	adds	r2, r3, #1
 80023d6:	61fa      	str	r2, [r7, #28]
 80023d8:	69ba      	ldr	r2, [r7, #24]
 80023da:	4413      	add	r3, r2
 80023dc:	222b      	movs	r2, #43	; 0x2b
 80023de:	701a      	strb	r2, [r3, #0]
 80023e0:	e00b      	b.n	80023fa <_ntoa_format+0x192>
    }
    else if (flags & FLAGS_SPACE) {
 80023e2:	6b3b      	ldr	r3, [r7, #48]	; 0x30
 80023e4:	f003 0308 	and.w	r3, r3, #8
 80023e8:	2b00      	cmp	r3, #0
 80023ea:	d006      	beq.n	80023fa <_ntoa_format+0x192>
      buf[len++] = ' ';
 80023ec:	69fb      	ldr	r3, [r7, #28]
 80023ee:	1c5a      	adds	r2, r3, #1
 80023f0:	61fa      	str	r2, [r7, #28]
 80023f2:	69ba      	ldr	r2, [r7, #24]
 80023f4:	4413      	add	r3, r2
 80023f6:	2220      	movs	r2, #32
 80023f8:	701a      	strb	r2, [r3, #0]
    }
  }

  return _out_rev(out, buffer, idx, maxlen, buf, len, width, flags);
 80023fa:	6b3b      	ldr	r3, [r7, #48]	; 0x30
 80023fc:	9303      	str	r3, [sp, #12]
 80023fe:	6afb      	ldr	r3, [r7, #44]	; 0x2c
 8002400:	9302      	str	r3, [sp, #8]
 8002402:	69fb      	ldr	r3, [r7, #28]
 8002404:	9301      	str	r3, [sp, #4]
 8002406:	69bb      	ldr	r3, [r7, #24]
 8002408:	9300      	str	r3, [sp, #0]
 800240a:	683b      	ldr	r3, [r7, #0]
 800240c:	687a      	ldr	r2, [r7, #4]
 800240e:	68b9      	ldr	r1, [r7, #8]
 8002410:	68f8      	ldr	r0, [r7, #12]
 8002412:	f7ff fed9 	bl	80021c8 <_out_rev>
 8002416:	4603      	mov	r3, r0
}
 8002418:	4618      	mov	r0, r3
 800241a:	3710      	adds	r7, #16
 800241c:	46bd      	mov	sp, r7
 800241e:	bd80      	pop	{r7, pc}

08002420 <_ntoa_long>:


// internal itoa for 'long' type
static size_t _ntoa_long(out_fct_type out, char* buffer, size_t idx, size_t maxlen, unsigned long value, bool negative, unsigned long base, unsigned int prec, unsigned int width, unsigned int flags)
{
 8002420:	b580      	push	{r7, lr}
 8002422:	b096      	sub	sp, #88	; 0x58
 8002424:	af08      	add	r7, sp, #32
 8002426:	60f8      	str	r0, [r7, #12]
 8002428:	60b9      	str	r1, [r7, #8]
 800242a:	607a      	str	r2, [r7, #4]
 800242c:	603b      	str	r3, [r7, #0]
  char buf[PRINTF_NTOA_BUFFER_SIZE];
  size_t len = 0U;
 800242e:	2300      	movs	r3, #0
 8002430:	637b      	str	r3, [r7, #52]	; 0x34

  // no hash for 0 values
  if (!value) {
 8002432:	6c3b      	ldr	r3, [r7, #64]	; 0x40
 8002434:	2b00      	cmp	r3, #0
 8002436:	d103      	bne.n	8002440 <_ntoa_long+0x20>
    flags &= ~FLAGS_HASH;
 8002438:	6d7b      	ldr	r3, [r7, #84]	; 0x54
 800243a:	f023 0310 	bic.w	r3, r3, #16
 800243e:	657b      	str	r3, [r7, #84]	; 0x54
  }

  // write if precision != 0 and value is != 0
  if (!(flags & FLAGS_PRECISION) || value) {
 8002440:	6d7b      	ldr	r3, [r7, #84]	; 0x54
 8002442:	f403 6380 	and.w	r3, r3, #1024	; 0x400
 8002446:	2b00      	cmp	r3, #0
 8002448:	d002      	beq.n	8002450 <_ntoa_long+0x30>
 800244a:	6c3b      	ldr	r3, [r7, #64]	; 0x40
 800244c:	2b00      	cmp	r3, #0
 800244e:	d033      	beq.n	80024b8 <_ntoa_long+0x98>
    do {
      const char digit = (char)(value % base);
 8002450:	6c3b      	ldr	r3, [r7, #64]	; 0x40
 8002452:	6cba      	ldr	r2, [r7, #72]	; 0x48
 8002454:	fbb3 f2f2 	udiv	r2, r3, r2
 8002458:	6cb9      	ldr	r1, [r7, #72]	; 0x48
 800245a:	fb01 f202 	mul.w	r2, r1, r2
 800245e:	1a9b      	subs	r3, r3, r2
 8002460:	f887 3033 	strb.w	r3, [r7, #51]	; 0x33
      buf[len++] = digit < 10 ? '0' + digit : (flags & FLAGS_UPPERCASE ? 'A' : 'a') + digit - 10;
 8002464:	f897 3033 	ldrb.w	r3, [r7, #51]	; 0x33
 8002468:	2b09      	cmp	r3, #9
 800246a:	d804      	bhi.n	8002476 <_ntoa_long+0x56>
 800246c:	f897 3033 	ldrb.w	r3, [r7, #51]	; 0x33
 8002470:	3330      	adds	r3, #48	; 0x30
 8002472:	b2da      	uxtb	r2, r3
 8002474:	e00d      	b.n	8002492 <_ntoa_long+0x72>
 8002476:	6d7b      	ldr	r3, [r7, #84]	; 0x54
 8002478:	f003 0320 	and.w	r3, r3, #32
 800247c:	2b00      	cmp	r3, #0
 800247e:	d001      	beq.n	8002484 <_ntoa_long+0x64>
 8002480:	2241      	movs	r2, #65	; 0x41
 8002482:	e000      	b.n	8002486 <_ntoa_long+0x66>
 8002484:	2261      	movs	r2, #97	; 0x61
 8002486:	f897 3033 	ldrb.w	r3, [r7, #51]	; 0x33
 800248a:	4413      	add	r3, r2
 800248c:	b2db      	uxtb	r3, r3
 800248e:	3b0a      	subs	r3, #10
 8002490:	b2da      	uxtb	r2, r3
 8002492:	6b7b      	ldr	r3, [r7, #52]	; 0x34
 8002494:	1c59      	adds	r1, r3, #1
 8002496:	6379      	str	r1, [r7, #52]	; 0x34
 8002498:	f107 0138 	add.w	r1, r7, #56	; 0x38
 800249c:	440b      	add	r3, r1
 800249e:	f803 2c28 	strb.w	r2, [r3, #-40]
      value /= base;
 80024a2:	6c3a      	ldr	r2, [r7, #64]	; 0x40
 80024a4:	6cbb      	ldr	r3, [r7, #72]	; 0x48
 80024a6:	fbb2 f3f3 	udiv	r3, r2, r3
 80024aa:	643b      	str	r3, [r7, #64]	; 0x40
    } while (value && (len < PRINTF_NTOA_BUFFER_SIZE));
 80024ac:	6c3b      	ldr	r3, [r7, #64]	; 0x40
 80024ae:	2b00      	cmp	r3, #0
 80024b0:	d002      	beq.n	80024b8 <_ntoa_long+0x98>
 80024b2:	6b7b      	ldr	r3, [r7, #52]	; 0x34
 80024b4:	2b1f      	cmp	r3, #31
 80024b6:	d9cb      	bls.n	8002450 <_ntoa_long+0x30>
  }

  return _ntoa_format(out, buffer, idx, maxlen, buf, len, negative, (unsigned int)base, prec, width, flags);
 80024b8:	6d7b      	ldr	r3, [r7, #84]	; 0x54
 80024ba:	9306      	str	r3, [sp, #24]
 80024bc:	6d3b      	ldr	r3, [r7, #80]	; 0x50
 80024be:	9305      	str	r3, [sp, #20]
 80024c0:	6cfb      	ldr	r3, [r7, #76]	; 0x4c
 80024c2:	9304      	str	r3, [sp, #16]
 80024c4:	6cbb      	ldr	r3, [r7, #72]	; 0x48
 80024c6:	9303      	str	r3, [sp, #12]
 80024c8:	f897 3044 	ldrb.w	r3, [r7, #68]	; 0x44
 80024cc:	9302      	str	r3, [sp, #8]
 80024ce:	6b7b      	ldr	r3, [r7, #52]	; 0x34
 80024d0:	9301      	str	r3, [sp, #4]
 80024d2:	f107 0310 	add.w	r3, r7, #16
 80024d6:	9300      	str	r3, [sp, #0]
 80024d8:	683b      	ldr	r3, [r7, #0]
 80024da:	687a      	ldr	r2, [r7, #4]
 80024dc:	68b9      	ldr	r1, [r7, #8]
 80024de:	68f8      	ldr	r0, [r7, #12]
 80024e0:	f7ff fec2 	bl	8002268 <_ntoa_format>
 80024e4:	4603      	mov	r3, r0
}
 80024e6:	4618      	mov	r0, r3
 80024e8:	3738      	adds	r7, #56	; 0x38
 80024ea:	46bd      	mov	sp, r7
 80024ec:	bd80      	pop	{r7, pc}

080024ee <_ntoa_long_long>:


// internal itoa for 'long long' type
#if defined(PRINTF_SUPPORT_LONG_LONG)
static size_t _ntoa_long_long(out_fct_type out, char* buffer, size_t idx, size_t maxlen, unsigned long long value, bool negative, unsigned long long base, unsigned int prec, unsigned int width, unsigned int flags)
{
 80024ee:	b590      	push	{r4, r7, lr}
 80024f0:	b097      	sub	sp, #92	; 0x5c
 80024f2:	af08      	add	r7, sp, #32
 80024f4:	60f8      	str	r0, [r7, #12]
 80024f6:	60b9      	str	r1, [r7, #8]
 80024f8:	607a      	str	r2, [r7, #4]
 80024fa:	603b      	str	r3, [r7, #0]
  char buf[PRINTF_NTOA_BUFFER_SIZE];
  size_t len = 0U;
 80024fc:	2300      	movs	r3, #0
 80024fe:	637b      	str	r3, [r7, #52]	; 0x34

  // no hash for 0 values
  if (!value) {
 8002500:	e9d7 3412 	ldrd	r3, r4, [r7, #72]	; 0x48
 8002504:	4323      	orrs	r3, r4
 8002506:	d103      	bne.n	8002510 <_ntoa_long_long+0x22>
    flags &= ~FLAGS_HASH;
 8002508:	6ebb      	ldr	r3, [r7, #104]	; 0x68
 800250a:	f023 0310 	bic.w	r3, r3, #16
 800250e:	66bb      	str	r3, [r7, #104]	; 0x68
  }

  // write if precision != 0 and value is != 0
  if (!(flags & FLAGS_PRECISION) || value) {
 8002510:	6ebb      	ldr	r3, [r7, #104]	; 0x68
 8002512:	f403 6380 	and.w	r3, r3, #1024	; 0x400
 8002516:	2b00      	cmp	r3, #0
 8002518:	d003      	beq.n	8002522 <_ntoa_long_long+0x34>
 800251a:	e9d7 3412 	ldrd	r3, r4, [r7, #72]	; 0x48
 800251e:	4323      	orrs	r3, r4
 8002520:	d039      	beq.n	8002596 <_ntoa_long_long+0xa8>
    do {
      const char digit = (char)(value % base);
 8002522:	e9d7 0112 	ldrd	r0, r1, [r7, #72]	; 0x48
 8002526:	e9d7 2316 	ldrd	r2, r3, [r7, #88]	; 0x58
 800252a:	f7fe fb47 	bl	8000bbc <__aeabi_uldivmod>
 800252e:	461c      	mov	r4, r3
 8002530:	4613      	mov	r3, r2
 8002532:	f887 3033 	strb.w	r3, [r7, #51]	; 0x33
      buf[len++] = digit < 10 ? '0' + digit : (flags & FLAGS_UPPERCASE ? 'A' : 'a') + digit - 10;
 8002536:	f897 3033 	ldrb.w	r3, [r7, #51]	; 0x33
 800253a:	2b09      	cmp	r3, #9
 800253c:	d804      	bhi.n	8002548 <_ntoa_long_long+0x5a>
 800253e:	f897 3033 	ldrb.w	r3, [r7, #51]	; 0x33
 8002542:	3330      	adds	r3, #48	; 0x30
 8002544:	b2da      	uxtb	r2, r3
 8002546:	e00d      	b.n	8002564 <_ntoa_long_long+0x76>
 8002548:	6ebb      	ldr	r3, [r7, #104]	; 0x68
 800254a:	f003 0320 	and.w	r3, r3, #32
 800254e:	2b00      	cmp	r3, #0
 8002550:	d001      	beq.n	8002556 <_ntoa_long_long+0x68>
 8002552:	2241      	movs	r2, #65	; 0x41
 8002554:	e000      	b.n	8002558 <_ntoa_long_long+0x6a>
 8002556:	2261      	movs	r2, #97	; 0x61
 8002558:	f897 3033 	ldrb.w	r3, [r7, #51]	; 0x33
 800255c:	4413      	add	r3, r2
 800255e:	b2db      	uxtb	r3, r3
 8002560:	3b0a      	subs	r3, #10
 8002562:	b2da      	uxtb	r2, r3
 8002564:	6b7b      	ldr	r3, [r7, #52]	; 0x34
 8002566:	1c59      	adds	r1, r3, #1
 8002568:	6379      	str	r1, [r7, #52]	; 0x34
 800256a:	f107 0138 	add.w	r1, r7, #56	; 0x38
 800256e:	440b      	add	r3, r1
 8002570:	f803 2c28 	strb.w	r2, [r3, #-40]
      value /= base;
 8002574:	e9d7 2316 	ldrd	r2, r3, [r7, #88]	; 0x58
 8002578:	e9d7 0112 	ldrd	r0, r1, [r7, #72]	; 0x48
 800257c:	f7fe fb1e 	bl	8000bbc <__aeabi_uldivmod>
 8002580:	4603      	mov	r3, r0
 8002582:	460c      	mov	r4, r1
 8002584:	e9c7 3412 	strd	r3, r4, [r7, #72]	; 0x48
    } while (value && (len < PRINTF_NTOA_BUFFER_SIZE));
 8002588:	e9d7 3412 	ldrd	r3, r4, [r7, #72]	; 0x48
 800258c:	4323      	orrs	r3, r4
 800258e:	d002      	beq.n	8002596 <_ntoa_long_long+0xa8>
 8002590:	6b7b      	ldr	r3, [r7, #52]	; 0x34
 8002592:	2b1f      	cmp	r3, #31
 8002594:	d9c5      	bls.n	8002522 <_ntoa_long_long+0x34>
  }

  return _ntoa_format(out, buffer, idx, maxlen, buf, len, negative, (unsigned int)base, prec, width, flags);
 8002596:	6dbb      	ldr	r3, [r7, #88]	; 0x58
 8002598:	6eba      	ldr	r2, [r7, #104]	; 0x68
 800259a:	9206      	str	r2, [sp, #24]
 800259c:	6e7a      	ldr	r2, [r7, #100]	; 0x64
 800259e:	9205      	str	r2, [sp, #20]
 80025a0:	6e3a      	ldr	r2, [r7, #96]	; 0x60
 80025a2:	9204      	str	r2, [sp, #16]
 80025a4:	9303      	str	r3, [sp, #12]
 80025a6:	f897 3050 	ldrb.w	r3, [r7, #80]	; 0x50
 80025aa:	9302      	str	r3, [sp, #8]
 80025ac:	6b7b      	ldr	r3, [r7, #52]	; 0x34
 80025ae:	9301      	str	r3, [sp, #4]
 80025b0:	f107 0310 	add.w	r3, r7, #16
 80025b4:	9300      	str	r3, [sp, #0]
 80025b6:	683b      	ldr	r3, [r7, #0]
 80025b8:	687a      	ldr	r2, [r7, #4]
 80025ba:	68b9      	ldr	r1, [r7, #8]
 80025bc:	68f8      	ldr	r0, [r7, #12]
 80025be:	f7ff fe53 	bl	8002268 <_ntoa_format>
 80025c2:	4603      	mov	r3, r0
}
 80025c4:	4618      	mov	r0, r3
 80025c6:	373c      	adds	r7, #60	; 0x3c
 80025c8:	46bd      	mov	sp, r7
 80025ca:	bd90      	pop	{r4, r7, pc}
 80025cc:	0000      	movs	r0, r0
	...

080025d0 <_ftoa>:
#endif


// internal ftoa for fixed decimal floating point
static size_t _ftoa(out_fct_type out, char* buffer, size_t idx, size_t maxlen, double value, unsigned int prec, unsigned int width, unsigned int flags)
{
 80025d0:	b590      	push	{r4, r7, lr}
 80025d2:	b09d      	sub	sp, #116	; 0x74
 80025d4:	af04      	add	r7, sp, #16
 80025d6:	6178      	str	r0, [r7, #20]
 80025d8:	6139      	str	r1, [r7, #16]
 80025da:	60fa      	str	r2, [r7, #12]
 80025dc:	60bb      	str	r3, [r7, #8]
 80025de:	ed87 0b00 	vstr	d0, [r7]
  char buf[PRINTF_FTOA_BUFFER_SIZE];
  size_t len  = 0U;
 80025e2:	2300      	movs	r3, #0
 80025e4:	65fb      	str	r3, [r7, #92]	; 0x5c
  double diff = 0.0;
 80025e6:	f04f 0300 	mov.w	r3, #0
 80025ea:	f04f 0400 	mov.w	r4, #0
 80025ee:	e9c7 3410 	strd	r3, r4, [r7, #64]	; 0x40

  // powers of 10
  static const double pow10[] = { 1, 10, 100, 1000, 10000, 100000, 1000000, 10000000, 100000000, 1000000000 };

  // test for special values
  if (value != value)
 80025f2:	e9d7 2300 	ldrd	r2, r3, [r7]
 80025f6:	e9d7 0100 	ldrd	r0, r1, [r7]
 80025fa:	f7fe fa15 	bl	8000a28 <__aeabi_dcmpeq>
 80025fe:	4603      	mov	r3, r0
 8002600:	2b00      	cmp	r3, #0
 8002602:	d10f      	bne.n	8002624 <_ftoa+0x54>
    return _out_rev(out, buffer, idx, maxlen, "nan", 3, width, flags);
 8002604:	6fbb      	ldr	r3, [r7, #120]	; 0x78
 8002606:	9303      	str	r3, [sp, #12]
 8002608:	6f7b      	ldr	r3, [r7, #116]	; 0x74
 800260a:	9302      	str	r3, [sp, #8]
 800260c:	2303      	movs	r3, #3
 800260e:	9301      	str	r3, [sp, #4]
 8002610:	4baf      	ldr	r3, [pc, #700]	; (80028d0 <_ftoa+0x300>)
 8002612:	9300      	str	r3, [sp, #0]
 8002614:	68bb      	ldr	r3, [r7, #8]
 8002616:	68fa      	ldr	r2, [r7, #12]
 8002618:	6939      	ldr	r1, [r7, #16]
 800261a:	6978      	ldr	r0, [r7, #20]
 800261c:	f7ff fdd4 	bl	80021c8 <_out_rev>
 8002620:	4603      	mov	r3, r0
 8002622:	e237      	b.n	8002a94 <_ftoa+0x4c4>
  if (value < -DBL_MAX)
 8002624:	f04f 32ff 	mov.w	r2, #4294967295
 8002628:	f46f 1380 	mvn.w	r3, #1048576	; 0x100000
 800262c:	e9d7 0100 	ldrd	r0, r1, [r7]
 8002630:	f7fe fa04 	bl	8000a3c <__aeabi_dcmplt>
 8002634:	4603      	mov	r3, r0
 8002636:	2b00      	cmp	r3, #0
 8002638:	d00f      	beq.n	800265a <_ftoa+0x8a>
    return _out_rev(out, buffer, idx, maxlen, "fni-", 4, width, flags);
 800263a:	6fbb      	ldr	r3, [r7, #120]	; 0x78
 800263c:	9303      	str	r3, [sp, #12]
 800263e:	6f7b      	ldr	r3, [r7, #116]	; 0x74
 8002640:	9302      	str	r3, [sp, #8]
 8002642:	2304      	movs	r3, #4
 8002644:	9301      	str	r3, [sp, #4]
 8002646:	4ba3      	ldr	r3, [pc, #652]	; (80028d4 <_ftoa+0x304>)
 8002648:	9300      	str	r3, [sp, #0]
 800264a:	68bb      	ldr	r3, [r7, #8]
 800264c:	68fa      	ldr	r2, [r7, #12]
 800264e:	6939      	ldr	r1, [r7, #16]
 8002650:	6978      	ldr	r0, [r7, #20]
 8002652:	f7ff fdb9 	bl	80021c8 <_out_rev>
 8002656:	4603      	mov	r3, r0
 8002658:	e21c      	b.n	8002a94 <_ftoa+0x4c4>
  if (value > DBL_MAX)
 800265a:	f04f 32ff 	mov.w	r2, #4294967295
 800265e:	4b9e      	ldr	r3, [pc, #632]	; (80028d8 <_ftoa+0x308>)
 8002660:	e9d7 0100 	ldrd	r0, r1, [r7]
 8002664:	f7fe fa08 	bl	8000a78 <__aeabi_dcmpgt>
 8002668:	4603      	mov	r3, r0
 800266a:	2b00      	cmp	r3, #0
 800266c:	d01d      	beq.n	80026aa <_ftoa+0xda>
    return _out_rev(out, buffer, idx, maxlen, (flags & FLAGS_PLUS) ? "fni+" : "fni", (flags & FLAGS_PLUS) ? 4U : 3U, width, flags);
 800266e:	6fbb      	ldr	r3, [r7, #120]	; 0x78
 8002670:	f003 0304 	and.w	r3, r3, #4
 8002674:	2b00      	cmp	r3, #0
 8002676:	d001      	beq.n	800267c <_ftoa+0xac>
 8002678:	4b98      	ldr	r3, [pc, #608]	; (80028dc <_ftoa+0x30c>)
 800267a:	e000      	b.n	800267e <_ftoa+0xae>
 800267c:	4b98      	ldr	r3, [pc, #608]	; (80028e0 <_ftoa+0x310>)
 800267e:	6fba      	ldr	r2, [r7, #120]	; 0x78
 8002680:	f002 0204 	and.w	r2, r2, #4
 8002684:	2a00      	cmp	r2, #0
 8002686:	d001      	beq.n	800268c <_ftoa+0xbc>
 8002688:	2204      	movs	r2, #4
 800268a:	e000      	b.n	800268e <_ftoa+0xbe>
 800268c:	2203      	movs	r2, #3
 800268e:	6fb9      	ldr	r1, [r7, #120]	; 0x78
 8002690:	9103      	str	r1, [sp, #12]
 8002692:	6f79      	ldr	r1, [r7, #116]	; 0x74
 8002694:	9102      	str	r1, [sp, #8]
 8002696:	9201      	str	r2, [sp, #4]
 8002698:	9300      	str	r3, [sp, #0]
 800269a:	68bb      	ldr	r3, [r7, #8]
 800269c:	68fa      	ldr	r2, [r7, #12]
 800269e:	6939      	ldr	r1, [r7, #16]
 80026a0:	6978      	ldr	r0, [r7, #20]
 80026a2:	f7ff fd91 	bl	80021c8 <_out_rev>
 80026a6:	4603      	mov	r3, r0
 80026a8:	e1f4      	b.n	8002a94 <_ftoa+0x4c4>

  // test for very large values
  // standard printf behavior is to print EVERY whole number digit -- which could be 100s of characters overflowing your buffers == bad
  if ((value > PRINTF_MAX_FLOAT) || (value < -PRINTF_MAX_FLOAT)) {
 80026aa:	a385      	add	r3, pc, #532	; (adr r3, 80028c0 <_ftoa+0x2f0>)
 80026ac:	e9d3 2300 	ldrd	r2, r3, [r3]
 80026b0:	e9d7 0100 	ldrd	r0, r1, [r7]
 80026b4:	f7fe f9e0 	bl	8000a78 <__aeabi_dcmpgt>
 80026b8:	4603      	mov	r3, r0
 80026ba:	2b00      	cmp	r3, #0
 80026bc:	d109      	bne.n	80026d2 <_ftoa+0x102>
 80026be:	a382      	add	r3, pc, #520	; (adr r3, 80028c8 <_ftoa+0x2f8>)
 80026c0:	e9d3 2300 	ldrd	r2, r3, [r3]
 80026c4:	e9d7 0100 	ldrd	r0, r1, [r7]
 80026c8:	f7fe f9b8 	bl	8000a3c <__aeabi_dcmplt>
 80026cc:	4603      	mov	r3, r0
 80026ce:	2b00      	cmp	r3, #0
 80026d0:	d00f      	beq.n	80026f2 <_ftoa+0x122>
#if defined(PRINTF_SUPPORT_EXPONENTIAL)
    return _etoa(out, buffer, idx, maxlen, value, prec, width, flags);
 80026d2:	6fbb      	ldr	r3, [r7, #120]	; 0x78
 80026d4:	9302      	str	r3, [sp, #8]
 80026d6:	6f7b      	ldr	r3, [r7, #116]	; 0x74
 80026d8:	9301      	str	r3, [sp, #4]
 80026da:	6f3b      	ldr	r3, [r7, #112]	; 0x70
 80026dc:	9300      	str	r3, [sp, #0]
 80026de:	ed97 0b00 	vldr	d0, [r7]
 80026e2:	68bb      	ldr	r3, [r7, #8]
 80026e4:	68fa      	ldr	r2, [r7, #12]
 80026e6:	6939      	ldr	r1, [r7, #16]
 80026e8:	6978      	ldr	r0, [r7, #20]
 80026ea:	f000 f9dd 	bl	8002aa8 <_etoa>
 80026ee:	4603      	mov	r3, r0
 80026f0:	e1d0      	b.n	8002a94 <_ftoa+0x4c4>
    return 0U;
#endif
  }

  // test for negative
  bool negative = false;
 80026f2:	2300      	movs	r3, #0
 80026f4:	f887 305b 	strb.w	r3, [r7, #91]	; 0x5b
  if (value < 0) {
 80026f8:	f04f 0200 	mov.w	r2, #0
 80026fc:	f04f 0300 	mov.w	r3, #0
 8002700:	e9d7 0100 	ldrd	r0, r1, [r7]
 8002704:	f7fe f99a 	bl	8000a3c <__aeabi_dcmplt>
 8002708:	4603      	mov	r3, r0
 800270a:	2b00      	cmp	r3, #0
 800270c:	d00e      	beq.n	800272c <_ftoa+0x15c>
    negative = true;
 800270e:	2301      	movs	r3, #1
 8002710:	f887 305b 	strb.w	r3, [r7, #91]	; 0x5b
    value = 0 - value;
 8002714:	e9d7 2300 	ldrd	r2, r3, [r7]
 8002718:	f04f 0000 	mov.w	r0, #0
 800271c:	f04f 0100 	mov.w	r1, #0
 8002720:	f7fd fd62 	bl	80001e8 <__aeabi_dsub>
 8002724:	4603      	mov	r3, r0
 8002726:	460c      	mov	r4, r1
 8002728:	e9c7 3400 	strd	r3, r4, [r7]
  }

  // set default precision, if not set explicitly
  if (!(flags & FLAGS_PRECISION)) {
 800272c:	6fbb      	ldr	r3, [r7, #120]	; 0x78
 800272e:	f403 6380 	and.w	r3, r3, #1024	; 0x400
 8002732:	2b00      	cmp	r3, #0
 8002734:	d10e      	bne.n	8002754 <_ftoa+0x184>
    prec = PRINTF_DEFAULT_FLOAT_PRECISION;
 8002736:	2306      	movs	r3, #6
 8002738:	673b      	str	r3, [r7, #112]	; 0x70
  }
  // limit precision to 9, cause a prec >= 10 can lead to overflow errors
  while ((len < PRINTF_FTOA_BUFFER_SIZE) && (prec > 9U)) {
 800273a:	e00b      	b.n	8002754 <_ftoa+0x184>
    buf[len++] = '0';
 800273c:	6dfb      	ldr	r3, [r7, #92]	; 0x5c
 800273e:	1c5a      	adds	r2, r3, #1
 8002740:	65fa      	str	r2, [r7, #92]	; 0x5c
 8002742:	f107 0260 	add.w	r2, r7, #96	; 0x60
 8002746:	4413      	add	r3, r2
 8002748:	2230      	movs	r2, #48	; 0x30
 800274a:	f803 2c48 	strb.w	r2, [r3, #-72]
    prec--;
 800274e:	6f3b      	ldr	r3, [r7, #112]	; 0x70
 8002750:	3b01      	subs	r3, #1
 8002752:	673b      	str	r3, [r7, #112]	; 0x70
  while ((len < PRINTF_FTOA_BUFFER_SIZE) && (prec > 9U)) {
 8002754:	6dfb      	ldr	r3, [r7, #92]	; 0x5c
 8002756:	2b1f      	cmp	r3, #31
 8002758:	d802      	bhi.n	8002760 <_ftoa+0x190>
 800275a:	6f3b      	ldr	r3, [r7, #112]	; 0x70
 800275c:	2b09      	cmp	r3, #9
 800275e:	d8ed      	bhi.n	800273c <_ftoa+0x16c>
  }

  int whole = (int)value;
 8002760:	e9d7 0100 	ldrd	r0, r1, [r7]
 8002764:	f7fe f992 	bl	8000a8c <__aeabi_d2iz>
 8002768:	4603      	mov	r3, r0
 800276a:	657b      	str	r3, [r7, #84]	; 0x54
  double tmp = (value - whole) * pow10[prec];
 800276c:	6d78      	ldr	r0, [r7, #84]	; 0x54
 800276e:	f7fd fe89 	bl	8000484 <__aeabi_i2d>
 8002772:	4603      	mov	r3, r0
 8002774:	460c      	mov	r4, r1
 8002776:	461a      	mov	r2, r3
 8002778:	4623      	mov	r3, r4
 800277a:	e9d7 0100 	ldrd	r0, r1, [r7]
 800277e:	f7fd fd33 	bl	80001e8 <__aeabi_dsub>
 8002782:	4603      	mov	r3, r0
 8002784:	460c      	mov	r4, r1
 8002786:	4618      	mov	r0, r3
 8002788:	4621      	mov	r1, r4
 800278a:	4a56      	ldr	r2, [pc, #344]	; (80028e4 <_ftoa+0x314>)
 800278c:	6f3b      	ldr	r3, [r7, #112]	; 0x70
 800278e:	00db      	lsls	r3, r3, #3
 8002790:	4413      	add	r3, r2
 8002792:	e9d3 3400 	ldrd	r3, r4, [r3]
 8002796:	461a      	mov	r2, r3
 8002798:	4623      	mov	r3, r4
 800279a:	f7fd fedd 	bl	8000558 <__aeabi_dmul>
 800279e:	4603      	mov	r3, r0
 80027a0:	460c      	mov	r4, r1
 80027a2:	e9c7 340e 	strd	r3, r4, [r7, #56]	; 0x38
  unsigned long frac = (unsigned long)tmp;
 80027a6:	e9d7 010e 	ldrd	r0, r1, [r7, #56]	; 0x38
 80027aa:	f7fe f997 	bl	8000adc <__aeabi_d2uiz>
 80027ae:	4603      	mov	r3, r0
 80027b0:	653b      	str	r3, [r7, #80]	; 0x50
  diff = tmp - frac;
 80027b2:	6d38      	ldr	r0, [r7, #80]	; 0x50
 80027b4:	f7fd fe56 	bl	8000464 <__aeabi_ui2d>
 80027b8:	4603      	mov	r3, r0
 80027ba:	460c      	mov	r4, r1
 80027bc:	461a      	mov	r2, r3
 80027be:	4623      	mov	r3, r4
 80027c0:	e9d7 010e 	ldrd	r0, r1, [r7, #56]	; 0x38
 80027c4:	f7fd fd10 	bl	80001e8 <__aeabi_dsub>
 80027c8:	4603      	mov	r3, r0
 80027ca:	460c      	mov	r4, r1
 80027cc:	e9c7 3410 	strd	r3, r4, [r7, #64]	; 0x40

  if (diff > 0.5) {
 80027d0:	f04f 0200 	mov.w	r2, #0
 80027d4:	4b44      	ldr	r3, [pc, #272]	; (80028e8 <_ftoa+0x318>)
 80027d6:	e9d7 0110 	ldrd	r0, r1, [r7, #64]	; 0x40
 80027da:	f7fe f94d 	bl	8000a78 <__aeabi_dcmpgt>
 80027de:	4603      	mov	r3, r0
 80027e0:	2b00      	cmp	r3, #0
 80027e2:	d018      	beq.n	8002816 <_ftoa+0x246>
    ++frac;
 80027e4:	6d3b      	ldr	r3, [r7, #80]	; 0x50
 80027e6:	3301      	adds	r3, #1
 80027e8:	653b      	str	r3, [r7, #80]	; 0x50
    // handle rollover, e.g. case 0.99 with prec 1 is 1.0
    if (frac >= pow10[prec]) {
 80027ea:	6d38      	ldr	r0, [r7, #80]	; 0x50
 80027ec:	f7fd fe3a 	bl	8000464 <__aeabi_ui2d>
 80027f0:	4a3c      	ldr	r2, [pc, #240]	; (80028e4 <_ftoa+0x314>)
 80027f2:	6f3b      	ldr	r3, [r7, #112]	; 0x70
 80027f4:	00db      	lsls	r3, r3, #3
 80027f6:	4413      	add	r3, r2
 80027f8:	e9d3 3400 	ldrd	r3, r4, [r3]
 80027fc:	461a      	mov	r2, r3
 80027fe:	4623      	mov	r3, r4
 8002800:	f7fe f930 	bl	8000a64 <__aeabi_dcmpge>
 8002804:	4603      	mov	r3, r0
 8002806:	2b00      	cmp	r3, #0
 8002808:	d01a      	beq.n	8002840 <_ftoa+0x270>
      frac = 0;
 800280a:	2300      	movs	r3, #0
 800280c:	653b      	str	r3, [r7, #80]	; 0x50
      ++whole;
 800280e:	6d7b      	ldr	r3, [r7, #84]	; 0x54
 8002810:	3301      	adds	r3, #1
 8002812:	657b      	str	r3, [r7, #84]	; 0x54
 8002814:	e014      	b.n	8002840 <_ftoa+0x270>
    }
  }
  else if (diff < 0.5) {
 8002816:	f04f 0200 	mov.w	r2, #0
 800281a:	4b33      	ldr	r3, [pc, #204]	; (80028e8 <_ftoa+0x318>)
 800281c:	e9d7 0110 	ldrd	r0, r1, [r7, #64]	; 0x40
 8002820:	f7fe f90c 	bl	8000a3c <__aeabi_dcmplt>
 8002824:	4603      	mov	r3, r0
 8002826:	2b00      	cmp	r3, #0
 8002828:	d10a      	bne.n	8002840 <_ftoa+0x270>
  }
  else if ((frac == 0U) || (frac & 1U)) {
 800282a:	6d3b      	ldr	r3, [r7, #80]	; 0x50
 800282c:	2b00      	cmp	r3, #0
 800282e:	d004      	beq.n	800283a <_ftoa+0x26a>
 8002830:	6d3b      	ldr	r3, [r7, #80]	; 0x50
 8002832:	f003 0301 	and.w	r3, r3, #1
 8002836:	2b00      	cmp	r3, #0
 8002838:	d002      	beq.n	8002840 <_ftoa+0x270>
    // if halfway, round up if odd OR if last digit is 0
    ++frac;
 800283a:	6d3b      	ldr	r3, [r7, #80]	; 0x50
 800283c:	3301      	adds	r3, #1
 800283e:	653b      	str	r3, [r7, #80]	; 0x50
  }

  if (prec == 0U) {
 8002840:	6f3b      	ldr	r3, [r7, #112]	; 0x70
 8002842:	2b00      	cmp	r3, #0
 8002844:	d136      	bne.n	80028b4 <_ftoa+0x2e4>
    diff = value - (double)whole;
 8002846:	6d78      	ldr	r0, [r7, #84]	; 0x54
 8002848:	f7fd fe1c 	bl	8000484 <__aeabi_i2d>
 800284c:	4603      	mov	r3, r0
 800284e:	460c      	mov	r4, r1
 8002850:	461a      	mov	r2, r3
 8002852:	4623      	mov	r3, r4
 8002854:	e9d7 0100 	ldrd	r0, r1, [r7]
 8002858:	f7fd fcc6 	bl	80001e8 <__aeabi_dsub>
 800285c:	4603      	mov	r3, r0
 800285e:	460c      	mov	r4, r1
 8002860:	e9c7 3410 	strd	r3, r4, [r7, #64]	; 0x40
    if ((!(diff < 0.5) || (diff > 0.5)) && (whole & 1)) {
 8002864:	2301      	movs	r3, #1
 8002866:	461c      	mov	r4, r3
 8002868:	f04f 0200 	mov.w	r2, #0
 800286c:	4b1e      	ldr	r3, [pc, #120]	; (80028e8 <_ftoa+0x318>)
 800286e:	e9d7 0110 	ldrd	r0, r1, [r7, #64]	; 0x40
 8002872:	f7fe f8e3 	bl	8000a3c <__aeabi_dcmplt>
 8002876:	4603      	mov	r3, r0
 8002878:	2b00      	cmp	r3, #0
 800287a:	d101      	bne.n	8002880 <_ftoa+0x2b0>
 800287c:	2300      	movs	r3, #0
 800287e:	461c      	mov	r4, r3
 8002880:	b2e3      	uxtb	r3, r4
 8002882:	f083 0301 	eor.w	r3, r3, #1
 8002886:	b2db      	uxtb	r3, r3
 8002888:	2b00      	cmp	r3, #0
 800288a:	d109      	bne.n	80028a0 <_ftoa+0x2d0>
 800288c:	f04f 0200 	mov.w	r2, #0
 8002890:	4b15      	ldr	r3, [pc, #84]	; (80028e8 <_ftoa+0x318>)
 8002892:	e9d7 0110 	ldrd	r0, r1, [r7, #64]	; 0x40
 8002896:	f7fe f8ef 	bl	8000a78 <__aeabi_dcmpgt>
 800289a:	4603      	mov	r3, r0
 800289c:	2b00      	cmp	r3, #0
 800289e:	d069      	beq.n	8002974 <_ftoa+0x3a4>
 80028a0:	6d7b      	ldr	r3, [r7, #84]	; 0x54
 80028a2:	f003 0301 	and.w	r3, r3, #1
 80028a6:	2b00      	cmp	r3, #0
 80028a8:	f000 8087 	beq.w	80029ba <_ftoa+0x3ea>
      // exactly 0.5 and ODD, then round up
      // 1.5 -> 2, but 2.5 -> 2
      ++whole;
 80028ac:	6d7b      	ldr	r3, [r7, #84]	; 0x54
 80028ae:	3301      	adds	r3, #1
 80028b0:	657b      	str	r3, [r7, #84]	; 0x54
 80028b2:	e082      	b.n	80029ba <_ftoa+0x3ea>
    }
  }
  else {
    unsigned int count = prec;
 80028b4:	6f3b      	ldr	r3, [r7, #112]	; 0x70
 80028b6:	64fb      	str	r3, [r7, #76]	; 0x4c
    // now do fractional part, as an unsigned number
    while (len < PRINTF_FTOA_BUFFER_SIZE) {
 80028b8:	e039      	b.n	800292e <_ftoa+0x35e>
 80028ba:	bf00      	nop
 80028bc:	f3af 8000 	nop.w
 80028c0:	00000000 	.word	0x00000000
 80028c4:	41cdcd65 	.word	0x41cdcd65
 80028c8:	00000000 	.word	0x00000000
 80028cc:	c1cdcd65 	.word	0xc1cdcd65
 80028d0:	08009cb0 	.word	0x08009cb0
 80028d4:	08009cb4 	.word	0x08009cb4
 80028d8:	7fefffff 	.word	0x7fefffff
 80028dc:	08009cbc 	.word	0x08009cbc
 80028e0:	08009cc4 	.word	0x08009cc4
 80028e4:	08009f60 	.word	0x08009f60
 80028e8:	3fe00000 	.word	0x3fe00000
      --count;
 80028ec:	6cfb      	ldr	r3, [r7, #76]	; 0x4c
 80028ee:	3b01      	subs	r3, #1
 80028f0:	64fb      	str	r3, [r7, #76]	; 0x4c
      buf[len++] = (char)(48U + (frac % 10U));
 80028f2:	6d39      	ldr	r1, [r7, #80]	; 0x50
 80028f4:	4b69      	ldr	r3, [pc, #420]	; (8002a9c <_ftoa+0x4cc>)
 80028f6:	fba3 2301 	umull	r2, r3, r3, r1
 80028fa:	08da      	lsrs	r2, r3, #3
 80028fc:	4613      	mov	r3, r2
 80028fe:	009b      	lsls	r3, r3, #2
 8002900:	4413      	add	r3, r2
 8002902:	005b      	lsls	r3, r3, #1
 8002904:	1aca      	subs	r2, r1, r3
 8002906:	b2d2      	uxtb	r2, r2
 8002908:	6dfb      	ldr	r3, [r7, #92]	; 0x5c
 800290a:	1c59      	adds	r1, r3, #1
 800290c:	65f9      	str	r1, [r7, #92]	; 0x5c
 800290e:	3230      	adds	r2, #48	; 0x30
 8002910:	b2d2      	uxtb	r2, r2
 8002912:	f107 0160 	add.w	r1, r7, #96	; 0x60
 8002916:	440b      	add	r3, r1
 8002918:	f803 2c48 	strb.w	r2, [r3, #-72]
      if (!(frac /= 10U)) {
 800291c:	6d3b      	ldr	r3, [r7, #80]	; 0x50
 800291e:	4a5f      	ldr	r2, [pc, #380]	; (8002a9c <_ftoa+0x4cc>)
 8002920:	fba2 2303 	umull	r2, r3, r2, r3
 8002924:	08db      	lsrs	r3, r3, #3
 8002926:	653b      	str	r3, [r7, #80]	; 0x50
 8002928:	6d3b      	ldr	r3, [r7, #80]	; 0x50
 800292a:	2b00      	cmp	r3, #0
 800292c:	d003      	beq.n	8002936 <_ftoa+0x366>
    while (len < PRINTF_FTOA_BUFFER_SIZE) {
 800292e:	6dfb      	ldr	r3, [r7, #92]	; 0x5c
 8002930:	2b1f      	cmp	r3, #31
 8002932:	d9db      	bls.n	80028ec <_ftoa+0x31c>
 8002934:	e00a      	b.n	800294c <_ftoa+0x37c>
        break;
 8002936:	bf00      	nop
      }
    }
    // add extra 0s
    while ((len < PRINTF_FTOA_BUFFER_SIZE) && (count-- > 0U)) {
 8002938:	e008      	b.n	800294c <_ftoa+0x37c>
      buf[len++] = '0';
 800293a:	6dfb      	ldr	r3, [r7, #92]	; 0x5c
 800293c:	1c5a      	adds	r2, r3, #1
 800293e:	65fa      	str	r2, [r7, #92]	; 0x5c
 8002940:	f107 0260 	add.w	r2, r7, #96	; 0x60
 8002944:	4413      	add	r3, r2
 8002946:	2230      	movs	r2, #48	; 0x30
 8002948:	f803 2c48 	strb.w	r2, [r3, #-72]
    while ((len < PRINTF_FTOA_BUFFER_SIZE) && (count-- > 0U)) {
 800294c:	6dfb      	ldr	r3, [r7, #92]	; 0x5c
 800294e:	2b1f      	cmp	r3, #31
 8002950:	d804      	bhi.n	800295c <_ftoa+0x38c>
 8002952:	6cfb      	ldr	r3, [r7, #76]	; 0x4c
 8002954:	1e5a      	subs	r2, r3, #1
 8002956:	64fa      	str	r2, [r7, #76]	; 0x4c
 8002958:	2b00      	cmp	r3, #0
 800295a:	d1ee      	bne.n	800293a <_ftoa+0x36a>
    }
    if (len < PRINTF_FTOA_BUFFER_SIZE) {
 800295c:	6dfb      	ldr	r3, [r7, #92]	; 0x5c
 800295e:	2b1f      	cmp	r3, #31
 8002960:	d82b      	bhi.n	80029ba <_ftoa+0x3ea>
      // add decimal
      buf[len++] = '.';
 8002962:	6dfb      	ldr	r3, [r7, #92]	; 0x5c
 8002964:	1c5a      	adds	r2, r3, #1
 8002966:	65fa      	str	r2, [r7, #92]	; 0x5c
 8002968:	f107 0260 	add.w	r2, r7, #96	; 0x60
 800296c:	4413      	add	r3, r2
 800296e:	222e      	movs	r2, #46	; 0x2e
 8002970:	f803 2c48 	strb.w	r2, [r3, #-72]
    }
  }

  // do whole part, number is reversed
  while (len < PRINTF_FTOA_BUFFER_SIZE) {
 8002974:	e021      	b.n	80029ba <_ftoa+0x3ea>
    buf[len++] = (char)(48 + (whole % 10));
 8002976:	6d7a      	ldr	r2, [r7, #84]	; 0x54
 8002978:	4b49      	ldr	r3, [pc, #292]	; (8002aa0 <_ftoa+0x4d0>)
 800297a:	fb83 1302 	smull	r1, r3, r3, r2
 800297e:	1099      	asrs	r1, r3, #2
 8002980:	17d3      	asrs	r3, r2, #31
 8002982:	1ac9      	subs	r1, r1, r3
 8002984:	460b      	mov	r3, r1
 8002986:	009b      	lsls	r3, r3, #2
 8002988:	440b      	add	r3, r1
 800298a:	005b      	lsls	r3, r3, #1
 800298c:	1ad1      	subs	r1, r2, r3
 800298e:	b2ca      	uxtb	r2, r1
 8002990:	6dfb      	ldr	r3, [r7, #92]	; 0x5c
 8002992:	1c59      	adds	r1, r3, #1
 8002994:	65f9      	str	r1, [r7, #92]	; 0x5c
 8002996:	3230      	adds	r2, #48	; 0x30
 8002998:	b2d2      	uxtb	r2, r2
 800299a:	f107 0160 	add.w	r1, r7, #96	; 0x60
 800299e:	440b      	add	r3, r1
 80029a0:	f803 2c48 	strb.w	r2, [r3, #-72]
    if (!(whole /= 10)) {
 80029a4:	6d7b      	ldr	r3, [r7, #84]	; 0x54
 80029a6:	4a3e      	ldr	r2, [pc, #248]	; (8002aa0 <_ftoa+0x4d0>)
 80029a8:	fb82 1203 	smull	r1, r2, r2, r3
 80029ac:	1092      	asrs	r2, r2, #2
 80029ae:	17db      	asrs	r3, r3, #31
 80029b0:	1ad3      	subs	r3, r2, r3
 80029b2:	657b      	str	r3, [r7, #84]	; 0x54
 80029b4:	6d7b      	ldr	r3, [r7, #84]	; 0x54
 80029b6:	2b00      	cmp	r3, #0
 80029b8:	d003      	beq.n	80029c2 <_ftoa+0x3f2>
  while (len < PRINTF_FTOA_BUFFER_SIZE) {
 80029ba:	6dfb      	ldr	r3, [r7, #92]	; 0x5c
 80029bc:	2b1f      	cmp	r3, #31
 80029be:	d9da      	bls.n	8002976 <_ftoa+0x3a6>
 80029c0:	e000      	b.n	80029c4 <_ftoa+0x3f4>
      break;
 80029c2:	bf00      	nop
    }
  }

  // pad leading zeros
  if (!(flags & FLAGS_LEFT) && (flags & FLAGS_ZEROPAD)) {
 80029c4:	6fbb      	ldr	r3, [r7, #120]	; 0x78
 80029c6:	f003 0302 	and.w	r3, r3, #2
 80029ca:	2b00      	cmp	r3, #0
 80029cc:	d124      	bne.n	8002a18 <_ftoa+0x448>
 80029ce:	6fbb      	ldr	r3, [r7, #120]	; 0x78
 80029d0:	f003 0301 	and.w	r3, r3, #1
 80029d4:	2b00      	cmp	r3, #0
 80029d6:	d01f      	beq.n	8002a18 <_ftoa+0x448>
    if (width && (negative || (flags & (FLAGS_PLUS | FLAGS_SPACE)))) {
 80029d8:	6f7b      	ldr	r3, [r7, #116]	; 0x74
 80029da:	2b00      	cmp	r3, #0
 80029dc:	d015      	beq.n	8002a0a <_ftoa+0x43a>
 80029de:	f897 305b 	ldrb.w	r3, [r7, #91]	; 0x5b
 80029e2:	2b00      	cmp	r3, #0
 80029e4:	d104      	bne.n	80029f0 <_ftoa+0x420>
 80029e6:	6fbb      	ldr	r3, [r7, #120]	; 0x78
 80029e8:	f003 030c 	and.w	r3, r3, #12
 80029ec:	2b00      	cmp	r3, #0
 80029ee:	d00c      	beq.n	8002a0a <_ftoa+0x43a>
      width--;
 80029f0:	6f7b      	ldr	r3, [r7, #116]	; 0x74
 80029f2:	3b01      	subs	r3, #1
 80029f4:	677b      	str	r3, [r7, #116]	; 0x74
    }
    while ((len < width) && (len < PRINTF_FTOA_BUFFER_SIZE)) {
 80029f6:	e008      	b.n	8002a0a <_ftoa+0x43a>
      buf[len++] = '0';
 80029f8:	6dfb      	ldr	r3, [r7, #92]	; 0x5c
 80029fa:	1c5a      	adds	r2, r3, #1
 80029fc:	65fa      	str	r2, [r7, #92]	; 0x5c
 80029fe:	f107 0260 	add.w	r2, r7, #96	; 0x60
 8002a02:	4413      	add	r3, r2
 8002a04:	2230      	movs	r2, #48	; 0x30
 8002a06:	f803 2c48 	strb.w	r2, [r3, #-72]
    while ((len < width) && (len < PRINTF_FTOA_BUFFER_SIZE)) {
 8002a0a:	6dfa      	ldr	r2, [r7, #92]	; 0x5c
 8002a0c:	6f7b      	ldr	r3, [r7, #116]	; 0x74
 8002a0e:	429a      	cmp	r2, r3
 8002a10:	d202      	bcs.n	8002a18 <_ftoa+0x448>
 8002a12:	6dfb      	ldr	r3, [r7, #92]	; 0x5c
 8002a14:	2b1f      	cmp	r3, #31
 8002a16:	d9ef      	bls.n	80029f8 <_ftoa+0x428>
    }
  }

  if (len < PRINTF_FTOA_BUFFER_SIZE) {
 8002a18:	6dfb      	ldr	r3, [r7, #92]	; 0x5c
 8002a1a:	2b1f      	cmp	r3, #31
 8002a1c:	d82a      	bhi.n	8002a74 <_ftoa+0x4a4>
    if (negative) {
 8002a1e:	f897 305b 	ldrb.w	r3, [r7, #91]	; 0x5b
 8002a22:	2b00      	cmp	r3, #0
 8002a24:	d009      	beq.n	8002a3a <_ftoa+0x46a>
      buf[len++] = '-';
 8002a26:	6dfb      	ldr	r3, [r7, #92]	; 0x5c
 8002a28:	1c5a      	adds	r2, r3, #1
 8002a2a:	65fa      	str	r2, [r7, #92]	; 0x5c
 8002a2c:	f107 0260 	add.w	r2, r7, #96	; 0x60
 8002a30:	4413      	add	r3, r2
 8002a32:	222d      	movs	r2, #45	; 0x2d
 8002a34:	f803 2c48 	strb.w	r2, [r3, #-72]
 8002a38:	e01c      	b.n	8002a74 <_ftoa+0x4a4>
    }
    else if (flags & FLAGS_PLUS) {
 8002a3a:	6fbb      	ldr	r3, [r7, #120]	; 0x78
 8002a3c:	f003 0304 	and.w	r3, r3, #4
 8002a40:	2b00      	cmp	r3, #0
 8002a42:	d009      	beq.n	8002a58 <_ftoa+0x488>
      buf[len++] = '+';  // ignore the space if the '+' exists
 8002a44:	6dfb      	ldr	r3, [r7, #92]	; 0x5c
 8002a46:	1c5a      	adds	r2, r3, #1
 8002a48:	65fa      	str	r2, [r7, #92]	; 0x5c
 8002a4a:	f107 0260 	add.w	r2, r7, #96	; 0x60
